:020000040000FA
:100000000EEF00F0FFFFFFFFE4EF0CF0FFFFFFFF3C
:10001000FFFFFFFFFFFFFFFF9CEF17F045EF0BF027
:10002000D66F91D04D0EC26FFA0EC36F0B0EC46F18
:10003000010EC56F020EC66F3F0EC76F000EC86F70
:10004000010EC96F000ECA6F000ECB6F000ECC6F91
:10005000000ECD6FF6C0CEF0F8ECFEF012004D0EA3
:10006000C26FFA0EC36F0B0EC46F010EC56F030E85
:10007000C66F3F0EC76F000EC86F010EC96F000E2E
:10008000CA6F000ECB6F000ECC6F000ECD6FF6C0A6
:10009000CEF0F8ECFEF012004D0EC26FFA0EC36FF8
:1000A0000B0EC46F010EC56F040EC66F3F0EC76FF7
:1000B000000EC86F010EC96F000ECA6F000ECB6F25
:1000C000000ECC6F000ECD6FF6C0CEF0F8ECFEF057
:1000D00012004D0EC26FFA0EC36F0B0EC46F010EED
:1000E000C56F050EC66F3F0EC76F000EC86F010EBD
:1000F000C96F000ECA6F000ECB6F000ECC6F000EE2
:10010000CD6FF6C0CEF0F8ECFEF012004D0EC26FCF
:10011000FA0EC36F0B0EC46F010EC56F000EC66FD3
:100120003F0EC76F000EC86F010EC96F000ECA6F79
:10013000000ECB6F000ECC6F000ECD6FF6C0CEF070
:10014000F8ECFEF012000001D651000AD8B4C1D775
:10015000210AD8B4A1D7630AD8B481D7260AD8B463
:1001600061D7D4D7C46F0001C451D8A4BFAF1AD08F
:10017000BCC0C0F0BDC0C1F0BEC0C2F0BFC0C3F0C3
:10018000C01FC11FC21FC31FC02B000EC123C2232B
:10019000C323C0C0C6F0C1C0C7F0C2C0C8F0C3C04E
:1001A000C9F008D0BCC0C6F0BDC0C7F0BEC0C8F022
:1001B000BFC0C9F0BC51BD11BE11BF11D8A409D038
:1001C000000EBC6F000EBD6F000EBE6F000EBF6F45
:1001D0001200960EC56F06D0C52BD890C933C83310
:1001E000C733C633000EC615C06F000EC715C16FEA
:1001F000000EC815C26FFE0EC915C36FC051C111E4
:10020000C211C311D8B40DD0E7D7C52B010EC62734
:10021000000EC723C823C923D890C933C833C733B6
:10022000C633000EC615C06F000EC715C16F000E95
:10023000C815C26FFF0EC915C36FC051C111C211DD
:10024000C311D8B407D0E1D7C507D890C637C73790
:10025000C837C937C8BF03D0020EC561F5D7C5A1DD
:10026000C89FD890C533C5C0C0F0C16BC26BC36B0B
:10027000C0C0C3F0C26BC16BC06BC051C613C151CB
:10028000C713C251C813C351C913C451D8A4BFAFB7
:1002900001D0C98FC6C0BCF0C7C0BDF0C8C0BEF099
:1002A000C9C0BFF01200000E0001D06F000ECF6F6A
:1002B0000301E751FC0B0001D06F0301E751030B71
:1002C0000001CF6F82D04E04D8A41200D0C0C9F074
:1002D000230EE8ECF8F0010EAF6F000E0101BA6FCB
:1002E000010EBB6F000E676F000E656F0001860583
:1002F000D8A412000101E651D8A412009B2B1200D1
:10030000D0514118D8A406D0010E406E000E010154
:10031000656F02D0000E406E4D04D8A40AD0405044
:10032000D8A407D0D0C041F0010E406E010E0101EB
:10033000666F4E50D8A41200420E0001B519D8A421
:1003400012004004D8A409D0420EB2651200470E34
:10035000B2611200E9EC16F012000101652B040EE7
:1003600065651200000E656F000E406E000E020102
:10037000986F000E0001AF6F010E0101AC6F000E0F
:10038000676F470E0001B56FB551B5253D016F6F21
:10039000FE0E706F010E0101B16F1200D0A51200A8
:1003A0004D04D8A412004004D8A41200D0C0CDF04F
:1003B000700ECD17D8B41200D0390F0B070B400FB9
:1003C0000101B06FB0C1B2F0C5D7CF51000AD8B4A7
:1003D0007AD7010AD8B494D7030AD8B4DFD7010A70
:1003E0001200C2C0C9F0C3C0C8F0C15104E1020E7E
:1003F000C05DD8A03BD0C0B139D05A0EC419D8A422
:1004000035D0C0C0BCF0C1C0BDF027EC18F0000171
:10041000C919D8B414D0C0C0BCF0C1C0BDF0C9C0A7
:10042000BEF05BEC14F0FF0E0001C025BC6FFF0EA8
:10043000C121BD6FC4C0BEF05BEC14F01200FF0E12
:10044000C025BC6FFF0EC121BD6F27EC18F0000165
:10045000C419D8B41200FF0EC025BC6FFF0EC12115
:10046000BD6FC4C0BEF05BEC14F01200C15104E1DA
:10047000210EC05DD8A012005B0EC419D8A41200D2
:10048000010EC025BC6F000EC121BD6F27EC18F016
:100490000001C56F080EC527C0C0BCF0C1C0BDF0CB
:1004A00027EC18F00001C66FC76BC52B03D0D8909E
:1004B000C637C737C52FFBD70001C251C61904E1A3
:1004C000C351C719D8B41FD0C0C0BCF0C1C0BDF063
:1004D000C8C0BEF05BEC14F0010E0001C025BC6F7B
:1004E000000EC121BD6FC9C0BEF05BEC14F0FF0E61
:1004F0000001C025BC6FFF0EC121BD6FC4C0BEF09E
:100500005BEC14F01200FF0EC025BC6FFF0EC12182
:10051000BD6F27EC18F09BD7000ED06FC9C0C2F09A
:10052000CAC0C3F0030EC56FE80EC46F2DEC13F004
:10053000C251D26FD2C0BCF0BD6BFC0EBF6F180EA3
:10054000BE6FFEEC16F0C951BC25C26FCA51BD2169
:10055000C36F000EC56F640EC46F2DEC13F0C25153
:10056000D16FD2C0BCF0BD6BFC0EBF6F180EBE6F5A
:10057000FEEC16F0BCC0CCF0BDC0CDF0D1C0BCF0DC
:10058000BD6BFF0EBF6F9C0EBE6FFEEC16F0BC5134
:10059000CC27BD51CD23C951CC25C26FCA51CD2125
:1005A000C36F000EC56F0A0EC46F2DEC13F0C2515D
:1005B000CF6FD251180D6F00CCFFCCF0D1519C0DF4
:1005C0006F00CCFFCDF0CF51F60DF350CD25CC25EB
:1005D000C925CE6F540ECB19D8B404D0740ECB19E4
:1005E000D8A403D0D2C0D0F01FD0480ECB19D8B4B5
:1005F00004D0680ECB19D8A403D0D1C0D0F014D049
:100600005A0ECB19D8B404D07A0ECB19D8A403D083
:10061000CFC0D0F009D0450ECB19D8B403D0650EA9
:10062000CB19D8B4CEC0D0F0D0511200D76F020E83
:100630000101EB6FD7C0ECF15AD0CCC0EDF1030E45
:100640002DD0CC51CD25D56FD5290101ED6FCEC070
:10065000EEF1040E0001D86FCD05D8A404D0D0C0AF
:10066000EFF1050ED86F020ECD19D8A406D0CFC079
:10067000EFF1D0C0F0F1060ED86F030ECD19D8A45B
:100680004AD0CFC0EFF1D0C0F0F1D1C0F1F1070EE8
:1006900005D0000E0101ED6F030E27D0D86F3BD0BF
:1006A000010E0101ED6FD0C0EEF1040E0001D86F14
:1006B000D105D8A030D00101ED2BD1C0EFF1050E4E
:1006C00014D0010EE7D7020E0101ED6FD2C0EEF19A
:1006D000D3C0EFF1050E0001D86FD405D8A01BD010
:1006E0000101ED2BD4C0F0F1060E0001D7D70001B7
:1006F000D751000AD8B4A1D7010AD8B4A2D7040AA6
:10070000D8B4C7D70D0AD8B4CBD7010AD8B4DBD731
:10071000180AD8B4D6D7CAC0C1F0CBC0C2F0EDC158
:10072000C3F0D8C0C4F012EC0AF0D66FD6C0BCF04B
:100730000101EB5163EC17F01200216E71D04D04F2
:10074000D8A412005504D8A414D0000E0201AF6F33
:10075000000EB06F3E0EB16F000EB26F000EB36FA1
:10076000AF0E1E6E020E1F6E050E206EAEEC15F063
:1007700013D0000E0201C46F000EC56F3E0EC66F8F
:10078000000EC76F000EC86FC40E1E6E020E1F6EE5
:10079000050E206EAEEC15F0050E0201886F100EEE
:1007A000876F12004D04D8A4120018C237F119C285
:1007B00036F136C159F037C15AF0010E0101B36F5D
:1007C000010E4E6E5504D8A414D05AC0AFF259C0D1
:1007D000B0F23F0E0201B16F59C0B2F2000EB36F1A
:1007E000AF0E1E6E020E1F6E050E206EAEEC15F0E3
:1007F00013D05AC0C4F259C0C5F23F0E0201C66FF1
:1008000059C0C7F2000EC86FC40E1E6E020E1F6ED6
:10081000050E206EAEEC15F0050E0201886F120079
:100820002150220AD8B41200010AD8B412000D0ACD
:10083000D8B485D7010AD8A41200B4D70101E905BC
:10084000D8A44ED079C2EDF07AC2EEF05AEC12F094
:10085000EDC00CF1EEC00DF1010E01015E6F5D51B6
:10086000D8A40CD0000EBE6F000EBD6F0CC1BCF042
:100870000DC1BDF085EC12F0010113D0010EBE6F69
:10088000270EBD6523D0000EBD6F0DD0000E09D020
:10089000640E07D0500E05D03C0E03D0280E01D0B8
:1008A000140E5F6F13D06051000AD8B4F9D7140A40
:1008B000D8B4F4D73C0AD8B4EFD7140AD8B4EAD7DE
:1008C0006C0AD8B4E5D7340AD8B4E0D760515F19C0
:1008D000D8B404D05FC160F1010E776F000EE96FEC
:1008E0000001B405D8B403D0AD05D8A406D0010EDC
:1008F00001015D6F000E5C6F1200800E01010C5D46
:100900000C0E0D59D8B014D05D51D8A4120050501F
:10091000D8A412000201465104E1650E455DD8A03D
:1009200004D0010E01015C6F1200454B462B1200F2
:10093000000E5D6F000E5C6F12000101EA05D8A485
:1009400012007DC2EDF07EC2EEF02FEC12F0EDC091
:100950001AF1EEC01BF1010E01017E6F1AC1EFF01A
:100960001BC1F0F01AC151F21BC152F2A10E0001DD
:10097000EF5D0F0EF059D8A002D0000E4FD0B90E87
:10098000EF5D0B0EF059D8B0F8D7D10EEF5D070E22
:10099000F059D8A002D0640E41D0E90EEF5D030EED
:1009A000F059D8A002D05A0E39D0590EEF5D020E80
:1009B000F059D8A002D0500E31D0C30EEF5D010E19
:1009C000F059D8A002D04B0E29D02D0EEF5D010EAC
:1009D000F059D8A002D0400E21D0F05104E1A10E70
:1009E000EF5DD8A002D0320E19D0F05104E16F0EA5
:1009F000EF5DD8A002D0300E11D0F05104E15B0EB3
:100A0000EF5DD8A002D0200E09D0F05104E1470ECE
:100A1000EF5DD8A002D0190E01D0100E4A6E010170
:100A2000A605D8A405D02F0E4A6402D0000E4A6E47
:100A3000000EEA6F1200000EE76F000EE86F5CD048
:100A4000600EC26FE50EC36F070EC46F020EC56F56
:100A5000E851D625E06F000ED721E16F600083F3E7
:100A6000F6FF600087F3F7FF000EF86E0800F55000
:100A7000E00FC66FE751FC0D6F00CCFFE2F0E851CC
:100A8000080DF350E225D925C76FDAC0C8F0DBC0E6
:100A9000C9F0DCC0CAF0DDC0CBF0DEC0CCF0DFC0F6
:100AA000CDF0F6C0CEF0F8ECFEF0E851D625E06FC0
:100AB000000ED721E16F600083F3F6FF600087F33B
:100AC000F7FF000EF86E0800F550490AD8B412D0AE
:100AD000E851D625E06F000ED721E16F600083F367
:100AE000F6FF600087F3F7FF000EF86E0800F55080
:100AF000690AD8B4E72BE82BFF0EE06FFF0EE16F19
:100B0000D851E26FE36BE051E227E151E323E85172
:100B1000E46FE56BE251E45DE551800AE66FE35175
:100B2000800AE659D8B012008BD71C6E020E010164
:100B3000EB6F1CC0ECF14ED011C0EDF1030E48D0AC
:100B4000115012241A6E1A28ED6F13C0EEF1040E24
:100B50001D6E1204D8A404D015C0EFF1050E1D6E51
:100B6000020E1218D8A406D014C0EFF115C0F0F18F
:100B7000060E1D6E030E1218D8A43FD014C0EFF15C
:100B800015C0F0F116C0F1F1070E22D0000EED6F86
:100B9000D5D7010EED6F15C0EEF1040E1D6E1604D3
:100BA000D8A02BD0ED2B16C0EFF1050E11D0010E01
:100BB000EED7020EED6F17C0EEF118C0EFF1050E83
:100BC0001D6E1904D8A019D0ED2B19C0F0F1060E36
:100BD0001D6E13D01C50000AD8B4AED7010AD8B489
:100BE000AFD7040AD8B4D2D70D0AD8B4D2D7010AE5
:100BF000D8B4DFD7180AD8B4DAD70FC006F010C0BF
:100C000007F0EDC108F01DC009F063EC0AF01B6E9F
:100C10001BC001F00101EB51E5EC17F01200216E51
:100C2000050E0201176506D00C0E1C6103D01CC214
:100C300000F202D0000E006F0051D8B45ED0010E59
:100C4000226E10D01C0E2224D96EDA6A020EDA222D
:100C5000000E2224E16EE26A020EE2226F007FFFA4
:100C6000E7FF222A2250005DD8B0ECD7010E010127
:100C7000616F43D04C50D8A44C065504D8A413D06F
:100C80005AC0AFF259C0B0F2310E0201B16F34C197
:100C9000B2F2AF0E1E6E020E1F6EB351050F206E24
:100CA000AEEC15F012D05AC0C4F259C0C5F2310EE4
:100CB0000201C66F34C1C7F2C40E1E6E020E1F6E53
:100CC000C851050F206EAEEC15F05450D8B411D0B9
:100CD0000F0E0201CD17CDC2B8F23F0EC9171C0E80
:100CE000CA171C0ECB173F0EB4171C0EB5171C0EDF
:100CF000B6170B0E0201886F12002150210AD8B4DA
:100D0000B9D7030AD8B41200010A1200000E00017C
:100D1000C06F000EC16F010EC26FC251020D2A0ECC
:100D2000F324D96E020EF420DA6EBC51DE1807E10E
:100D3000BD51DE18D8A403D0010EC06F11D0C2512E
:100D4000020D2A0EF324D96E020EF420DA6EDE5064
:100D5000DE10D8B4C2C0C1F0C22B050EC265DDD70B
:100D6000C051D8A41200C151D8B434D0C151020D21
:100D70002A0EF324D96E020EF420DA6E6000F3F22C
:100D8000DEFF6000F7F2DDFFC1C054F11200BCC00D
:100D90002EF2BDC02FF2020E546F1200BCC030F212
:100DA000BDC031F2030E546F1200BCC032F2BDC0A0
:100DB00033F2040E546F1200BCC034F2BDC035F2E1
:100DC000050E546F1200BCC02CF2BDC02DF2010EF6
:100DD000546F120001015451010AD8B4D8D7030A44
:100DE000D8B4DCD7010AD8B4E0D7070AD8B4E4D71E
:100DF000010AD8A41200E7D70001BD6F0101E50583
:100E0000D8B433D0000ED36F000E0001BE6F0ED0E9
:100E1000BE51600FD96EDA6ADB0EBE25E16EE26A62
:100E2000030EE2226F007FFFE7FFBE2BBD51BE5DC8
:100E3000D8A0EED75BC0BCF0030EBC17D8A45B886B
:100E4000040E5418D8A402D0010E546E040E531888
:100E5000D8A402D0010E536E040E5218D8A402D0AA
:100E6000010E526E010E0101D36F020EE519D8B4C6
:100E70001200000E556E000E0001BF6F10D0DA0E8A
:100E8000BF25D96EDA6A030EDA22CE0EBF25E16ED7
:100E9000E26A030EE2226F007FFFE7FFBF2BBF5124
:100EA000BD5DD8B0ECD75BC0BCF0030EBC17D8A4B6
:100EB0005B8A5404D8A402D0020E546E5304D8A402
:100EC00002D0020E536E5204D8A402D0020E526E0B
:100ED000010E556E1200BC6F05D0000E01D0010E40
:100EE000BD6F66D00001BC51000AD8B4F6D70A0A1B
:100EF000D8B4F3D7010AD8B4F0D7070AD8B4EDD7DD
:100F0000010AD8B4EAD7030AD8B4E7D7010AD8B49B
:100F1000E4D71F0AD8B4E1D7010AD8B4DED70F0A44
:100F2000D8B4DBD7010AD8B4D8D73F0AD8B4D5D7BC
:100F3000010AD8B4D2D7030AD8B4CFD7010AD8B49B
:100F4000CCD70B0AD8B4C9D7010AD8B4C6D7030A7C
:100F5000D8B4C3D7010AD8B4C0D7070AD8B4BDD70C
:100F6000010AD8B4BAD7030AD8B4B7D7010AD8B49B
:100F7000B4D71C0AD8B4B1D7070AD8B4AED7010A7F
:100F8000D8B4ABD70C0AD8B4A8D7780AD8B4A5D7A8
:100F9000030AD8B4A2D7010AD8B49FD7080AD8B494
:100FA0009CD7070AD8B499D7010AD8B496D797D74F
:100FB000BD511200C76F0001C005D8A402D01E0E9B
:100FC000BE27010ECA6F5CD0BB98BB9ACA51BF2521
:100FD000AF0F52EC18F0BB8A0001C005D8A40FD0A7
:100FE000BB98BB9ABE510F0B52EC18F0BB8ABB9A50
:100FF0000001BE390F0B100F52EC18F00ED0BB9849
:10100000BB9ABE390F0B100F52EC18F0BB8ABB9A7B
:101010000001BE510F0B52EC18F0BB8ABB88000ECA
:101020000001C96F28D0000EC86FCA05D8B4C881A6
:10103000BD51CA19D8B4C88FC951D8B414D0C95138
:10104000C16FC26BFF0EC36FFF0EC46FC751C56F78
:10105000C66BC351C527C451C623C151C51904E18C
:10106000C251C619D8B4C869BB9AC85152EC18F01D
:10107000BB8A0001C92BC751C95DD8A0D4D7CA2BE0
:10108000CA51BD5DD8B0A0D7BB8812004305D8A413
:1010900018D07E0E0001D66FFF0ED76F0A0ED86FE4
:1010A000000ED96F070EDA6F000EDB6F000EDC6FDB
:1010B000000EDD6F000EDE6F010EDF6F8DECE6F0CF
:1010C00012004805D8A418D0B30E0001D66FFF0E49
:1010D000D76F070ED86F000ED96F070EDA6F000EAC
:1010E000DB6F000EDC6F000EDD6F000EDE6F010E99
:1010F000DF6F8DECE6F012004105D8A418D0740E15
:101100000001D66FFF0ED76F0A0ED86F000ED96F91
:10111000070EDA6F000EDB6F000EDC6F000EDD6F66
:10112000000EDE6F010EDF6F8DECE6F01200F50EA3
:101130000001D66FFE0ED76F0D0ED86F000ED96F5F
:10114000070EDA6F000EDB6F000EDC6F000EDD6F36
:10115000000EDE6F000EDF6F8DECE6F01200E5355D
:10116000E635EC6FEC51D8A409D0000EE36F000E09
:10117000E46F000EE56F000EE66F1200E3C0E7F0CB
:10118000E4C0E8F0E5C0E9F0E6C0EAF0200E05D0E2
:10119000D890EA33E933E833E733E82EF9D7E7515B
:1011A000EB6FE58FFF0EE317FF0EE417FF0EE51759
:1011B000000EE617960EEC5FECAF0DD0EC51800AF6
:1011C000970FD8A0D2D7D890E633E533E433E33392
:1011D000EC3FF9D70DD01F0EEC6507D0C6D7D890DD
:1011E000E337E437E537E637EC07EC51D8A4F7D717
:1011F000EB51D8B408D0E61FE51FE41FE36D000EE5
:10120000E423E523E623E3C0E3F0E4C0E4F0E5C033
:10121000E5F0E6C0E6F01200040EBE6E000EBD6EF4
:10122000010EBA6E500EBB6E980EBC6E030EC66EEB
:10123000FE0EC26E030EC36E270EC46EFC0EC56E8C
:101240000C0E3A01706F000E606F040E506F010EAD
:10125000806F020E406FF00E716F040E816F000EF2
:10126000516FFC0E416F070E616F040E826F000E0E
:10127000426F000E526F180E626F030E726F436959
:10128000536963697369070E836F180EE36F210E4C
:10129000136F220E146F090EE56F130EE16F190E16
:1012A000E46F0B0EDE6F140EE26F040ED96F1F0E8B
:1012B0000A6F1E0E0B6F230E186F240E196F050E8A
:1012C000DA6F130E166F160EDF6F12004E04D8A4DD
:1012D00013D05450D8A410D05350D8A40DD052508D
:1012E000D8A40AD0020EC96F230EA6ECE2F00301C7
:1012F000DA6FDA51FCEC06F00101CF05D8A405D075
:1013000053EC01F0000E0101CF6F4D04D8A415D0AD
:101310006751D8A412D0CE05D8A40FD0410E000139
:10132000B519D8B40AD0010EC06F410E45EC10F0CB
:10133000030E416E000E0001B26F0101AD05D8A48D
:101340001200470E0001B56FB551B5253D016F6F15
:10135000FE0E706F010E0101B16F000E0201986F59
:10136000000E0001AF6F010E0101AC6F000EAD6FFA
:10137000000E4D6E000E676F1200BD6F000E000173
:10138000BF6FBB98BB9ABF51B00F52EC18F0BB8A2D
:101390000001BD05D8A40AD0BB9A0E0E52EC18F07D
:1013A000BB8ABB9A110E52EC18F009D0BB9A000E02
:1013B00052EC18F0BB8ABB9A100E52EC18F0BB8AA4
:1013C000BB88000E0001BE6FBB9A000E52EC18F0F5
:1013D000BB8A0001BE2B650EBE65F6D7BF2B070E7C
:1013E000BF65CFD7BB98BB9AB00E52EC18F0BB8A42
:1013F0000001BD05D8A40AD0BB9A0E0E52EC18F01D
:10140000BB8ABB9A110E52EC18F009D0BB9A000EA1
:1014100052EC18F0BB8ABB9A100E52EC18F0BB8A43
:10142000BB881200000EC96F2CD0C951C125C56FF1
:10143000000EC221C66F600017F3F6FF60001BF3B9
:10144000F7FF000EF86EEB0EC76F010EC86FC951A3
:10145000C727000EC823C451C725D96E000EC82166
:10146000DA6E1F0EF76403D00800F55007D06F0046
:10147000DBFFE1FF6F00DFFFE2FFE750DF6E0001FF
:10148000C92BC351C95DD8A0D0D7EB0EBC6F010EDC
:10149000BD6FC951C425BE6F13EC17F0C56FEB0EBD
:1014A000C66F010EC76FC951C627000EC723C451AE
:1014B000C625D96E000EC721DA6E600017F3DFFF74
:1014C000C951C4251200000E0E6E2BD00E500624FA
:1014D0000A6E000E07200B6E60002BF0F6FF600016
:1014E0002FF0F7FF000EF86EEB0E0C6E010E0D6E76
:1014F0000E500C26000E0D2209500C24D96E000E41
:101500000D20DA6E1F0EF76403D00800F55007D0E7
:101510006F00DBFFE1FF6F00DFFFE2FFE750DF6EF0
:101520000E2A08500E5CD8A0D1D7EB0E016E010E2A
:10153000026E0E500924036E4FEC17F00A6EEB0E8C
:101540000B6E010E0C6E0E500B26000E0C22095075
:101550000B24D96E000E0C20DA6E60002BF0DFFF3A
:101560000E5009241200BE6F47C0BDF0180E0001D6
:10157000BD17D8B41DD047380F0B010B491A4904C9
:10158000D8A40CD04850FF0ABD6FBE51BD5DD8A095
:101590002BD04850BE2729D01F0E05D04850BE5D25
:1015A000D8B003D0000EBE6F24D04850BE5F21D00B
:1015B00047A41FD04904D8A40FD0BC51D8B4E2D757
:1015C000BE51D8A403D0000E0101596F485000014C
:1015D000BE5DD8A0E7D7E9D7BC51D8A4D3D7BE51B8
:1015E000D8A4F4D7010EF0D7BE691F0EBE6501D096
:1015F000D3D7000E486EBE511200BE6F4904D8A466
:1016000036D04850FF0A0001BD6FBE51BD5DD8B055
:1016100002D0BE6912D04850BE270FD0050EBE655D
:1016200030D0050E2AD0030EBE652BD0030E25D078
:10163000020EBE6526D0020E20D0BC51640AD8B47A
:10164000EDD70A0AD8B4EFD7010AD8B4ECD7150AF7
:10165000D8B4E9D7060AD8B4EBD7FE0AD8B4E8D78D
:10166000010AD8B4E0D7070AD8B4DDD7D7D700012C
:10167000BE51485CD8A003D0010EBE6F02D04850C6
:10168000BE5F000E486EBE5112006C0EF66E300E3C
:10169000F76E000EF86E00EEDBF210EE1CF00900A3
:1016A0006F00D7FFEEFFE550E150F9E1FE0EF66E58
:1016B000FF0EF76E010EF86E09006F00D4FFF6F012
:1016C00000EE00F3F20EEE6AE806FDE100EE00F235
:1016D000DB0EEE6AE806FDE100EE00F110EE00F12F
:1016E000EE6AE550E150FCE1E250FAE100EE60F014
:1016F000590EEE6AE806FDE100EE2FF02D0EEE6ABF
:10170000E806FDE1080ED56E000ED66E000ED76E0F
:10171000000159EFA9F09397A40E0001BC6F1F0EB2
:10172000BD6F000EBE6F9FEC18F039019399AC0E9F
:101730000001BC6F2A0EBD6F000EBE6F98EC18F052
:10174000000E3D01EC6F000EED6F000EEE6F000E0F
:10175000EF6F000EF06F000EF16FB00EF26F800EA3
:10176000F36F000EF46F8A0EF56F000EF66F000E29
:10177000F76F000EF86F000EF96F000EFA6F000E93
:10178000576E000E0101D96F150E0201FF6F000E9A
:10179000586E000E0101D86F000EDB6F3901938780
:1017A00012000201745104E13D0E735DD8A00DD00A
:1017B000000E0001B46F000E0101676F000ED46FC0
:1017C000000E0201746F000E736F3C0E0101BA65CA
:1017D0001ED0000EBB6F000EBA6F000E0001AF6F7F
:1017E000010E0101AC6F000E676F000E406E420EDD
:1017F0000001B56FB551B5253D016F6FFE0E706FDD
:10180000010E0101B16F000E4E6E010EA96F0201B3
:101810005B51571904E15C515819D8B412005BC2EE
:1018200057F25CC258F2010E0101A06F1200D96F8D
:101830000A0E0001D76502D00A0ED76FF10EC26FF3
:10184000F80EC36F570EC46F020EC56F010EC66F40
:10185000D9C0C7F0D6C0C8F0000EC96F000ECA6F5D
:10186000000ECB6F000ECC6F000ECD6FF6C0CEF029
:10187000F8ECFEF0CA0EC26FFD0EC36F050EC46F0A
:10188000020EC56F000EC66FD751080DF350D92553
:10189000D86FD829C76FD6C0C8F0000EC96F000E28
:1018A000CA6F000ECB6F000ECC6F000ECD6FF6C06E
:1018B000CEF0F8ECFEF0D75112004904D8A41FD0A6
:1018C0004850BE6FBF6BBE1DC06FBF1DC16FBC5106
:1018D000C05DBD51C159D8B003D0BC69BD6904D049
:1018E0004850BC27000EBD23BC51335CBD51345859
:1018F000D8B020D033C0BCF034C0BDF01BD0FF0E38
:10190000BE6FFF0EBF6FBCC0C0F0BDC0C1F0BE5106
:10191000C027BF51C1234850C05D000EC159D8B087
:1019200005D0000EBD6F010EBC6F04D04850BC5FE7
:10193000000EBD5B000E486EBCC0BCF0BDC0BDF06B
:101940001200C06F000E0001C16FC005D8A42FD0D7
:10195000010E0101C26F0001BC51BE6FBF6BBE51D1
:101960000101245D0001BF5101012559D8A006D015
:1019700000019705D8A402D0000E12D00001BD517D
:10198000BE6FBF6BBE510101245D0001BF5101015B
:101990002559D8A016D000019751D8A412D0010E15
:1019A000976F000E0101256F000E246F07D0000E07
:1019B0000101256F000E246F000EC26F010E0001A1
:1019C000C16F0001C15112006F00D8FF2BF06F00F2
:1019D000DCFF2CF06F00E0FF2DF06F00D4FF2EF045
:1019E000390193B1A3A103D098ECFDF023D093A3C8
:1019F00002D0A3B3F9D793B7A3A703D0D2EC0FF0CB
:101A000019D093B9A3A903D056EC15F013D09AB30B
:101A1000AAA303D0A7EC0EF00DD093A502D0A3B5D6
:101A2000E3D792AF02D0A2BFDFD79AB3AAA302D066
:101A3000C8EC18F06000BBF0F5FF6000B7F0F8FFED
:101A40006000B3F0F7FF6000AFF0F6FF1100000197
:101A5000D66F890E0001C26FF70EC36F0F0EC46FF1
:101A6000020EC56FD651020DF350060FC66F4A0E17
:101A7000C76F040EC86F000EC96F000ECA6F000E4C
:101A8000CB6F000ECC6F000ECD6FF6C0CEF0F8EC31
:101A9000FEF0890EC26FF70EC36F0F0EC46F020EF9
:101AA000C56FD651020DF350070FC66F590EC76FA1
:101AB000040EC86F000EC96F000ECA6F000ECB6F08
:101AC000000ECC6F000ECD6FF6C0CEF0F8ECFEF03D
:101AD000120078EC18F0F7EC17F00CEC09F06CEC55
:101AE00018F0BDEC18F0ACEC11F07DEC16F018EC31
:101AF00018F044EC18F066EC16F093EC16F04EEC8F
:101B000016F0BDEC14F09DEC14F08BEC0BF060ECD7
:101B100018F0D4EC16F07DEC10F0A00E0001BD6FB3
:101B2000C80EBE6FA40EBF6FA60EC06FA20EC16F0F
:101B30002F0EC26F270EC36F810EC46F100EC56FBC
:101B4000FA0EC66F900EC76FAF0EC86F400E0DEC49
:101B500010F01200D66F040E0001D66502D0040EFC
:101B6000D66F560EC26FEB0EC36F220EC46F040EFB
:101B7000C56FD629C66F220EC76F030EC86F000E41
:101B8000C96F000ECA6F000ECB6F000ECC6F000E37
:101B9000CD6FF6C0CEF0F8ECFEF0420EC26FF10E43
:101BA000C36F0A0EC46F030EC56FD6510A0FC66FFE
:101BB000480EC76F040EC86F000EC96F000ECA6FC3
:101BC000000ECB6F000ECC6F000ECD6FF6C0CEF0C6
:101BD000F8ECFEF01200D66F040E0001D66502D0BC
:101BE000040ED66F890EC26FF70EC36F0F0EC46F4F
:101BF000020EC56FD629C66F3A0EC76F060EC86FA4
:101C0000000EC96F000ECA6F000ECB6F000ECC6FB6
:101C1000000ECD6FF6C0CEF0F8ECFEF0D70EC26F1E
:101C2000FC0EC36F050EC46F010EC56FD6C0C6F0A3
:101C30004D0EC76F070EC86F000EC96F000ECA6F3A
:101C4000000ECB6F000ECC6F000ECD6FF6C0CEF045
:101C5000F8ECFEF01200EC51FD0DF350360FEE6F74
:101C6000ECC0EDF0FF0EED27EDB1EE2B690EC26F6B
:101C7000FC0EC36F660EC46F010EC56F000EC66FFB
:101C8000000EC76F010EC86F000EC96F000ECA6F3D
:101C9000010ECB6F000ECC6F000ECD6FF6C0CEF0F4
:101CA000F8ECFEF0EAC0D6F0EBC0D7F0ECC0D8F00C
:101CB000EEC0D9F0010EDA6F000EDB6F000EDC6FA4
:101CC000010EDD6F000EDE6F000EDF6F8DECE6F0B3
:101CD0001200C66F240E0001C66102D0240E04D08B
:101CE000F00EC66502D0F00EC66FC6C0C4F0C43B8D
:101CF0000F0EC417C451C65D01017D6FC6C0C4F08C
:101D00000001C43B0F0EC417C6C0C5F0D890C53340
:101D1000C451C55D01017C6FD8907C317B6F00019F
:101D2000C6390F0B01017A6F140E0001C06FC65146
:101D300038EC15F00101796F160E0001C06FC65125
:101D400038EC15F00101786F0001C6511200AA931A
:101D50003C016AAB02D0010E01D0000E4918D8B484
:101D600005D0000E6ABB010E496E2AD056AB27D0B3
:101D70009E50D8B424D0010178519E5CD8B002D0D6
:101D80004F0E17D079519E5CD8B002D0270E11D0DB
:101D90007A519E5CD8B002D0130E0BD07B519E5C62
:101DA000D8B002D0090E05D07C519E5CD8B003D0CB
:101DB000040E482604D07D519E5CD8A0482A482AAB
:101DC000010E0101A76F1200C16F05D0000E01D0F6
:101DD000010EC06F21D00001C1510A0AD8B4F6D754
:101DE000010AD8B4F3D7070AD8B4F0D7010AD8B497
:101DF000EDD7030AD8B4EAD7240AD8B4E7D7190A2A
:101E0000D8B4E4D7070AD8B4E1D7010AD8B4DED7EA
:101E10000C0AD8B4DBD7DCD70A0EBC6FC151A9ECD1
:101E200016F0080AD8B408D00A0EBC6FC151A9EC4C
:101E300016F0090AD8A402D0000EC06FC0511200DB
:101E400001011C511D11D8B402D0010EA76F000171
:101E5000A351D8B403D0010E0101A76F0101A7055A
:101E6000D8A406D0000E216F000E206F000EA76FC1
:101E70000001AD51D8A406D0B451D8A403D0AE51BE
:101E8000D8B402D0000E01D0010E0101B96FB9051E
:101E9000D8A41200E00E205D2E0E2159D8A0120009
:101EA000060E0001A219D8B41200A2C0A1F0060EBD
:101EB000A26F010E9F6F12004904D8A422D048508F
:101EC000BE6FBF6BBE1DC06FBF1DC16FBC51C05D7B
:101ED000BD51C159D8B003D0BC69BD6904D04850C8
:101EE000BC27000EBD23BC510101085D0001BD519E
:101EF00001010959D8B014D008C1BCF009C1BDF026
:101F00000FD04850BC5D000EBD59D8B005D0000EB2
:101F1000BD6F000EBC6F04D04850BC5F000EBD5BAF
:101F2000000E486EBCC0BCF0BDC0BDF01200010187
:101F30002A510001CA5DC26F01012B510001CB592A
:101F4000C36F000EC56F640EC46F2DEC13F0C25149
:101F5000936F0101705100019319D8B40DD00101A4
:101F60002A510001CA5D01012B510001CB59D8A0B3
:101F700003D0010E01016F6F0001CA5101012A5DFA
:101F80000001CB5101012B59D8A012004EECFEF0FC
:101F900003D01BECFCF04F6E4F50D8B4FAD7C1EC15
:101FA00018F01200000E926E010E0101D76F150E8F
:101FB0005824D96EDA6A020EDA226F00A3F7DFFF27
:101FC000582A140E586402D0000E586E030E58188A
:101FD000D8B417C2DEF15850276E286ADE51296E38
:101FE0002A6A040E2926000E2A222750291812E1F7
:101FF00028502A18D8A40ED0000ED76F58C0DCF194
:10200000000E586E59C023F05A509DECFFF00101AC
:10201000DD6F1200000ED66F1200C96FC9C0CAF082
:10202000BDC0CBF0BEC0CCF0BFC0CDF0C0C0CEF0C4
:10203000C1C0CFF0C2C0D0F0C3C0D1F0C4C0D2F094
:10204000C5C0D3F0C6C0D4F0C7C0D5F0C8C0D6F064
:10205000BA90E40E00D000D0E82EFCD700D000D01B
:10206000BA80BB98000E0001D76FBB9AD751CA0F38
:10207000D96EDA6ADF5052EC18F0BB8A0001D72B18
:102080000C0ED765F2D7BB881200C16FC1C0B5F086
:102090000001B551B5253D016F6FFE0E706F010E49
:1020A0000101B16F010E676F000E0201986F000E03
:1020B0000001AF6F010E0101AC6F000E656F4004AF
:1020C000D8A40FD0000E0001606FC051D8B402D068
:1020D0000C0E01D0000E616F000E626F000E636F78
:1020E00008D0000E0001606FC051D8B4F3D71C0EA9
:1020F000F2D7040EFCEC06F01200420E0001B56FA0
:10210000B551B5253D016F6FFE0E706F000E716FFA
:10211000000E726F000E746F100E756F000E7B6FE5
:102120006C69900E736F3901A29FA3933D0179955D
:102130003901A391A3953D01769979973901928F41
:1021400093833D017A853901938193853D017681A1
:102150007A87210E3A01136F000E3D01796F000E50
:10216000766F73991200C15104E1020EC05DD8A0D0
:1021700012D0C15110E11F0EC05DD8A0C0B10BD06C
:10218000FF0EC025BC6FFF0EC121BD6F27EC18F0FC
:102190005A0AD8B412D00001C15104E1210EC05D29
:1021A000D8A01200FF0EC025BC6FFF0EC121BD6F6D
:1021B00027EC18F05B0AD8A41200FF0E0001C0251E
:1021C000BC6FFF0EC121BD6FFF0EBE6F5BEC14F044
:1021D000120001013805D8A41CD0000E386F000E83
:1021E0003B6F000E3A6F000E0001CC6F39C0CDF08E
:1021F0003AC0CEF0020ED06F020ECF6F040ED26F37
:10220000040ED16F090E09ECDCF0CCC039F0CDC062
:102210003AF001013905D8A402D0000E396F3BC154
:10222000DCF03B5038ECF4F001013A6F3B513A19C5
:10223000D8B412003AC13BF1120001011C511D112A
:10224000D8B402D0010EA76F0001A351D8B403D0B7
:10225000010E0101A76F5050D8A403D0010E010157
:10226000B86F0101A705D8A408D0000E0201646F61
:10227000000E636F000E0101A66FA00E0201635DE8
:102280000F0E6459D8A012000001AD51D8A412005D
:10229000B451D8A41200010E0101A66F1200BD6F47
:1022A000010E0001BC6FBD05D8A402D0010E23D0E1
:1022B000020EBD19D8A402D0020E1DD0040EBD1905
:1022C000D8A402D0030E17D0080EBD19D8A402D08E
:1022D000040E11D0100EBD19D8A402D0050E0BD0DB
:1022E000200EBD19D8A402D0060E05D0400EBD198F
:1022F000D8A402D0070EBC6FBC511200CB6F0001F6
:10230000C851D8B40DD0C851070BC46F180E1BECC0
:1023100016F0020E0001C46F150E1BEC16F005D06E
:10232000010EC46F150E1BEC16F00001CB51D8B492
:102330000DD0CB51070BC46F190E1BEC16F0020E1B
:102340000001C46F160E1BEC16F01200010EC46FD4
:10235000160E1BEC16F01200000EDE6F000EDF6F83
:10236000000EE06F000EE16F000EE46F000EE56FEF
:10237000000EEA6F000EEC6F000EF16F000EF36FAF
:10238000000EF46F000EF56F000EF66F000EF76F83
:10239000000EF96F000EFA6F000EFB6F000EFC6F5F
:1023A000030EFD6F160EFE6F1F0EFF6F940EF86F7B
:1023B0001200AE0E0001CE6F470ECF6FA10ED06F90
:1023C0003F0ED16FEDC0BCF0EEC0BDF0BE6BBF6B79
:1023D000000EB2EC00F0BCC0CAF0BDC0CBF0BEC075
:1023E000CCF0BFC0CDF04BECE8F0CAC0E3F0CBC0FE
:1023F000E4F0CCC0E5F0CDC0E6F0AFEC08F0E3C00F
:10240000EDF0E4C0EEF01200AE0E0001CE6F470E0C
:10241000CF6FA10ED06F3F0ED16FEDC0BCF0EEC0FC
:10242000BDF0BE6BBF6B000EB2EC00F0BCC0CAF0DA
:10243000BDC0CBF0BEC0CCF0BFC0CDF04BECE8F0DF
:10244000CAC0E3F0CBC0E4F0CCC0E5F0CDC0E6F00C
:10245000AFEC08F0E3C0EDF0E4C0EEF01200000EC7
:102460000001CE6F000ECF6F800ED06F3F0ED16F88
:10247000EDC0BCF0EEC0BDF0BE6BBF6B000EB2ECA9
:1024800000F0BCC0CAF0BDC0CBF0BEC0CCF0BFC035
:10249000CDF04BECE8F0CAC0E3F0CBC0E4F0CCC028
:1024A000E5F0CDC0E6F0AFEC08F0E3C0EDF0E4C03D
:1024B000EEF01200140E0001CE6FAE0ECF6FC70EFD
:1024C000D06F3F0ED16FEDC0BCF0EEC0BDF0BE6B63
:1024D000BF6B000EB2EC00F0BCC0CAF0BDC0CBF0C8
:1024E000BEC0CCF0BFC0CDF04BECE8F0CAC0E3F00A
:1024F000CBC0E4F0CCC0E5F0CDC0E6F0AFEC08F026
:10250000E3C0EDF0E4C0EEF01200050E0001BC5D8A
:10251000100EBD59D8A002D0640E12001F0EBC5D73
:102520000F0EBD59D8A002D0500E1200610EBC5D36
:102530000E0EBD59D8A002D03C0E1200C10EBC5DDB
:102540000D0EBD59D8A002D0280E1200E50EBC5DBC
:102550000C0EBD59D8A002D0140E1200000E1200AD
:102560000001C76F000E0001C56F000EC66F640E3C
:10257000C06FC75138EC15F0300FC46F0A0EC06F32
:10258000640EBC6FC751A9EC16F038EC15F0300F93
:10259000C56F0A0EBC6FC751A9EC16F0300FC66F9D
:1025A000C4C0F2F22E0E0201F36FC5C0F4F2C6C031
:1025B000F5F21200C16FBEC0C2F0BFC0C3F0D4ECD0
:1025C00016F00001C151C1253D01586F89EC17F08B
:1025D000600003F356FD3D015D8B76EC17F00CD0E7
:1025E00060000BF3D9FF60000FF3DAFFDF5035EC2A
:1025F00016F00001C24BC32B0001C007C029D8A4AC
:10260000EFD7AFEC17F012000101E805D8A41200D3
:1026100075C2EDF076C2EEF0D9EC11F0EDC059F2D2
:10262000EEC05AF2A10E0201595D0F0E5A59D8A000
:1026300006D00001B451D8A402D0010E01D0000E82
:102640000101AA6F0001AD510101AA19D8B412000D
:10265000AAC1ADF0010E776F1200000EC86F000E18
:10266000C76FC451C511D8B41CD0010EC66F04D0B9
:10267000D890C437C537C62BC5AFFAD7D890C7375F
:10268000C837C451C25DC551C359D8A005D0C45183
:10269000C25FC551C35BC781D890C533C433C62F51
:1026A000EDD7C7C0C2F0C8C0C3F012000001BD6FB3
:1026B0004904D8A411D04850FF0A0001BC6FBD5195
:1026C000BC5DD8B002D0BD6902D04850BD27120E03
:1026D000BD6511D0120E0ED00001BD51485CD8A0CE
:1026E00003D0010EBD6F02D04850BD5F080EBD6122
:1026F00002D0080EBD6F000E486EBD5112000001E1
:10270000BD6F0001BD05D8A40FD0BB98BB9AA00E29
:1027100052EC18F0BB8A350EE82EFED700F0BB9ABB
:10272000C80E52EC18F00ED0BB98BB9AA10E52EC1A
:1027300018F0BB8A350EE82EFED700F0BB9AC00E0B
:1027400052EC18F0BB8ABB880001BD511200D86F53
:10275000D8C0D9F01DD0690EC26FFC0EC36F660ED3
:10276000C46F010EC56F000EC66F000EC76FD9C0D3
:10277000C8F0000EC96F000ECA6F000ECB6F000EBE
:10278000CC6F000ECD6FD7C0CEF0F8ECFEF0D92B99
:102790000001D951D65DD8A01200DDD7BD6F490424
:1027A000D8A413D04850FF0A0001BC6FBD51BC5DD6
:1027B000D8B002D0BD6902D04850BD27BD513E5CA3
:1027C000D8B00DD03EC0BDF00AD048500001BD5D6C
:1027D000D8B003D0000EBD6F02D04850BD5F000ED0
:1027E000486EBD511200BD6F4904D8A411D04850A5
:1027F000FF0A0001BC6FBD51BC5DD8B002D0BD69FD
:1028000002D04850BD27040EBD650CD0040E06D082
:1028100048500001BD5DD8B003D0000EBD6F02D09E
:102820004850BD5F000E486EBD5112000101D751E6
:10283000D8A41AD034C1BCF0A50E0001BC6502D0EA
:10284000640E0BD09B0EBC6502D0420E06D0960ED5
:10285000BC6502D0210E01D0000EBC6F34C164F102
:10286000010E0101636F02D062C1BCF00001BC51D6
:1028700012003C0174AB04D00001BC6BBC2B02D035
:102880000001BC6B3C0174AB02D0010E01D0000E04
:102890000101B519D8B402D0010E01D0000E00011B
:1028A000BC15BD6F3C01000E74BB010E0101B56F7C
:1028B0000001BD511200000ED2BE010EBF6FBD510E
:1028C000030B3901E16F6000F3F2E0F96000FBF205
:1028D000E3F93F0EE517E585D29E550EE66FAA0E89
:1028E000E66FE583E5B3FED7E5950001BFB102D001
:1028F000D29E01D0D28E1200BE51BF11D8B418D0D2
:10290000010EC06F04D0D890BE37BF37C02BBFAF09
:10291000FAD7BE51BC5DBF51BD59D8A004D0BE513D
:10292000BC5FBF51BD5BD890BF33BE33C02FF1D762
:10293000BCC0BCF0BDC0BDF01200000EB36E000EF6
:10294000B46E050EB56EEC0EB16E780EB06EB05072
:102950006F00C4FEBCF00001BD6BBCC0BDF0BC6B21
:10296000BC110201FD6F0001BD510201FE6F390172
:10297000A4919481010EB26E1200000E9B6E000EA7
:102980009C6E020E9D6EE20E996E000E986E98502F
:102990006F0064FEBCF00001BD6BBCC0BDF0BC6B41
:1029A000BC110301F56F0001BD510301F66F390140
:1029B000A89D010E9A6E1200C95101011C1500015B
:1029C000C26FCA5101011D150001C36FC9C0C4F017
:1029D000CAC0C5F02DEC13F0C251CB6FCB51D8B4A7
:1029E00007D00A0EA219D8A403D0010E01017F6FEF
:1029F0000001CB511200C951020153150001C26FF1
:102A0000CA51020154150001C36FC9C0C4F0CAC045
:102A1000C5F02DEC13F0C251CB6FCB51D8B407D019
:102A20000A0EA219D8A403D0010E01017F6F000184
:102A3000CB511200000E0001BE6FCABE02D0010EC3
:102A400001D0000EBE6FBE51A519BD6FBD51BE15A0
:102A5000A36FBE51D8A403D0BC6BBC2B02D0000125
:102A6000BC6BBD51BE19BC15A46FBEC0A5F0120051
:102A7000C16F000E0001C36FC051D8B415D0010E54
:102A8000C26F03D0D890C037C22BC0AFFBD7D8904D
:102A9000C337C051C15DD8A003D0C051C15FC3814D
:102AA000D890C033C22FF3D7C35112000201FF5197
:102AB000D8B410D0EB0E5724D96EDA6A010EDA22A0
:102AC000DF503D01EA6F572A150E57640AD0150EE4
:102AD000576E07D039019399000E0101D56F000E92
:102AE000586E0201FF0712004D0EC26FFA0EC36F3F
:102AF0000B0EC46F010EC56F060EC66F3F0EC76F7B
:102B0000000EC86F010EC96F000ECA6F000ECB6FAA
:102B1000000ECC6F000ECD6FF6C0CEF0F8ECFEF0DC
:102B200012004D0EC26FFA0EC36F0B0EC46F010E72
:102B3000C56F010EC66F3F0EC76F000EC86F010E46
:102B4000C96F000ECA6F000ECB6F000ECC6F000E67
:102B5000CD6FF6C0CEF0F8ECFEF012000D0E206046
:102B600012001EC00FF01FC010F020C011F0000EA8
:102B7000126E000E136E000E146E000E166E000E16
:102B8000156E000E176E000E196E000E186E000EF8
:102B900095EC05F01200010E0001CA6FFF0ECB6F1D
:102BA000000ECC6F000ECD6F000ECE6F000ECF6FFB
:102BB000000ED16F000ED06F000ED26F000ED46FDA
:102BC000000ED36F050E16EC03F012000001BD6F6E
:102BD0001F0E0001BD6502D01F0EBD6FBB98BB9AD2
:102BE000270E52EC18F0BB8ABB9A810E52EC18F0FB
:102BF000BB8ABB9A0001BD5152EC18F0BB8ABB885E
:102C00001200C56FD90E0001C66F020EC76FC5C096
:102C1000D9F2C4C0DAF2080EC4611200C451D8B4AB
:102C20001200C6C0BEF0C7C0BFF0020EC06F580E83
:102C3000DAEC12F01200C56FD90E0001C66F020E59
:102C4000C76FC5C0D9F2C4C0DAF2080EC461120061
:102C5000C451D8B41200C6C0BEF0C7C0BFF0020E47
:102C6000C06F580EDAEC12F012000001BC6F0001C8
:102C7000BD695650D8A412000BD03D0162AB04D000
:102C80006000F3F255FD1200050EE82EFED700F0AD
:102C90000001BD2FF2D7010E566E1200050E576FC0
:102CA000000E586F070E596F010E5A6F070E5B6FBB
:102CB000110E5C6F000E5D6F220E5E6F000E5F6F77
:102CC0009B0E566F3901AA939A831200010E966EDD
:102CD000000E956E000E976E9368000E926EA9918D
:102CE0009981000E0001BC6F000EBD6F000EBE6F1B
:102CF000A6EC18F0D00E946E12000F0E3C016B6F14
:102D0000000E6C6F010E6D6F270E6E6F070E6F6FEA
:102D1000260E706F190E716F290E726F160E736F7B
:102D2000830E6A6F12000A0E3C01756F0E0E766FED
:102D3000050E776F050E786F050E796F020E7A6FAC
:102D4000000E7B6F000E7C6F000E7D6F860E746F21
:102D50001200BD6F080E0001BE6F000EBF6FD8904D
:102D6000BD35BF35BF6FD890BD37BC51BF5DD8A052
:102D700002D0BC51BF5FBE2FF2D7BF511200BC6F53
:102D80000001BC05D8A40BD0010EBD6F120E3F642C
:102D900008D0120E8F6F010E01015B6F02D0000E82
:102DA000BD6F0001BD5112003D015DAF03D0565013
:102DB000D8B41200000E566E800E5E6F200E5F6F4C
:102DC000030E656F840E5D6F000E636F000E606F03
:102DD0001200B2C0B5F00001B251B2253D016F6FD3
:102DE000FE0E706F010E0101B16F010E4E6E010EED
:102DF0000001AF6F010E0101AC6F1200BC51BE03A8
:102E00006F00CCFFC0F06F00D0FFC1F0BC51BF031A
:102E1000F350C127BD51BE03F350C127C0C0BCF061
:102E2000C1C0BDF01200000EBF6F000EC06F09D010
:102E3000C051BC25D96E000EBD21DA6EDF50BF1B1C
:102E4000C02BBE51C05DD8A0F3D7BF511200070EF2
:102E50000001926503D0120E926504D00D0E926FA0
:102E600092C06BF1B051D8B403D0030EB06512001C
:102E7000020EB06F1200C951020155150001C26F58
:102E8000CA51020156150001C36FC9C0C4F0CAC0BF
:102E9000C5F02DEC13F0C251CB6FCB511200000ED8
:102EA000046E000E056E09D005500124D96E000E87
:102EB0000220DA6EDF50041A052A0350055CD8A000
:102EC000F3D7045012000001BD6F010E0101D56F50
:102ED000BCC0DAF1BCC0FFF2390193B905D0600083
:102EE000F7F2EAFD010E576E938912000001BC69EA
:102EF0005650D8A4120007D03D015DAB1200050E5C
:102F0000E82EFED700F00001BC2FF6D7010E566E5A
:102F100012000001BC695650D8A4120007D03D0130
:102F200061BF1200050EE82EFED700F00001BC2F95
:102F3000F6D7010E566E12006F0060FFBBF039012C
:102F400094B1A4A103D08EEC18F005D099B1A9A139
:102F500002D0ADEC18F06000EFF2D8FF1100BC69B0
:102F60005650D8A4120007D03D0163B51200050EDB
:102F7000E82EFED700F00001BC2FF6D7010E566EEA
:102F800012000001BC6F0101E4510001BC19D8B46A
:102F900007D03E01F89F6000F3F2F1FEF88FF89D34
:102FA0000001BC511200B2A409D0B2906000EBF253
:102FB000B1FF6000E7F2B0FFB28012006000EBF2F8
:102FC000B1FF6000E7F2B0FF1200026E010E0101D6
:102FD000D56F01C0DAF101C0FFF2390193B905D014
:102FE00060000BF0EAFD010E576E93891200000E8F
:102FF000C06F000EC16F000EC26F000EC36F000ED7
:10300000C46F000EC56F000EC66F000EC76F1200B2
:103010003E01F0510001BF6FBE6B3E01EF51000158
:10302000BE25BC6F3E01000E0001BF21BD6F120026
:10303000040EA26E130EA16E140EA36EF00E9F6E00
:10304000000E9E6E3901A791E00EA06E1200BD51D8
:10305000030B3901E16F6000F3F2E0F93F0EE51771
:10306000E58100F000F03901E3511200AE47A13FC5
:10307000AE47A13F6666663F14AEC73F0000803F83
:103080005E01052020202000060EAE6E000EAD6E03
:10309000000EAF6E610EAB6E000EAA6EA495C00E50
:1030A000AC6E12000001BC6F010E3D01126F60009A
:1030B000F3F211FD3901A2A9FDD73D011051120013
:1030C000200E3D01156F030E166F070E196F010ECE
:1030D0001C6F830E146F1200600E3901D96F000E41
:1030E000DB6F000EDD6F080EDF6F000EDE6F12006B
:1030F000D28A390183818383838783898385828F01
:103100008A8384918991120000019051D8B403D030
:10311000DAECFCF0120066EC09F01200A491FDC29A
:10312000B9F0FEC2BAF0D3EC17F02AECF7F01200B7
:10313000BCC0F7F2BDC0F8F2BEC0F9F21200BCC0CC
:10314000FAF2BDC0FBF2BEC0FCF21200BCC0F2F34A
:10315000BDC0F3F3BEC0F4F31200A991010E01014A
:10316000E26F000E586E12000001BC6F0001BC51EE
:103170001200BC6FBCC09DF01200820E3E01C16FF8
:103180001200BE92C6921200AC8E1200B2801200E3
:10319000AA931200FFFFFFFFFFFFFFFFFFFFFFFFEC
:1031A000FFFFFFFFFFFFFFFFFFFFFFFFFFFFFFFF2F
:1031B000FFFFFFFFFFFFFFFFFFFFFFFFFFFFFFFF1F
:1031C000FFFFFFFFFFFFFFFFFFFFFFFFFFFFFFFF0F
:1031D000FFFFFFFFFFFFFFFFFFFFFFFFFFFFFFFFFF
:10AE7000FFFFFFFFFFFFFFFFFFFF000000000000DC
:10AE8000000000000000000000FEFE0000000000C6
:10AE90007F7F606060606080C0C0C0C0C0803F7F56
:10AEA0006060607F3FFEFE0080C0C0407F7F1F3B30
:10AEB0007160400000606000000000000C0C0000A9
:10AEC00000F0FC1E061EFCF07F7F0303037F7FC0A3
:10AED000E0F070E0FEFE1F3F7870387F7FF0F0807A
:10AEE000C0E070707F7F03010000000000000000E0
:10AEF0000000005A7765697465204C6F6B00496EDD
:10AF0000746572666163650050726F6772616D008F
:10AF100053746174757300536574757000A00000FC
:10AF20000000000000000000000000000000000021
:10AF30000000000000000000000000000000000011
:10AF40000000000000000000000000000000000001
:10AF500000000000000000000000000000000000F1
:10AF600000000000000000000000000000000000E1
:10AF700000000000000000000000000000000000D1
:10AF800000000000000000000000000000000000C1
:10AF900000000000000000000000000000000000B1
:10AFA00000000000000000000000000000000000A1
:10AFB0000000000000000000000000000000000091
:10AFC0000000000000000000000000000000000081
:10AFD0000000000000000000000000000000000071
:10AFE0000000000000000000000000000000000061
:10AFF0000000000000000000000000000000000051
:10B000000000000000000000000000000000000040
:10B010000000000000000000000000000000000030
:10B020000000000000000000000000000000000020
:10B030000000000000000000000000000000000010
:10B040000000000000000000000000000000000000
:10B0500000000000000000000000000000000000F0
:10B0600000000000000000000000000000000000E0
:10B07000000000FE020202020202020202020202BA
:10B0800002020202020202020202020202020202A0
:10B090000202020202020202020202020202020290
:10B0A0000202020202020202020202020202020280
:10B0B00002020202FE0000FF00000000000000008B
:10B0C0000000000000000000000000000000000080
:10B0D0000000000000000000000000000000000070
:10B0E0000000000000000000000000000000000060
:10B0F0000000000000000000FF0000FF0000000052
:10B10000000000000000000000000000000000003F
:10B11000000000000000000000000000000000002F
:10B12000000000000000000000000000000000001F
:10B13000000000000000000000000000FF0000FF11
:10B1400000000000000000000000000000000000FF
:10B1500000000000000000000000000000000000EF
:10B1600000000000000000000000000000000000DF
:10B1700000000000000000000000000000000000CF
:10B18000FF00007F40404040404040404040404041
:10B1900040404040404040404040404040404040AF
:10B1A000404040404040404040404040404040409F
:10B1B000404040404040404040404040404040408F
:10B1C000404040407F0000FE0202020202020202F2
:10B1D000020202020202FA32C202FA02824242422F
:10B1E000820242FA420202FA8242428202824242CF
:10B1F00082C202FA020242FA42020202020202027F
:10B200000202020202020202FE0000FF0000000031
:10B21000808000800080000000800780E09317009D
:10B22000F304848403000083840400F70080800713
:10B230000003848402078003848400030404000064
:10B240000000A0008000808000000000FF0000FFE0
:10B25000000000070808050F00070808040F000099
:10B260000F0000000F0100000F00070A0A0B000F7B
:10B270000908080700070A0A0B000F0100000F0069
:10B280000000000000000F000F0100000F00000090
:10B29000FF0000FF000000000000000000000000B0
:10B2A0000000000000000000000000FF010101019B
:10B2B00001FF000000FF0101010101FF000000008B
:10B2C000000000000000000000000000000000007E
:10B2D00000000000FF00007F4040404040404040F0
:10B2E000404040404040404040404040404040FF9F
:10B2F0008080808080FF404040FF8080808080FF91
:10B30000404040404040404040404040404040403D
:10B3100040404040404040407F0000FE02020202A8
:10B32000FA02020202E29AE20202FA82422202FADD
:10B3300082422202C2020202C2028242424202420D
:10B34000FA42020282424282C202C2824242820225
:10B3500082424282FA020202FA020202FE0000FF68
:10B3600000008080058000F0078080000700878152
:10B3700082040087818204F00384840207008485AC
:10B38000058200F0030484F0830404028780070030
:10B390008000878003040404A700800085800000EB
:10B3A000FF0000FF00070808050F000F0908080745
:10B3B00000090A0A040007080808000F0100000F2E
:10B3C00000070808050F000708080007080800071D
:10B3D0000A0A0B000F0100000F0000000F000F0110
:10B3E00000000F00FF0000FF000000000000000050
:10B3F0000000000000000000000000FF010101014A
:10B4000001FF0000FF0101010101FF000000FF0139
:10B4100001010101FF000000000000000000000029
:10B420000000000000000000FF00007F404040409E
:10B43000404040404040404040404040404040FF4D
:10B440008080808080FF4040FF8080808080FF403F
:10B450004040FF8080808080FF404040404040402E
:10B460004040404040404040404040407F0000FE5F
:10B4700002020202020282424282C202FA82424274
:10B48000820282424242028242424202FA824243A3
:10B49000820282424282C202FA020242FA4202025C
:10B4A0008242428202C282424282020202020202BC
:10B4B000FE0000FF0000000000000304040207007B
:10B4C0000704040403000405050200030404040047
:10B4D000A70080008780030404020700030404001F
:10B4E0000304040003050505000700000007000031
:10B4F00000000000FF0000FF00000000000000004E
:10B50000000000000000000000000000000000003B
:10B51000000000000F000F0100000F0000000000FD
:10B52000000000000000000000000000000000001B
:10B530000000000000000000FF0000FF000000000D
:10B5400000000000000000000000000000000000FB
:10B55000000000FF0101010101FF000000FF0101E7
:10B56000010101FF000000000000000000000000D9
:10B57000000000000000000000000000FF00007F4D
:10B5800040404040404040404040404040404040BB
:10B5900040404040404040FF8080808080FF4040ED
:10B5A00040FF8080808080FF4040404040404040DD
:10B5B000404040404040404040404040404040408B
:10B5C0007F0000FE020202020202020202020202E6
:10B5D0000202F2628202F20202828282020282F29B
:10B5E000820202F20282820202028282028202F25B
:10B5F000020282F28202020202020202020202023B
:10B6000002020202FE0000FF000000000000000035
:10B610000000000000000F0001060F0007080808E6
:10B62000070000070808000F0100000F00070808C6
:10B63000050F0007080800070808000000000000C8
:10B640000000000000000000FF0000FF00000000FC
:10B6500000000000000070888850F800788080406A
:10B66000F80008FE090100FF100808F00070A8A803
:10B67000B000FF908888700070A8A8B000F810088B
:10B6800008F000000000000000000000FF0000FFC4
:10B690000080008080000090000080808000F0002A
:10B6A0008080000080F080010000000080800000A9
:10B6B0008000008000F0000000008080008000809A
:10B6C0000000008000F0008080000080F08000001A
:10B6D000FF00007F404F4140404F404F40474848A7
:10B6E00048404F4140404F40404748484040404715
:10B6F0004A4A4B404F4241404047484840474848EB
:10B70000454F40474848444F404F494848474040CC
:10B71000474848407F0000FE0202C232C2020202D5
:10B72000828202F202820202820202828202020209
:10B730008282820202828282029202028282020259
:10B740008202028202820202028202820282820259
:10B750000202828202820202FE0000FF000E01014C
:10B76000010E00070808090F000F02010000070A78
:10B770000A0B00090A0A0400090A0A04000F00075C
:10B780000A0A0B000F02010000070808040F000F4F
:10B790000100000F00072828251F0000FF0000FF00
:10B7A0000000000000000000000000000000000099
:10B7B0000000000000F8100808F000F90070888808
:10B7C0008800FF100808F000087F88800000000053
:10B7D0000000000000000000000000000000000069
:10B7E000FF0000FF0000000000000000000000005B
:10B7F000000000E02020C02020C000C0242024C081
:10B8000000C0202040E000FC000000E400C0202038
:10B810002000FC402020C0000000000000000000CC
:10B8200000000000FF00007F40404040404040409A
:10B8300040404040404040434040434040434041FE
:10B840004242424140414A4A4947404142424043C4
:10B8500040414242424043404040434040404040DB
:10B8600040404040404040407F0000FE0202C24253
:10B8700042428202020202020202020202020202A8
:10B880000202020202024202020202020202020258
:10B89000020202824242020202020202C2020202C8
:10B8A0000202020202020202C2020202FE0000FFC3
:10B8B00000003F060A1221001C2222143E003E0412
:10B8C00002023C001CA2A2947E003E001C2A2A2CEC
:10B8D000003E0804020002FF02001C2222143E0067
:10B8E0003F0402023C003E08040200021F22200026
:10B8F000FF0000FF0000000000000000000000004A
:10B900000000000000000000000000000000000037
:10B910000000000000000000000000000000000027
:10B920000000000000000000000000000000000017
:10B9300000000000FF0000FF000000000000000009
:10B94000000000000000000000000000E01010A057
:10B95000F000FE40A0100010FE100000F20030C009
:10B9600000C03000000000000000000000000000E7
:10B970000000000000000000FF00007F4040404049
:10B9800040404040404040404040404040404040B7
:10B9900040414140414041404041404040414140A0
:10B9A0004140404041404040404040404040404095
:10B9B0004040404040404040404040407F0000FE0A
:10B9C00002020202020202020202020202020282D7
:10B9D00082828202020202020202020202020202C7
:10B9E0000202020202020202020202020202020237
:10B9F0000202020202020202020202020202020227
:10BA0000FE0000FF00000000000000000000000039
:10BA10000000007F4444443B007C1008040038547C
:10BA20005458007C040478040478004854542400DA
:10BA300038545458000000000000000000000000CE
:10BA400000000000FF0000FF0000000000000000F8
:10BA500000000000000000000000000000000000E6
:10BA600000000000000000000000000000000000D6
:10BA700000000000000000000000000000000000C6
:10BA80000000000000000000FF0000FF00000000B8
:10BA900000000000000000000000000000000000A6
:10BAA000E01010A0F000FE40A0100010FE100000FA
:10BAB000F20030C000C030000000000000000000B4
:10BAC000000000000000000000000000FF00007FF8
:10BAD0004040404040404040404040404040404066
:10BAE0004040404040414140414041404041404051
:10BAF0004041414041404040414040404040404042
:10BB00004040404040404040404040404040404035
:10BB10007F0000FE0202020202020202C232C202E0
:10BB20000282020202820282F28202020282828285
:10BB300002028282820282820202028282028202E5
:10BB400082F28202029202F20202820202020202E5
:10BB500002020202FE0000FF000000000000000ED2
:10BB60000101010E00070808040F000007C8282083
:10BB7000070808080700EF00000F00000F00070883
:10BB80000805EF0000070808000F000F0205080075
:10BB90000101010101000000FF0000FF00000000A2
:10BBA0000000000000000000000000000000000095
:10BBB000017F01000E11110A1F001F0201011E006A
:10BBC0001F04020100010F1110000000000000001E
:10BBD000000000000000000000000000FF0000FF67
:10BBE0000000000000000000000000000000000055
:10BBF00000000000E01010A0F000FE40A0100010B7
:10BC0000FE100000F20030C000C030000000000054
:10BC10000000000000000000000000000000000024
:10BC2000FF00007F40404040404040404040404096
:10BC30004040404040404040404141404140414000
:10BC400040414040404141404140404041404040EF
:10BC500040404040404040404040404040404040E4
:10BC6000404040407F0000FE020202021AE202E26F
:10BC70001A0202C2A2A2C20202E28242220202FA14
:10BC8000422222C20202EA0202E2422222C202024C
:10BC9000C2222242FA0202C2A2A2C20202E242224C
:10BCA00022C2020202020202FE0000FFF8F8F8F8C7
:10BCB000F8F8FBF8F8F8F8F9FAFAFAF8F8FBF8F8F7
:10BCC000F8F8F8FBFAFAFAF9F8F8FBF8F8FBF8F8E4
:10BCD000F8FBF8F8F9FA1A1A1B1818191A1A1A1890
:10BCE000181B1818181B181818181818FF0000FF30
:10BCF0000303FBFBFBFBFBFBFB0303FFFFFFFFFF60
:10BD0000FFFFFFFFFFFFFFFFFFFFFFFFFFFFFFFF43
:10BD1000FFFFFFFFFFFFFFFFFFFF0080C04040C0AD
:10BD20008000C0C04040C0800040404040C0C000D3
:10BD3000FF0000FFFE00E2F0FAF8FAF0E200FEFF7A
:10BD4000FFFFFFFFFFFFFFFFFFFFFFFFFFFFFFFF03
:10BD5000FFFFFFFFFFFFFFFFFFFFFFFFFFFF000FE2
:10BD60001F10101D0D001F1F10101F0F00181C1694
:10BD700013111000FF00007F414054414B434B41E1
:10BD80005440417F7F7F7F7F7F7F7F7F7F7F7F7F6B
:10BD90007F7F7F7F7F7F7F7F7F7F7F7F7F7F7F7FB3
:10BDA0007F7F404040404040404040404040404015
:10BDB00040404040404040407F0000FE02020202FE
:10BDC00002020202020202020202020202E29AE2FB
:10BDD000020202FA028242020242FA42020202CA4B
:10BDE000020282424242820202C282424282020233
:10BDF000020202020202020202020202FE0000FF2E
:10BE00000000000000000000000000000000000032
:10BE100007000000070000070102040000000304FF
:10BE200004000007000003040404030000070000EE
:10BE300000070000000000000000000000000000FB
:10BE4000FF0000FF000000000000000000000000F4
:10BE500000000000000000F8100808F00000F900E1
:10BE600000708888880000FF100808F00000087F34
:10BE700088800000000000000000000000000000BA
:10BE800000000000FF0000FF00804040800000C074
:10BE9000008040000040F0480000804040408000AA
:10BEA00000F80000000080404080C00000C000801A
:10BEB000400000804040800000C8000080404040BA
:10BEC0000000F88040408000FF00007F404345456F
:10BED000454040474140404040405F40404043442F
:10BEE00044444340404344444040435454524F40F0
:10BEF0004047414040404043454545404047404021
:10BF00004344444440404740404047407F0000FE97
:10BF10000202020202020202020202020202020201
:10BF200002826282020202E2020202020202E202D1
:10BF300002020222020202020202020202020202C1
:10BF400002020202020202020202020202020202D1
:10BF5000FE0000FF000000000000000000000000E4
:10BF6000000000001C0302031C00001F040A110053
:10BF700000010F111000001F00000E1111110E0022
:10BF8000001F0201011E0000000000000000000070
:10BF900000000000FF0000FF0000000000000000A3
:10BFA000000000000000C0200000000000000000B1
:10BFB00000E00000000000000000000000000000A1
:10BFC0000000000000000000002000000000000051
:10BFD0000000E00000000000FF0000FF000E15154B
:10BFE0001600001F0402010000017F0100000E1175
:10BFF00011110E00000F101000000E51514A3F00A9
:10C00000001F04020100000E15151600001F00009D
:10C010000E11111100001F0201011E00FF00007F20
:10C020004040404040404040404040404040404010
:10C030004040404040404040404040404040404000
:10C0400040404040404040404040404040404040F0
:10C0500040404040404040404040404040404040E0
:10C060007F0000FE0202020202020202020202E25B
:10C070009AE20202C2020202C20242FA42020282B0
:10C080004242428302028282820202F20A0A0AF2D7
:10C090000242F24A0A0242F24A0A02020202020280
:10C0A00002020202FE0000FF00000000000000008B
:10C0B000000007000000070003040402070000035B
:10C0C00004040003A4048403808000000000000333
:10C0D0000404040300001F000000001F0000000013
:10C0E0000000000000000000FF0000FF0000000052
:10C0F0000000000000000000000000000000000040
:10C1000000000000000000000F000F0100000F0001
:10C11000000000000000000000000000000000001F
:10C12000000000000000000000000000FF0000FF11
:10C1300000000000000000000000000000000000FF
:10C1400000000000000000FF0101010101FF0000EC
:10C1500000FF0101010101FF0000000000000000DC
:10C1600000000000000000000000000000000000CF
:10C17000FF00007F40404040404040404040404041
:10C180004040404040404040404040FF80808080F0
:10C1900080FF404040FF8080808080FF40404040E2
:10C1A000404040404040404040404040404040408F
:10C1B000404040407F0000FE020202020202FA02FA
:10C1C000020202824242428202FA824222028242F7
:10C1D0004282C20282424282FA02C2824242028207
:10C1E00042428202824242420282424242028242EF
:10C1F0004282020202020202FE0000FF0000000072
:10C2000000000704048400030404048300078182FF
:10C2100004000384848207F0038484040700878079
:10C2200080000083850505F00405058200848505EE
:10C23000020003850505000000000000FF0000FF6C
:10C2400000000000000000000001060C070C0601C1
:10C2500000070A0A0B0007080808000F0100000F7A
:10C2600000090A0A0400070A0A0B00070808000F61
:10C270000100000F000000040000000000000000AA
:10C28000FF0000FF00000000000000000000FF01B0
:10C2900001010101FF0000FF0101010101FF000098
:10C2A000FF0101010101FF0000FF0101010101FF88
:10C2B000000000000000000000000000000000007E
:10C2C00000000000FF00007F4040404040404040F0
:10C2D0004040FF8080808080FF4040FF80808080E1
:10C2E00080FF4040FF8080808080FF4040FF808052
:10C2F000808080FF404040404040404040404040BF
:10C3000040404040404040407F00000000000000AE
:10C31000000000000000000000000000000000001D
:10C32000000000000000000000000000000000000D
:10C3300000000000000000000000000000000000FD
:10C3400000000000000000000000000000000000ED
:10C3500000000000000000000000000000000000DD
:10C3600000000000000000000000000000000000CD
:10C3700000000000000000000000000000000000BD
:10C3800000000000000000000000000000000000AD
:10C39000000000FCFA060606060606060606064625
:10C3A000A6262626460606068686860606068606ED
:10C3B000868606060606868606E6060606868686BD
:10C3C000060606860686860606060606060606068D
:10C3D000060606FAFC00003F5F6060606060606017
:10C3E000606060646869696A646060676A6A6A63F9
:10C3F00060606F6160606F6060676868656F6060F3
:10C40000676A6A6A6360606F6160606F60606060E5
:10C41000606060606060605F3F0000FCFA0606E6F6
:10C42000C686060606060646A626262646060606EC
:10C43000868686060606860686860606060686869C
:10C4400006E60606068686860606068606868606AC
:10C4500006060606060686C6E60606FAFCFE003F47
:10C460005FE0E0EFE7E3E1E0E0E0E0E4E8E9E9EA0B
:10C47000E4E0E0E7EAEAEAE3E0E0EFE1E0E0EFE071
:10C48000E0E7E8E8E5EFE0E0E7EAEAEAE3E0E0EF4A
:10C49000E1E0E0EFE0E0E0E0E0E1E3E7EFE0E0DF73
:10C4A000BF7FFF0305F9F9F9F9F9F9F9F9F9F9B9D4
:10C4B00059D9D9D9B9F9F9F9797979F9F9F979F92C
:10C4C0007979F9F9F9F97979F919F9F9F97979793C
:10C4D000F9F9F979F97979F9F9F9F9F9F9F9F9F94C
:10C4E000F9F9F90503FFFFC0A09F9F9F9F9F9F9FA2
:10C4F0009F9F9F9B979696959B9F9F989595959CA0
:10C500009F9F909E9F9F909F9F9897979A909F9F85
:10C51000989595959C9F9F909E9F9F909F9F9F9F72
:10C520009F9F9F9F9F9F9FA0C0FF00FCFA0606064B
:10C53000060606060606060606060606060606069B
:10C5400006060606E6F63636F6E6060606F6F6C6EB
:10C55000E6763606060606060606060606060606FB
:10C560000606060606060606060606FAFC00003F54
:10C570005F606060606060606060606060606060BC
:10C580006060606060606060676F6C6C6F67606067
:10C59000606F6F63676E6C60606060606060606059
:10C5A0006060606060606060606060606060605F8C
:10C5B0003F0000FCFA0606E6C686060606060606E4
:10C5C000060606060606060606060606E6F63636DB
:10C5D000F6E6060606F6F6C6E6763606060606060B
:10C5E000060606060606060606060606060686C6AB
:10C5F000E60606FAFCFE003F5FE0E0EFE7E3E1E07D
:10C60000E0E0E0E0E0E0E0E0E0E0E0E0E0E0E0E02A
:10C61000E7EFECECEFE7E0E0E0EFEFE3E7EEECE094
:10C62000E0E0E0E0E0E0E0E0E0E0E0E0E0E0E0E00A
:10C63000E0E1E3E7EFE0E0DFBF7FFF0305F9F9F9B1
:10C64000F9F9F9F9F9F9F9F9F9F9F9F9F9F9F9F95A
:10C65000F9F9F9F91909C9C90919F9F9F9090939EA
:10C660001989C9F9F9F9F9F9F9F9F9F9F9F9F9F9BA
:10C67000F9F9F9F9F9F9F9F9F9F9F90503FFFFC041
:10C68000A09F9F9F9F9F9F9F9F9F9F9F9F9F9F9FB9
:10C690009F9F9F9F9F9F9F9F9890939390989F9FEE
:10C6A0009F90909C9891939F9F9F9F9F9F9F9F9FDC
:10C6B0009F9F9F9F9F9F9F9F9F9F9F9F9F9F9FA089
:10C6C000C0FF00FCFA06060606060606C626162663
:10C6D000C60606F6864646860606F686464686065A
:10C6E00006C6068646460606C6060606C60606862A
:10C6F000464646860606F68646468606060606062A
:10C70000060606FAFC00003F5F60606060606060E3
:10C710006F6161616F60606F6468686760606F64BB
:10C7200068686760606F61606060606067686864C7
:10C730006F6060676868686460606F6060606F60A9
:10C74000606060606060605F3F0000FCFA0606E6C3
:10C75000C6860606C6261626C60606F686464686F9
:10C760000606F6864646860606C606864646060639
:10C77000C6060606C6060686464646860606F686A9
:10C7800046468606060686C6E60606FAFCFE003F14
:10C790005FE0E0EFE7E3E1E0EFE1E1E1EFE0E0EFD0
:10C7A000E4E8E8E7E0E0EFE4E8E8E7E0E0EFE1E034
:10C7B000E0E0E0E0E7E8E8E4EFE0E0E7E8E8E8E42C
:10C7C000E0E0EFE0E0E0EFE0E0E1E3E7EFE0E0DF32
:10C7D000BF7FFF0305F9F9F9F9F9F9F939D9E9D971
:10C7E00039F9F90979B9B979F9F90979B9B979F959
:10C7F000F939F979B9B9F9F939F9F9F939F9F97969
:10C80000B9B9B979F9F90979B9B979F9F9F9F9F948
:10C81000F9F9F90503FFFFC0A09F9F9F9F9F9F9F6E
:10C82000909E9E9E909F9F909B9797989F9F909B76
:10C830009797989F9F909E9F9F9F9F9F9897979B4A
:10C84000909F9F989797979B9F9F909F9F9F909F48
:10C850009F9F9F9F9F9F9FA0C0FF00FE0202D2024A
:10C8600002C2824242820202C2020202C202028268
:10C87000424242820202C202824242020282424298
:10C8800042820202020202020202020206FE0602C4
:10C89000826212120A0A121262820206FE00007FEF
:10C8A00040404F40404F4040404F404040434C4349
:10C8B000404040474949494940404F41404040403D
:10C8C0004044494B4A444040404040404040404042
:10C8D000607F60404146484850504848464140606B
:10C8E0007F0000FE0202D20202C2824242820202A3
:10C8F000C2020202C2020282424242820202C20218
:10C900008242420202824242428202020202020247
:10C910000202020206FE0602826212120A0A1212C3
:10C9200062820206FEFE003F40C0CFC0C0CFC0C042
:10C93000C0CFC0C0C0C3CCC3C0C0C0C7C9C9C9C9AB
:10C94000C0C0CFC1C0C0C0C0C0C4C9CBCAC4C0C0B1
:10C95000C0C0C0C0C0C0C0C0E0FFE0C0C1C6C8C841
:10C96000D0D0C8C8C6C1C0C0BF7F00FE06FA2AFA30
:10C97000FA3A7ABABA7AFAFA3AFAFAFA3AFAFA7A57
:10C98000BABABA7AFAFA3AFA7ABABAFAFA7ABABA07
:10C99000BA7AFAFAFAFAFAFAFAFAFAFA06FE060293
:10C9A00082E2F2F2FAFAF2F2E2820206FE00007F7E
:10C9B000605F505F5F505F5F5F505F5F5F5C535CC5
:10C9C0005F5F5F58565656565F5F505E5F5F5F5FB2
:10C9D0005F5B5654555B5F5F5F5F5F5F5F5F5F5F8D
:10C9E000607F604041474F4F5F5F4F4F474140601E
:10C9F0007F0000FE06FA2AFAFA3A7ABABA7AFAFA06
:10CA00003AFAFAFA3AFAFA7ABABABA7AFAFA3AFA86
:10CA10007ABABAFAFA7ABABABA7AFAFAFAFAFAFA36
:10CA2000FAFAFAFA06FE060282E2F2F2FAFAF2F2F2
:10CA3000E2820206FEFE003F60DFD0DFDFD0DFDFF4
:10CA4000DFD0DFDFDFDCD3DCDFDFDFD8D6D6D6D642
:10CA5000DFDFD0DEDFDFDFDFDFDBD6D4D5DBDFDF1C
:10CA6000DFDFDFDFDFDFDFDFE0FFE0C0C1C7CFCF29
:10CA7000DFDFCFCFC7C1C0C0BF7F00FE0202F2829E
:10CA80008282F20202F29292926202023242824266
:10CA90003202020202020202020202020202020246
:10CAA00002020202020202020202020206FE060262
:10CAB000826212120A0A121262820206FE00007FCD
:10CAC00040404F4040404F40404F4142444840402A
:10CAD0004C4241424C404040404040404040404039
:10CAE0004040404040404040404040404040404046
:10CAF000607F604041464848505048484641406049
:10CB00007F0000FE0202F2828282F20202F2929220
:10CB100092620202324282423202020202020202A5
:10CB200002020202020202020202020202020202E5
:10CB30000202020206FE0602826212120A0A1212A1
:10CB400062820206FEFE003F40C0CFC0C0C0CFC020
:10CB5000C0CFC1C2C4C8C0C0CCC2C1C2CCC0C0C09A
:10CB6000C0C0C0C0C0C0C0C0C0C0C0C0C0C0C0C0C5
:10CB7000C0C0C0C0C0C0C0C0E0FFE0C0C1C6C8C81F
:10CB8000D0D0C8C8C6C1C0C0BF7F00FE06FA0A7AAE
:10CB90007A7A0AFAFA0A6A6A6A9AFAFACABA7ABA15
:10CBA000CAFAFAFAFAFAFAFAFAFAFAFAFAFAFAFA15
:10CBB000FAFAFAFAFAFAFAFAFAFAFAFA06FE0602B1
:10CBC00082E2F2F2FAFAF2F2E2820206FE00007F5C
:10CBD000605F505F5F5F505F5F505E5D5B575F5FA0
:10CBE000535D5E5D535F5F5F5F5F5F5F5F5F5F5F72
:10CBF0005F5F5F5F5F5F5F5F5F5F5F5F5F5F5F5F45
:10CC0000607F604041474F4F5F5F4F4F47414060FB
:10CC10007F0000FE06FA0A7A7A7A0AFAFA0A6A6A43
:10CC20006A9AFAFACABA7ABACAFAFAFAFAFAFAFAB4
:10CC3000FAFAFAFAFAFAFAFAFAFAFAFAFAFAFAFA54
:10CC4000FAFAFAFA06FE060282E2F2F2FAFAF2F2D0
:10CC5000E2820206FEFE003F60DFD0DFDFDFD0DFD2
:10CC6000DFD0DEDDDBD7DFDFD3DDDEDDD3DFDFDF0F
:10CC7000DFDFDFDFDFDFDFDFDFDFDFDFDFDFDFDFC4
:10CC8000DFDFDFDFDFDFDFDFE0FFE0C0C1C7CFCF07
:10CC9000DFDFCFCFC7C1C0C0BF7F00FE0202F2827C
:10CCA0008282F20202F29292926202020202020274
:10CCB000028202028202028282020282F282020264
:10CCC00082020282020282828202020206FE0602C0
:10CCD000826212120A0A121262820206FE00007FAB
:10CCE00040404F4040404F40404F41424448404107
:10CCF00041414141404F42414040474A4A4B4040F8
:10CD0000474848404F4241404047484848474040D4
:10CD1000607F604041464848505048484641406026
:10CD20007F0000FE0202F2828282F20202F29292FE
:10CD30009262020202020202028202028202028263
:10CD400082020282F2820202820202820202828253
:10CD50008202020206FE0602826212120A0A1212FF
:10CD600062820206FEFE003F40C0CFC0C0C0CFC0FE
:10CD7000C0CFC1C2C4C8C0C1C1C1C1C1C0CFC2C17E
:10CD8000C0C0C7CACACBC0C0C7C8C8C0CFC2C1C054
:10CD9000C0C7C8C8C8C7C0C0E0FFE0C0C1C6C8C8D7
:10CDA000D0D0C8C8C6C1C0C0BF7F00FE06FA0A7A8C
:10CDB0007A7A0AFAFA0A6A6A6A9AFAFAFAFAFAFAC3
:10CDC000FA7AFAFA7AFAFA7A7AFAFA7A0A7AFAFAB3
:10CDD0007AFAFA7AFAFA7A7A7AFAFAFA06FE06020F
:10CDE00082E2F2F2FAFAF2F2E2820206FE00007F3A
:10CDF000605F505F5F5F505F5F505E5D5B575F5E7F
:10CE00005E5E5E5E5F505D5E5F5F585555545F5F6E
:10CE10005857575F505D5E5F5F58575757585F5F71
:10CE2000607F604041474F4F5F5F4F4F47414060D9
:10CE30007F0000FE06FA0A7A7A7A0AFAFA0A6A6A21
:10CE40006A9AFAFAFAFAFAFAFA7AFAFA7AFAFA7AB2
:10CE50007AFAFA7A0A7AFAFA7AFAFA7AFAFA7A7AA2
:10CE60007AFAFAFA06FE060282E2F2F2FAFAF2F22E
:10CE7000E2820206FEFE003F60DFD0DFDFDFD0DFB0
:10CE8000DFD0DEDDDBD7DFDEDEDEDEDEDFD0DDDEE7
:10CE9000DFDFD8D5D5D4DFDFD8D7D7DFD0DDDEDFF1
:10CEA000DFD8D7D7D7D8DFDFE0FFE0C0C1C7CFCF0B
:10CEB000DFDFCFCFC7C1C0C0BF7F00FE0202F2825A
:10CEC0008282F20202F29292926202020202020252
:10CED00002020212121292720202221212926202D2
:10CEE00002820202028202020202020206FE06021E
:10CEF000826212120A0A121262820206FE00007F89
:10CF000040404F4040404F40404F414244484040E5
:10CF100041414141414040404E41404040404C4AE7
:10CF200049484840404845424548404040404040CC
:10CF3000607F604041464848505048484641406004
:10CF40007F0000FE0202F2828282F20202F29292DC
:10CF50009262020202020202020202121212927291
:10CF60000202221212926202028202020282020271
:10CF70000202020206FE0602826212120A0A12125D
:10CF800062820206FEFE003F40C0CFC0C0C0CFC0DC
:10CF9000C0CFC1C2C4C8C0C0C1C1C1C1C1C0C0C06E
:10CFA000CEC1C0C0C0C0CCCAC9C8C8C0C0C8C5C234
:10CFB000C5C8C0C0C0C0C0C0E0FFE0C0C1C6C8C8CE
:10CFC000D0D0C8C8C6C1C0C0BF7F00FE06FA0A7A6A
:10CFD0007A7A0AFAFA0A6A6A6A9AFAFAFAFAFAFAA1
:10CFE000FAFAFAEAEAEA6A8AFAFADAEAEA6A9AFA01
:10CFF000FA7AFAFAFA7AFAFAFAFAFAFA06FE06026D
:10D0000082E2F2F2FAFAF2F2E2820206FE00007F17
:10D01000605F505F5F5F505F5F505E5D5B575F5F5B
:10D020005E5E5E5E5E5F5F5F515E5F5F5F5F53553A
:10D030005657575F5F575A5D5A575F5F5F5F5F5F35
:10D04000607F604041474F4F5F5F4F4F47414060B7
:10D050007F0000FE06FA0A7A7A7A0AFAFA0A6A6AFF
:10D060006A9AFAFAFAFAFAFAFAFAFAEAEAEA6A8A40
:10D07000FAFADAEAEA6A9AFAFA7AFAFAFA7AFAFA40
:10D08000FAFAFAFA06FE060282E2F2F2FAFAF2F28C
:10D09000E2820206FEFE003F60DFD0DFDFDFD0DF8E
:10D0A000DFD0DEDDDBD7DFDFDEDEDEDEDEDFDFDFB3
:10D0B000D1DEDFDFDFDFD3D5D6D7D7DFDFD7DADDCD
:10D0C000DAD7DFDFDFDFDFDFE0FFE0C0C1C7CFCFD0
:10D0D000DFDFCFCFC7C1C0C0BF7F00FCFA060606A6
:10D0E000060606060606060606060606060686E680
:10D0F000763676E686060606F6F6060606F6F606A0
:10D1000006E6F6B6B6B6B6360606060606060606FF
:10D110000606060606060606060606FAFC00003F98
:10D120005F60606060606060606060606060606000
:10D13000606E6F63636363636F6E6060676F6C6C78
:10D140006C6F6F60606C6D6D6D6D6F67606060605F
:10D150006060606060606060606060606060605FD0
:10D160003F0000FCFA0606E6C68606060606060628
:10D1700006060606060686E6763676E6860606067F
:10D18000F6F6060606F6F60606E6F6B6B6B6B636BF
:10D19000060606060606060606060606060686C6EF
:10D1A000E60606FAFCFE003F5FE0E0EFE7E3E1E0C1
:10D1B000E0E0E0E0E0E0E0E0E0EEEFE3E3E3E3E343
:10D1C000EFEEE0E0E7EFECECECEFEFE0E0ECEDEDC4
:10D1D000EDEDEFE7E0E0E0E0E0E0E0E0E0E0E0E01F
:10D1E000E0E1E3E7EFE0E0DFBF7FFF0305F9F9F9F6
:10D1F000F9F9F9F9F9F9F9F9F9F9F9F9F9F97919FF
:10D2000089E9891979F9F9F90909F9F9F90909F99E
:10D21000F91909494949C9F9F9F9F9F9F9F9F9F98E
:10D22000F9F9F9F9F9F9F9F9F9F9F90503FFFFC085
:10D23000A09F9F9F9F9F9F9F9F9F9F9F9F9F9F9FFD
:10D240009F91909C9C9C9C9C90919F9F9890939365
:10D250009390909F9F9392929290989F9F9F9F9F51
:10D260009F9F9F9F9F9F9F9F9F9F9F9F9F9F9FA0CD
:10D27000C0FF00FCFA0606060606060606060606B7
:10D28000060606066696961626060686F68606069E
:10D290000686464686C60606C606864646060686AE
:10D2A000F6860606060606060606060606060606AE
:10D2B000060606FAFC00003F5F6060606060606028
:10D2C000606060606060606064686969666060603A
:10D2D0006768686060676868646F60606F616060FD
:10D2E0006060606067686860606060606060606027
:10D2F000606060606060605F3F0000FCFA0606E608
:10D30000C6860606060606060606060666969616ED
:10D3100026060686F68606060686464686C606065D
:10D32000C606864646060686F686060606060606ED
:10D3300006060606060686C6E60606FAFCFE003F58
:10D340005FE0E0EFE7E3E1E0E0E0E0E0E0E0E0E044
:10D35000E4E8E9E9E6E0E0E0E7E8E8E0E0E7E8E87B
:10D36000E4EFE0E0EFE1E0E0E0E0E0E0E7E8E8E083
:10D37000E0E0E0E0E0E0E0E0E0E1E3E7EFE0E0DF94
:10D38000BF7FFF0305F9F9F9F9F9F9F9F9F9F9F9A5
:10D39000F9F9F9F9996969E9D9F9F9790979F9F99D
:10D3A000F979B9B97939F9F939F979B9B9F9F9796D
:10D3B0000979F9F9F9F9F9F9F9F9F9F9F9F9F9F94D
:10D3C000F9F9F90503FFFFC0A09F9F9F9F9F9F9FB3
:10D3D0009F9F9F9F9F9F9F9F9B979696999F9F9F81
:10D3E0009897979F9F9897979B909F9F909E9F9F9E
:10D3F0009F9F9F9F9897979F9F9F9F9F9F9F9F9F54
:10D400009F9F9F9F9F9F9FA0C0FF2A3E003E00F8C6
:10D41000080808080808080808C8380000000000C4
:10D42000FF0000000000000000F8070000000000FE
:10D4300000FF000000000000C03F000000000000EE
:10D440000000FF0000000000F80700000000001CC2
:10D45000221C000F080808080F0000000000002A26
:10D460003E003E00F8080808080808080808C83800
:10D470000000000000FF0000000000000000F807AE
:10D48000000000000000FF000000000000C03F009E
:10D4900000000000000000FF0000000000F807008E
:10D4A000000000001C221C000F0C0C0C0C0F0000D4
:10D4B000000000002A3E003E00F80808080808089E
:10D4C000080808C8380000000000FF000000000045
:10D4D000000000F807000000000000FF000000004E
:10D4E0000000C03F0000000000000000FF0000003E
:10D4F0000000F80700000000001C221C000F0E0EA8
:10D500000E0E0F0000000000002A3E003E00F8084A
:10D510000808080808080808C8380000000000FFCC
:10D520000000000000000000F807000000000000FC
:10D53000FF000000000000C03F00000000000000ED
:10D5400000FF0000000000F80700000000001C229F
:10D550001C000F0F0F0F0F0F0000000000002A3EED
:10D56000003E00F8080808080808080808C838003D
:10D5700000000000FF0000000000000000F80700AD
:10D580000000000000FF000000000000C03F00009D
:10D59000000000000000FF8080808080F80700000D
:10D5A0000000001C221C000F0F0F0F0F0F000000C7
:10D5B0000000002A3E003E00F80808080808080895
:10D5C0000808C8380000000000FF0000000000004C
:10D5D0000000F807000000000000FF00000000004D
:10D5E00000C03F0000000000000000FFC0C0C0C03D
:10D5F000C0F80700000000001C221C000F0F0F0FD6
:10D600000F0F0000000000002A3E003E00F808084E
:10D6100008080808080808C8380000000000FF00D3
:10D6200000000000000000F807000000000000FFFC
:10D63000000000000000C03F0000000000000000EB
:10D64000FFE0E0E0E0E0F80700000000001C221C22
:10D65000000F0F0F0F0F0F0000000000002A3E0008
:10D660003E00F8080808080808080808C83800003C
:10D67000000000FF0000000000000000F8070000AC
:10D6800000000000FF000000000000C03F0000009C
:10D690000000000000FFF0F0F0F0F0F807000000DC
:10D6A00000001C221C000F0F0F0F0F0F00000000C6
:10D6B00000002A3E003E00F808080808080808088C
:10D6C00008C8380000000000FF0000000000000053
:10D6D00000F807000000000000FF0000000000004C
:10D6E000C03F0000000000000000FFF8F8F8F8F864
:10D6F000F80700000000001C221C000F0F0F0F0F86
:10D700000F0000000000002A3E003E00F808080854
:10D71000080808080808C8380000000000FF0000DA
:10D72000000000000000F807000000000000FF00FB
:10D730000000000000C03F0000000000000000FFEB
:10D74000FCFCFCFCFCFC0700000000001C221C0090
:10D750000F0F0F0F0F0F0000000000002A3E003EC9
:10D7600000F8080808080808080808C83800000079
:10D770000000FF0000000000000000F807000000AB
:10D78000000000FF000000000000C03F000000009B
:10D7900000000000FFFEFEFEFEFEFE07000000008F
:10D7A000001C221C000F0F0F0F0F0F0000000000C5
:10D7B000002A3E003E00F808080808080808080883
:10D7C000C8380000000000FF00000000000000005A
:10D7D000F807000000000000FF000000000000C08B
:10D7E0003F0000000000000000FFFFFFFFFFFFFF01
:10D7F0000700000000001C221C000F0F0F0F0F0F6E
:10D800000000000000002A3E003E00F8080808085A
:10D810000808080808C8380000000000FF000000E1
:10D820000000000000F807000000000000FF8080FA
:10D8300080808080C03F0000000000000000FFFFEB
:10D84000FFFFFFFFFF0700000000001C221C000F6D
:10D850000F0F0F0F0F0000000000002A3E003E00D7
:10D86000F8080808080808080808C8380000000078
:10D8700000FF0000000000000000F80700000000AA
:10D880000000FFC0C0C0C0C0C0C03F00000000001A
:10D89000000000FFFFFFFFFFFFFF07000000000088
:10D8A0001C221C000F0F0F0F0F0F000000000000C4
:10D8B0002A3E003E00F8080808080808080808C8BA
:10D8C000380000000000FF0000000000000000F829
:10D8D00007000000000000FFE0E0E0E0E0E0E03FE3
:10D8E0000000000000000000FFFFFFFFFFFFFF0738
:10D8F00000000000001C221C000F0F0F0F0F0F0074
:10D9000000000000002A3E003E00F8080808080851
:10D9100008080808C8380000000000FF00000000E8
:10D9200000000000F807000000000000FFF0F0F029
:10D93000F0F0F0F03F0000000000000000FFFFFFEB
:10D94000FFFFFFFF0700000000001C221C000F0F5C
:10D950000F0F0F0F0000000000002A3E003E00F8ED
:10D96000080808080808080808C83800000000006F
:10D97000FF0000000000000000F8070000000000A9
:10D9800000FFF8F8F8F8F8F8F83F00000000000091
:10D990000000FFFFFFFFFFFFFF0700000000001C6B
:10D9A000221C000F0F0F0F0F0F0000000000002AB5
:10D9B0003E003E00F8080808080808080808C838AB
:10D9C0000000000000FF0000000000000000F80759
:10D9D000000000000000FFFCFCFCFCFCFCFC3F0025
:10D9E00000000000000000FFFFFFFFFFFFFF070037
:10D9F000000000001C221C000F0F0F0F0F0F000073
:10DA0000000000002A3E003E00F808080808080848
:10DA1000080808C8380000000000FF0000000000EF
:10DA2000000000F807000000000000FFFEFEFEFE00
:10DA3000FEFEFE3F0000000000000000FFFFFFFFB1
:10DA4000FFFFFF0700000000001C221C000F0F0F4B
:10DA50000F0F0F0000000000002A3E003E00F808F3
:10DA60000808080808080808C8380000000000FF77
:10DA70000000000000000000F807000000000000A7
:10DA8000FFFFFFFFFFFFFFFF3F000000000000005F
:10DA900000FFFFFFFFFFFFFF0700000000001C2248
:10DAA0001C000F0F0F0F0F0F0000000000002A3E98
:10DAB000003E00F8080808080808080808C83800E8
:10DAC00000000000FF8080808080808080F8070058
:10DAD0000000000000FFFFFFFFFFFFFFFF3F00000F
:10DAE000000000000000FFFFFFFFFFFFFF07000036
:10DAF0000000001C221C000F0F0F0F0F0F00000072
:10DB00000000002A3E003E00F8080808080808083F
:10DB10000808C8380000000000FFC0C0C0C0C0C076
:10DB2000C0C0F807000000000000FFFFFFFFFFFF7C
:10DB3000FFFF3F0000000000000000FFFFFFFFFFAD
:10DB4000FFFF0700000000001C221C000F0F0F0F3A
:10DB50000F0F0000000000002A3E003E00F80808F9
:10DB600008080808080808C8380000000000FFE09E
:10DB7000E0E0E0E0E0E0E0F807000000000000FF87
:10DB8000FFFFFFFFFFFFFF3F00000000000000005D
:10DB9000FFFFFFFFFFFFFF0700000000001C221C2B
:10DBA000000F0F0F0F0F0F0000000000002A3E00B3
:10DBB0003E00F8080808080808080808C8380000E7
:10DBC000000000FFF0F0F0F0F0F0F0F0F8070000D7
:10DBD00000000000FFFFFFFFFFFFFFFF3F0000000E
:10DBE0000000000000FFFFFFFFFFFFFF0700000035
:10DBF00000001C221C000F0F0F0F0F0F0000000071
:10DC000000002A3E003E00F8080808080808080836
:10DC100008C8380000000000FFF8F8F8F8F8F8F835
:10DC2000F8F807000000000000FFFFFFFFFFFFFF04
:10DC3000FF3F0000000000000000FFFFFFFFFFFFAC
:10DC4000FF0700000000001C221C000F0F0F0F0F29
:10DC50000F0000000000002A3E003E00F8080808FF
:10DC6000080808080808C8380000000000FFFCFC8D
:10DC7000FCFCFCFCFCFCFC07000000000000FFFFBB
:10DC8000FFFFFFFFFFFF3F0000000000000000FF5C
:10DC9000FFFFFFFFFFFF0700000000001C221C0029
:10DCA0000F0F0F0F0F0F0000000000002A3E003E74
:10DCB00000F8080808080808080808C83800000024
:10DCC0000000FFFEFEFEFEFEFEFEFEFE0700000060
:10DCD000000000FFFFFFFFFFFFFFFF3F000000000D
:10DCE00000000000FFFFFFFFFFFFFF070000000034
:10DCF000001C221C000F0F0F0F0F0F000000000070
:10DD0000002A3E003E00F80808080808080808082D
:10DD1000C8380000000000FFFFFFFFFFFFFFFFFF0C
:10DD2000FF07000000000000FFFFFFFFFFFFFFFFF5
:10DD30003F0000000000000000FFFFFFFFFFFFFFAB
:10DD40000700000000001C221C000F0F0F0F0F0F18
:10DD50000000000000002A3E003E00F88888888805
:10DD60008888888888C8380000000000FFFFFFFF0F
:10DD7000FFFFFFFFFFFF07000000000000FFFFFFA5
:10DD8000FFFFFFFFFF3F0000000000000000FFFF5B
:10DD9000FFFFFFFFFF0700000000001C221C000F18
:10DDA0000F0F0F0F0F0000000000002A3E003E0082
:10DDB000F8C8C8C8C8C8C8C8C8C8C8380000000063
:10DDC00000FFFFFFFFFFFFFFFFFFFF070000000056
:10DDD0000000FFFFFFFFFFFFFFFF3F00000000000C
:10DDE000000000FFFFFFFFFFFFFF07000000000033
:10DDF0001C221C000F0F0F0F0F0F0000000000006F
:10DE00002A3E003E00F8E8E8E8E8E8E8E8E8E8E864
:10DE1000380000000000FFFFFFFFFFFFFFFFFFFFD4
:10DE200007000000000000FFFFFFFFFFFFFFFF3FB4
:10DE30000000000000000000FFFFFFFFFFFFFF07E2
:10DE400000000000001C221C000F0F0F0F0F0F001E
:10DE500000000000002A3E003E00F8F8F8F8F8F84C
:10DE6000F8F8F8F8F8380000000000FFFFFFFFFFA7
:10DE7000FFFFFFFFFF07000000000000FFFFFFFFA4
:10DE8000FFFFFFFF3F0000000000000000FFFFFF5A
:10DE9000FFFFFFFF0700000000001C221C000F0F07
:10DEA0000F0F0F0F00000000000000000000000036
:10DEB0000000000000000000000000000000000062
:10DEC0000000000000000000000000000000000052
:10DED0000000000000000000000000000000000042
:10DEE0000000000000000000000000000000000032
:10DEF0000000000000000000000000000000000022
:10DF00000000000000000000000000000000000011
:10DF10000000000000000000000000000000000001
:10DF200000000000000000000000000000000000F1
:10DF300000000000000000000000000000000000E1
:10DF400000000000000000000000000000000000D1
:10DF500000000000000000000000000000000000C1
:10DF600000000000000000000000000000000000B1
:10DF700000000000000000000000000000000000A1
:10DF80000000000000000000000000000000000091
:10DF90000000000000000000000000000000000081
:10DFA0000000000000000000000000000000000071
:10DFB0000000000000000000000000000000000061
:10DFC0000000000000000000000000000000000051
:10DFD0000000000000000000000000000000000041
:10DFE0000000000000000000000000000000000031
:10DFF0000000000000000000000000000000000021
:10E000000000000000000000000000000000000010
:10E010000000000000000000000000000000000000
:10E0200000000000000000000000000000000000F0
:10E0300000000000000000000000000000000000E0
:10E0400000000000000000000000000000000000D0
:10E0500000000000000000000000000000000000C0
:10E0600000000000000000000000000000000000B0
:10E0700000000000000000000000000000000000A0
:10E080000000000000000000000000000000000090
:10E090000000000000000000000000000000008000
:10E0A000B0B4B6B636363636363636363636363618
:10E0B00036360600000000F0F0F0F0F0F0F0F0F07E
:10E0C000F0E0C00000F0F0F00000C0E0F0F0F0F090
:10E0D000F0F0F0E0C00000F0F0F00000F0F0F00030
:10E0E00000000000000000F0F0F0F0F0F0F0F0F0C0
:10E0F000E0C00000F0F0F0000000000000000000B0
:10E10000000000606C6D6D6D0D01000000000000EE
:10E1100000000000C0C0C0C0C0C0C0C000FFFFFF02
:10E12000000000000000FFFFFF0000F8F8F800000A
:10E13000FFFFFFC0C0C0C0C0FFFFFF0000F8F8F83D
:10E140000000FFFFFF1E1E1E1E1E1E0000F0F8FC3A
:10E150003C3C3C3C3CFCFFFF0000FFFFFF0000009C
:10E16000000000000000C0D8DBDBDBDBC3C0C0C0A8
:10E17000C0C0C0C0C0C0C0C0000001010101010199
:10E18000010100FFFFFFF0F0F0F0F0F0FF7F3F0033
:10E1900000FFFFFF0000F0F1F3F3F3F3F3F3FF7F71
:10E1A0003F0000FFFFFF00003F7FFFF0F0F0F0F0C6
:10E1B000F000003F7FFFF0F0F0F0F0FF7F3F000045
:10E1C0003F7FFFF0F0F0F0F0F000000206060606D8
:10E1D00006060606060606060606060606000000F1
:10E1E000000000000000000000000000000000002F
:10E1F000000000000000000000000000000000001F
:10E20000000000000000000000000000000000000E
:10E2100000000000000000000000000000000000FE
:10E2200000000000000000000000000000000000EE
:10E230000000000000000080F8FE7E0600000000E4
:10E24000000080F8FE7E060080F8FE7E0E0E0E0EA8
:10E250000E0E0E0ECEFEFC380000000E7EFEF0808C
:10E26000000000000080E0F07C1E0F0301000000B1
:10E27000000000000000000000000000000000009E
:10E28000000000000000000000000000000000008E
:10E290000000000000000000000000C0F8FFFFC701
:10E2A000C0C0C0C0C0C0C0F8FF3F0700C0F8FFFF3B
:10E2B000C7C0C0C0C0C0C0C0F0FE7F0F01000000DA
:10E2C000000000037FFFFCF0783E0F070100000014
:10E2D000000000000000000000000000000000003E
:10E2E000000000000000000000000000000000002E
:10E2F000000000000000000000000000000000E03E
:10E30000FCFF1F03030303030303E3FFFF1F0300DB
:10E31000E0FCFF1F070F3FFDF1C1010101010100FA
:10E3200000000000000080E0F07C1E0F0F3FFFF0B7
:10E33000C00000000000000000000000000000001D
:10E3400000000000000000000000000000000000CD
:10E3500000000000000000000000000000000000BD
:10E36000000000607E7F1F01000000000000607E52
:10E370007F1F0100607E7F1F010000000000030F6F
:10E380003F7C7040000080C0F0783E0F0701000025
:10E3900000000000010F7F7E700000000000000000
:10E3A000000000000000000000000000000000006D
:10E3B000000000000000000000000000000000005D
:10E3C000000000000000000000000000000000004D
:10E3D000000000000000000000000000000000003D
:10E3E000000000000000000000000000000000002D
:10E3F000000000000000000000000000000000001D
:10E40000000000000000000000000000000000000C
:10E4100000000000000000000000000000000000FC
:10E4200000000000000000000000000000000000EC
:10E4300000000000000000000000000000000000DC
:10E4400000000000000000000000000000000000CC
:10E4500000000000000000000000000000000000BC
:10E4600000000000000000000000000000000000AC
:10E47000000000000000000000000000000000009C
:10E48000000000000000000000000000000000008C
:10E49000000000000000000080808080808080807C
:10E4A000808080808080808080808080808080806C
:10E4B000808080808080808080808080808080805C
:10E4C000808080808080808080808080808080804C
:10E4D000808080808080808080808080808080803C
:10E4E000808080808080808080808080808080802C
:10E4F000808080808080808080000030F0F0F17922
:10E500003D3F3733F1F1F1793D3F3733F1F1F179A7
:10E510003D3F3733F1F1F1793D3F3733F1F1F17997
:10E520003D3F3733F1F1F1793D3F3733F1F1F17987
:10E530003D3F3733F1F1F1793D3F3733F1F1F17977
:10E540003D3F3733F1F1F1793D3F3733F1F1F17967
:10E550003D3F3733F1F1F1793D3F373301010100A0
:10E5600000000000000000000000000000000000AB
:10E57000FCFC00000000000D0D000000001C3C0031
:10E58000001C3C000000000000002020F02C20F0C7
:10E590002C120F02120F0202F0F898FE9898100841
:10E5A00019197F191F0F18242498E0380C301C0704
:10E5B000192424181834C48404040006091010090E
:10E5C000061B00003C1C00000000000000000000D2
:10E5D00000E0F81C0C000000071F383000000000AD
:10E5E0000C1CF8E000000030381F0700000080809D
:10E5F000000000000001010000008080E0E0808059
:10E6000000010107070101000000000000000000F8
:10E61000301E0E000000808080808080800101011B
:10E6200001010101000000000000000000181800B6
:10E63000000000000000C0300C00300C030000009F
:10E64000F0F87C840CF8F00F1F30213E1F0F30389B
:10E650001CFCFC00000030303F3F303030381C0CD8
:10E660009CF8F0383C3E37333130181C0C8C8CFC55
:10E67000F818383031313F1FFCFC808080FCFC00F2
:10E68000010101013F3FFCFCCCCCCC8C0C18383094
:10E6900030391F0FC0E0F0B89C8C041F3F3131317E
:10E6A0003F1F0C0C0C8CCCFC78003E3F030100009B
:10E6B000F8FC8C8C8CFCF81F3F3131313F1FF8FC8B
:10E6C0008C8C8CFCF818393131313F1F00006060B0
:10E6D000000000000006060000000000006060006E
:10E6E000000020301E0E000080C06030180C0401B5
:10E6F00003060C18302060606060606060060606EB
:10E7000006060606040C183060C0802030180C067F
:10E710000301181C0C8CCCFC78000037370100007A
:10E72000E0108848C810E007081112131209F0F829
:10E730009C8C9CF8F01F1F0101011F1FFCFCCCCC1E
:10E74000CCFC381F1F1818181F0FF8FC0C0C0C3CC1
:10E75000380F1F1818181E0EFCFC0C0C1CF8F01FAC
:10E760001F18181C0F07FCFCCCCCCC0C0C1F1F185E
:10E7700018181818FCFC8C8C8C0C0C1F1F01010144
:10E780000000F8FC0C8C8C9C980F1F1819191F0F97
:10E79000FCFCC0C0C0FCFC1F1F0000001F1F00FCD1
:10E7A000FC00000000001F1F000000000C0C0C0CFF
:10E7B0000CFCFC0E1E3830381F0FFCFCC0E070381B
:10E7C0001C1F1F0103070E1CFCFC00000000001FA3
:10E7D0001F1818181818FCFC70E070FCFC1F1F00B4
:10E7E00000001F1FFCFC3CF000FCFC1F1F00031E70
:10E7F0001F1FF0F81C0C1CF8F0070F1C181C0F074B
:10E80000FCFC8C8C8CFCF81F1F0101010100F0F84E
:10E810000C0C0CF8F0070F181A1C0F13FCFCCCCCD6
:10E82000CCFC781F1F0103071E1C70F8DCCC9C98E1
:10E8300030060C1C191D0F070C0C0CFC0C0C0C00EA
:10E8400000001F000000FCFC000000FCFC0F1F1873
:10E85000180C1F1FFCFC800080FCFC00030F1E0F27
:10E860000300FCFC00F800FCFC0F1F1C0F1C1F0F1A
:10E870000C3CF0C0F03C0C181E0701071E187CFC75
:10E88000C0C0FC7C0000001F1F0000000C0C8CCCE2
:10E89000EC7C3C1E1F1B19181818FCFC0C0C0C0CF3
:10E8A000003F3F30303030000C30C000000000002E
:10E8B0000000030C3000000C0C0C0CFCFC00303091
:10E8C00030303F3F6030180C18306000000000000E
:10E8D00000000000000000000030303030303030E8
:10E8E00000000C3C00000000000000000000006080
:10E8F000606060E0C00E1F1B1B0F1F1FFCFC80C070
:10E90000C0C0801F1F0D18181F0F80C0E06060E09E
:10E91000C0070F1C18181C0C80C0C0C080FCFC0F66
:10E920001F18180D1F1FC0E0606060E0C00F1F1BA4
:10E930001B1B1B0BC0C0F8FCCCCC0C00003F3F00E5
:10E940000000C0E0606060E0C001333636363F1F33
:10E95000FCFCC0C0C0C0801F1F0000001F1F00CCF7
:10E96000CC00000000001F1F00000000000000009D
:10E97000ECEC001C3C30303F3F00FCFC0080C0E071
:10E98000601F1F03070F1C18FCFC0000000000079D
:10E990000F1C181C0C00E0E060C060E0C01F1F00EE
:10E9A0001F001F1FE0E0C0E0E0E0C01F1F010000EB
:10E9B0001F1F80C0E060E0C080070F1C181C0F07FD
:10E9C000E0E0606060E0C03F3F0606060703C0E08D
:10E9D000606060E0E003070606063F3FE0E080C0BD
:10E9E000C060601F1F0101000000C0E06060606047
:10E9F0004008191B1B1B1E0CC0C0FCFCC0C0C00083
:10EA0000000F1F181818E0E0000000E0E0070F18E2
:10EA1000180C1F1FE0E0000000E0E000030F1C0FD7
:10EA20000300E0E0000000E0E0070F1C0F1C0F07F0
:10EA300060E0800080E060181C0703071C18E0E01D
:10EA4000000000E0E001333333333F1F606060E0DB
:10EA5000E0E0601C1E1F1B19181880C070080C0C09
:10EA60000001030E103030000000FCFC000000002C
:10EA7000003F3F000000000C0C0870C080003030E8
:10EA8000100E0301C0E0E0C00080C00301000307D6
:10EA90000703FCF8F0E0C080007F3F1F0F07030171
:10EAA000FCFE1F6183FEFC43474C484F47430C0E5E
:10EAB00007FFFF0000404C4C4F4F4C4C0C0E87C3DF
:10EAC000E77E3C4E4F4F4D4C4C4C0607036363FFB3
:10EAD000FE464E4C4C4C4F473F7F606060FFFF400E
:10EAE000404040404F4F3F3F333373E3C3464E4CAB
:10EAF0004C4E4743F0F87C6E67E3C1474F4C4C4C9B
:10EB00004F470383C3E3733F1E404F4F4040404095
:10EB1000FEFF636363FFFE474F4C4C4C4F473E7F05
:10EB2000636363FFFE464E4C4C4C4F4760F0B0B001
:10EB3000B03020444C4D4D4D4F460080C0E0F0F8C1
:10EB4000FC0103070F1F3F7F000000000000004092
:10EB50004040404040400000000000000000000035
:10EB600000000000000000000000000000000000A5
:10EB70000000000000000000000000000000000095
:10EB80000000000000000000000000000000000085
:10EB90000000000000000000000000000000000075
:10EBA0000000000000000000000000000000000065
:10EBB0000000000000000000000000000000000055
:10EBC0000000000000000000000000000000000045
:10EBD0000000000000000000000000000000000035
:10EBE000000000000000000010284444C404040495
:10EBF000C444442810000000000000000000000091
:10EC000000F008040404F4F404040484C4E4670079
:10EC10000000078484848484848404040404040835
:10EC2000F00000FF00000000FFFF1C3E77E3C18002
:10EC30000000003E7FE3C1C1C1C1C163FFFE00000F
:10EC40000000FF00003F2020202023232020202040
:10EC5000212323202020282C2C2C2C2C2C2C2F273B
:10EC6000202020203F0000000000000000000000E5
:10EC700010284444C4040404C44444281000000080
:10EC8000000000000000000000F008040404F4F498
:10EC900004040484C4E4670000000784848484843A
:10ECA0008484040404040408F00000FF0000000051
:10ECB000FFFF1C3E77E3C1800000003E7FE3C1C13F
:10ECC000C1C1C163FFFE00000000FF00003F3F3FE5
:10ECD0003F3F3C3C3F3F3F3F3E3C3C3F3F3F373365
:10ECE00033333333333330383F3F3F3F3F0000004F
:10ECF000000000000000000010284444C404040484
:10ED0000C44444281000000000000000000000007F
:10ED100000F008040404F4F404040484C4E4670068
:10ED20000000078484848484848404040404040824
:10ED3000F00000FFF8F8F8F80707E4C68F1B3978F1
:10ED4000F8F8F8C6873B39393939399B0706F8F89E
:10ED5000F8F8FF00003F3F3F3F3F3C3C3F3F3F3F15
:10ED60003E3C3C3F3F3F373333333333333330382C
:10ED70003F3F3F3F3F000000000000000000000058
:10ED800010284444C4040404C4444428100000006F
:10ED9000000000000000000000F0C8C4C4C4343407
:10EDA000C4C4C4440424A7C0C0C0C74444444444A9
:10EDB0004444C4C4C4C4C4C8F00000FFFFFFFFFF44
:10EDC0000000E3C1881C3E7FFFFFFFC1803C3E3E48
:10EDD0003E3E3E9C0001FFFFFFFFFF00003F3F3F24
:10EDE0003F3F3C3C3F3F3F3F3E3C3C3F3F3F373354
:10EDF00033333333333330383F3F3F3F3F0000003E
:10EE0000000000000000000010387C7CFCFCFCFCD2
:10EE1000FC7C7C38100000000000000000000000B6
:10EE200000F0F8FCFCFC0C0CFCFCFC7C3C1C9FFF88
:10EE3000FFFFFF7C7C7C7C7C7C7CFCFCFCFCFCF88D
:10EE4000F00000FFFFFFFFFF0000E3C1881C3E7FD2
:10EE5000FFFFFFC1803C3E3E3E3E3E9C0001FFFF67
:10EE6000FFFFFF00003F3F3F3F3F3C3C3F3F3F3FF6
:10EE70003E3C3C3F3F3F373333333333333330381B
:10EE80003F3F3F3F3F000000000000000000000047
:10EE90000000000000000000000000000000000072
:10EEA0000000000000000000000000000000000062
:10EEB0000000000000000000000000000000000052
:10EEC0000000000000000000000000000000000042
:10EED0000000000000000000000000000000000032
:10EEE00000000000000000000000FCFA0606060614
:10EEF0000606066696961626060686F68606060612
:10EF000086464686C60606C606864646060686F631
:10EF1000860606060606060606FAFC003F5F6060E7
:10EF200060606060606468696966606060676868A6
:10EF30006060676868646F60606F61606060606097
:10EF400060676868606060606060605F3F00FCFAF6
:10EF500006E6C6860606066696961626060686F611
:10EF60008606060686464686C60606C606864646C1
:10EF7000060686F6860606060686C6E606FAFCFE3F
:10EF80003F5FE0EFE7E3E1E0E0E4E8E9E9E6E0E065
:10EF9000E0E7E8E8E0E0E7E8E8E4EFE0E0EFE1E020
:10EFA000E0E0E0E0E0E7E8E8E0E0E1E3E7EFE0DF31
:10EFB000BF7FFF0305F9F9F9F9F9F9996969E9D909
:10EFC000F9F9790979F9F9F979B9B97939F9F939A1
:10EFD000F979B9B9F9F9790979F9F9F9F9F9F9F991
:10EFE000F90503FFFFC0A09F9F9F9F9F9F9B979640
:10EFF00096999F9F9F9897979F9F9897979B909F71
:10F000009F909E9F9F9F9F9F9F9897979F9F9F9F37
:10F010009F9F9FA0C0FFFCFA06060606060606068E
:10F0200006066696961626060686F68606060606E0
:10F030008686860606068606868606060606060670
:10F040000606060606FAFC003F5F606060606060CE
:10F050006060606064686969666060606768686075
:10F0600060676868686760607F656464636060604B
:10F07000606060606060605F3F00FCFA06E6C68624
:10F080000606060606066696961626060686F68680
:10F090000606060686868606060686068686060610
:10F0A000060606060686C6E606FAFCFE3F5FE0EFA9
:10F0B000E7E3E1E0E0E0E0E0E4E8E9E9E6E0E0E021
:10F0C000E7E8E8E0E0E7E8E8E8E7E0E0FFE5E4E4D7
:10F0D000E3E0E0E0E0E0E1E3E7EFE0DFBF7FFF0354
:10F0E00005F9F9F9F9F9F9F9F9F9996969E9D9F934
:10F0F000F9790979F9F9F9F9797979F9F9F979F970
:10F100007979F9F9F9F9F9F9F9F9F9F9F90503FF53
:10F11000FFC0A09F9F9F9F9F9F9F9F9F9B9796969B
:10F12000999F9F9F9897979F9F98979797989F9F32
:10F13000809A9B9B9C9F9F9F9F9F9F9F9F9F9FA00D
:10F14000C0FFF0F8FC1E0E0E1EFCF8F0FFFFFF00E3
:10F15000000000FFFFFF070F1F3C38383C1F0F0760
:10F1600080C0E0F0783C1EFEFEFE030301000000BC
:10F1700000FFFFFF000000000000003F3F3FF8FCE1
:10F18000FE1E0E0E9EFEFCF8000080E0F8FE3F0F13
:10F1900003003C3E3F3F3B38383838381C1E1E0EBB
:10F1A0000E0E1EFEFCF80000001C1C1C3EFFF7E3C8
:10F1B0001C3C3C3838383C3F1F0FFEFEFE00000070
:10F1C00000FEFEFE070F1F1C1C1C1CFFFFFF0000A3
:10F1D00000000000003F3F3FFEFEFE0E0E0E0E0E32
:10F1E0000E0E0F0F0F0E0E0E1EFEFCF838383838BC
:10F1F00038383C3F1F0FFCFEFE0E0E0E0E1E1E1C6E
:10F20000FFFFFF1C1C1C1CFCFCF81F3F3F3838385C
:10F21000383F3F1F0E0E0E0E0E0E0EFEFEFC0000BF
:10F2200000C0F0FC3F0F030100003F3F3F00000023
:10F230000000F8FCFE1E0E0E1EFEFCF8E3F7FF3E7B
:10F240001C1C3EFFF7E30F1F3F3C38383C3F1F0FAD
:10F25000FCFEFE0E0E0E0EFEFEFC0F1F1F1C1C1CE5
:10F260001CFFFFFF183838383838383F3F1FF8FC8C
:10F27000FE1E0E0E1EFEFCF8FFFFFF80000080FF4A
:10F28000FFFF0103070707070707030180C0E0F03E
:10F29000783C1EFEFEFE03030100000000FFFFFF9E
:10F2A00000000000000000070707F8FCFE1E0E0E1D
:10F2B0001EFEFCF8C0E0F0783C1E0F0703010707B4
:10F2C00007070707070707071C1E1E0E0E0E1EFE68
:10F2D000FEFC8080800006068FFFFFF9030707070A
:10F2E000070707070703FEFEFE00000000FEFEFE04
:10F2F00003070F0E0E0E0EFFFFFF000000000000C0
:10F3000000070707FEFEFE0E0E0E0E0E0E0E07077E
:10F310000707070707FFFFFE070707070707070796
:10F320000703FCFEFE0E0E0E0E1E1E1CFFFFFF0747
:10F33000070707FFFFFE030707070707070707037E
:10F340000E0E0E0E0E0ECEFEFE3C0000C0F0FC3F78
:10F350000F03000000000707070000000000F8FC92
:10F36000FE1E0E0E1EFEFCF8F9FFFF8F06068FFF35
:10F37000FFF901030707070707070301FCFEFE0E5D
:10F380000E0E0EFEFEFC03070707070707FFFFFF31
:10F39000030707070707070707030000000000002F
:10F3A000000000000000000000000000000000005D
:10F3B00000000000000000000080808080808080CD
:10F3C000808080808080808080808080808080803D
:10F3D000808080808080808080808080808080802D
:10F3E0008080808080808080808080FF808080809E
:10F3F0008482BE80808080FF80808080B2AAAAA4A0
:10F40000808080FF80808080A2A2AA94808080FF7C
:10F4100080808080868888BE808080FF80FF80809A
:10F4200080AEAAAA9280808080FF808080BCAAAA39
:10F43000BA80808080FF80808082B28A86808080CF
:10F4400080FF808080BEAAAABE80808080FF80FF6F
:10F45000808080AEAAAA9E80808080FF808084BE4B
:10F46000809CA2A29C8080FF80808084BE8084BE1D
:10F47000808080FF808084BE80A4B2AAA48080FFA8
:10F4800080FF808084BE80A2A2AA948080FF8080BA
:10F4900084BE80868888BE8080FF808084BE80AEE7
:10F4A000AAAA928080FF808084BE80BCAAAABA806B
:10F4B00080FF80FF808084BE8082B28A868080FF49
:10F4C000808084BE80BEAAAABE8080FF808084BE69
:10F4D00080AEAAAA9E8080FF80A2B2AAA4809CA22D
:10F4E000A29C80FF80FF80B2AAAAA480808482BEF2
:10F4F00080FF80B2AAAAA480B2AAAAA480FF80B288
:10F50000AAAAA480A2A2AA9480FF80B2AAAAA480D8
:10F51000868888BE80FF80FF80B2AAAAA480AEAA97
:10F52000AA9280FF80B2AAAAA480BCAAAABA80FF2D
:10F5300080B2AAAAA48082B28A8680FF80B2AAAAD8
:10F54000A480BEAAAABE80FF80FF80B2AAAAA4801F
:10F55000AEAAAA9E80FF80A2A2AA94809CA2A29C8E
:10F5600080FF80A2A2AA94808084BE8080FF80A2B7
:10F57000A2AA9480B2AAAAA480FF80FF80A2A2AA15
:10F580009480A2A2AA9480FF80A2A2AA94808688D6
:10F5900088BE80FF80A2A2AA9480AEAAAA9280FF11
:10F5A00080A2A2AA9480BCAAAABA80FF8000000010
:10F5B000000000002F00000003000300543F147EF1
:10F5C000152E2A7F2A3A22152A5422122D29112873
:10F5D0000003000000001C2241000041221C00002A
:10F5E0000C0C000008083E08080040300000080825
:10F5F000080808004000000040300806013E474966
:10F60000713E0402017F0062514946002241493E99
:10F61000000708087F004F494931003C4A49300043
:10F62000016119070036494936002649497E000024
:10F63000001200000040340000081422410014149D
:10F64000141414004122140802290502000E152B7F
:10F650002D123E0909093E3F2525251A1E2121218B
:10F66000123F2121211E3F252525213F090909019E
:10F670001E2121293A3F0404043F3F0000000021DD
:10F680004141413F3F0C1221003F202020003F0616
:10F690000C063F3F030E183F1E2121211E3F090982
:10F6A00009061E2129112E3F0909192612252912A2
:10F6B0000001013F01011F2020203F030C300C03FB
:10F6C0001F301C301F221408142203043804033195
:10F6D00029252321007F41410001060830400041D7
:10F6E000417F00040201020440404040400001020A
:10F6F0000000102A2A2A3C3F242424181C222222FB
:10F7000022182424243F1C2A2A2A2C087E090100BE
:10F710004C5252523C3F040404383D00000000208B
:10F7200040403D003F081422001F202020003C02E2
:10F730003C023C3E0402023C1C2222221C7E12128D
:10F74000120C0C1212127E3E0404020214262A32FB
:10F7500014041F2424001E2020203E061820180612
:10F760001E201C201E24181824004E5050503E22EB
:10F77000322A2622083641410000007F0000414124
:10F780003E0800180408100C0000000000000000F3
:10F790000000000000000000000000000000000069
:10F7A00000000000000000C02010D012151D111D27
:10F7B0001512101020C0FF80809F848A918086A936
:10F7C000A9BE8080FFC02010D012151D111D15127A
:10F7D000101020C0FFF0F0EFF4FAE1F0F6D9D9CE26
:10F7E000F0F0FFC02010D012151D111D15121010C1
:10F7F00020C0FFFEFEE1FAF4EFFEF8D7D7C0FEFE10
:10F80000FFC0E0D010D2D5DDD1DDD5D2D0D0E0C060
:10F81000FFFFFFE0FBF5EEFFF9D6D6C1FFFFFFC00B
:10F82000E0F030F2F7FFFFFFF7F2F0F0E0C0FFFF8B
:10F83000FFE0FBF5EEFFF9D6D6C1FFFFFF0F3FFF5C
:10F84000FCF0C00000C0F0FCFF3F0F000000000310
:10F850000F3F7E7E3F0F03000000005500810081B6
:10F86000008100412214000000006A000000000036
:10F870000001020468000000000316504000000070
:10F880000000004050160300000000010514404035
:10F8900014050100000000FFFFFFC7C7C7C7C7EF7F
:10F8A000FFFE7C0000007F7F7F01010103071F7FB7
:10F8B0007C780000000080404020202040408000F4
:10F8C000000000000E31404E9191914040310E00F9
:10F8D0000000008060100808E42424C408081060B8
:10F8E000800007182040409F8385984040201807DB
:10F8F0000000000000000000000000000000000008
:10F9000000000000000000000000000000000000F7
:10F9100000000000000000000000000000000000E7
:10F9200000000000000000000000000000000000D7
:10F9300000000000000000000000000000000000C7
:10F9400000000000000000000000000000000000B7
:10F9500000000000000000000000000000000000A7
:10F960000000000000000000000000000000000097
:10F970000000000000000000000000000000000087
:10F980000000000000000000000000000000000077
:10F99000000000000000000000000000000000FE69
:10F9A00002FA0A0A0A0A0A0A0A0A0A0A0A0A0A0ACF
:10F9B0000A0A0A0A0A0A0A0A0A0A0A0A0A0A0A0AA7
:10F9C0000A0A0A0A0A0A0A0A0A0A8A8A8A8A8A8A97
:10F9D0008A8A8A8A8A8ACACACACACACACACACACA07
:10F9E000CAEAEAEAEAEAEAEAEAEAEAEAEAFAFAFA67
:10F9F000FAFAFAFA02FE7F405F5858585858585C95
:10FA00005C5C5C5C5C5C5C5C5C5C5C5E5E5E5E5E2C
:10FA10005E5E5E5E5E5E5F5F5F5F5F5F5F5F5F5FFC
:10FA20005F5F5F5F5F5F5F5F5F5F5F5F5F5F5F5FE6
:10FA30005F5F5F5F5F5F5F5F5F5F5F5F5F5F5F5FD6
:10FA40005F5F5F5F5F5F5F5F5F5F5F407F80808062
:10FA500080808080808080808C8C8C9EBFBFBFBF68
:10FA60009292928482898595B595858982848080D9
:10FA7000888494B494848880808080808090B090C2
:10FA8000808080808080808080A080808080809F37
:10FA9000909F80969589809F958A8080BFA1A1A123
:10FAA000A1A18780808080BFA1A1A181819F80804A
:10FAB0008080BFA1818181A1BF808080809F818162
:10FAC000A1A1A1BF8080808087A1A1A1A1A1BF80A9
:10FAD000808080B1A1A1A1A1A1BF80808080BCA0B5
:10FAE000A1A1A1A1BF80808080BFA0A0A0A1A1BF33
:10FAF00080808080BFA1A1A0A0A0BF80808080BFA7
:10FB0000A1A1A1A1A0BC80808080BFA1A1A1A1A131
:10FB1000B18080808C92A1A1A181828C8080808C18
:10FB200092A18181A1928C8080808C8281A1A1A1EF
:10FB3000928C8080808092A1A1A1A1928C808080F3
:10FB40008C90A0A1A1A1928C8080808C92A1A0A079
:10FB5000A1928C8080808C92A1A1A1A0908C8080A9
:10FB6000808C92A1A1A1A192808080BE8989BE8053
:10FB7000B8A8BF80B888406070787C7E7C78706060
:10FB80004002060E1E3E7E3E1E0E060200000000D3
:10FB900000000000000000808080808080808080E5
:10FBA0008080808080808080808080809E9EBFBF9B
:10FBB000AFB7BBBDAFB7BBBDAFB7BBBDAFB7BBBDCD
:10FBC000BF9E92A1A1A1B1B9BDAFB7BBBDAFB7BB3D
:10FBD000BDAFB7BBBDBF9E92A1A1A1A1A1A1A1B183
:10FBE000B9BDAFB7BBBDAFB7BBBDBF9E92A1A1A111
:10FBF000A1A1A1A1A1A1A1A1B1B9BDAFB7BBBDBF39
:10FC00009E92A1A1A1A1A1A1A1A1A1A1A1A1A1A1F6
:10FC1000A1B1B9BDBF9E92A1A1A1A1A1A1A1A1A184
:10FC2000A1A1A1A1A1A1A1A1A1BF9E92A1A1B1A9A0
:10FC3000A5A3B1A9A5A3B1A9A5A3B1A9A5A3BFFCDB
:10FC4000FE9393FEFC8098BCE6E6BCFFFF8080FE3E
:10FC5000FE988C8698BEB7B3B3B383B0BCBFB7B3BE
:10FC6000BB9F86B0BBBBBFB7870000000000000091
:10FC70000000000000000000000000000000000084
:10FC80000000000000000000000000000000000074
:10FC90000000000000000000000000000000000064
:10FCA0000000000000000000000000000000000054
:10FCB0000000000000000000000000000000000044
:10FCC0000000000000000000000000000000000034
:10FCD000000000000000007EFFC3FF7E000607FF5B
:10FCE000FFE7F3FBDFCEC3DBDBFF7E0F1F18FFFF59
:10FCF000DFDFDBFB737EFFDBFB7103F3FB1F0F66B4
:10FD0000FFDBFF660EDFDBFFFE00000000000000EF
:10FD100000000000000000000000000406FF0604D0
:10FD200000E3F3FBDFCFC70406FF060400FFFF1864
:10FD300018FFFF0406FF0604000303FFFF03030090
:10FD4000000000000000111B1511110A04111B1FF7
:10FD50001F1F0E0446756E6B2D5369676E616C3AFA
:10FD60000050726F66692F45636F2F4E5A004465CD
:10FD7000636F64657235362F35370048656C6C6982
:10FD8000676B6569743A00416B6B756C6164756E85
:10FD9000673A00525353492D4261636B3A00486100
:10FDA0006E647265676C6572005A77656974652068
:10FDB0004C6F6B004C6F6B616472657373650046CA
:10FDC000756E6B74696F6E656E00FEFF01FFFE7FDE
:10FDD000FF80FF7F536F6674776172653A004164FC
:10FDE000722D46756E6B3A0056657262696E646577
:10FDF0006E004C6F6B2D5375636865002D2D2D2D96
:10FE00002D2D2D2D004B6F6E74726173740056652D
:10FE10007273696F6E0050726F6772616D004C6F24
:10FE20006B7761686C00537461747573005265730D
:10FE3000657400536574757000303A00200020002E
:10FE400020002000200056657262696E64756E673E
:10FE5000206D69742043445A002020206E6575206F
:10FE6000617566626175656E2E00204C6173742049
:10FE700065696E7374656C6C656E00447265686B61
:10FE80006E6F706620647275652D006475726368AC
:10FE90007A756675656872656E2E004C6F6B61646D
:10FEA00072657373652050726F67004465636F6499
:10FEB00065722050726F6772616D00636B656E2CA6
:10FEC00020756D2065696E656E0048616E647265AF
:10FED000676C65722D5479700049324320616B74F0
:10FEE00075656C6C3A200050726F6772616D6D6958
:10FEF0006572656E002020202020202020202020F8
:10FF000020004932432D416472657373653A0041A4
:10FF1000647265737365206E65753A004C6F6B6132
:10FF20006472657373653A0048617570746D656ECF
:10FF30007565005A7765697465204C6F6B004C6F6E
:10FF40006B7765636873656C004C6F6B20737563CA
:10FF500068656E0046756E6B74696F6E656E0049FC
:10FF600032432D5374617475730056657262696E05
:10FF700064656E0052616E67696572656E004175F9
:10FF8000746F66616872740043445A2D49443A2084
:10FF9000005A656E7472616C65004B6F6E747261AD
:10FFA000737400426567696E6E3A004C6F6B7761DF
:10FFB000686C004272656D736500204F4B20200015
:10FFC0004164723A2000585858582000456E6465C4
:10FFD0003A00436F64653A00576572743A005245BF
:10FFE000534554005365747570004572726F72000A
:10FFF0005265736574004164723A003F3F3F0000F0
:020000040001F9
:100000000401116F0A0E04011119D8A4FFD10001D7
:100010009F05D8A4A3D0000E9F6F070ED66FF6C021
:10002000D7F0010EA7EC13F0C00ED66FFF0ED76FFE
:10003000060ED86F000ED96F010EDA6F000EDB6F5F
:10004000000EDC6F000EDD6F000EDE6F000EDF6F46
:100050001BEC05F0010E0101556F00019A05D8A4B3
:1000600004D0010E0101536F70D0600EC26FE50E17
:10007000C36F070EC46F020EC56F000EC66F000E71
:10008000C76F050EC86F000EC96F000ECA6F000E55
:10009000CB6F000ECC6F000ECD6FF6C0CEF0F8EC3B
:1000A000FEF0600EC26FE50EC36F070EC46F020E46
:1000B000C56F000EC66F090EC76F050EC86F000E24
:1000C000C96F000ECA6F000ECB6F000ECC6F000E12
:1000D000CD6FF6C0CEF0F8ECFEF0600EC26FE50E0C
:1000E000C36F070EC46F020EC56F000EC66F120EEF
:1000F000C76F050EC86F000EC96F000ECA6F000EE5
:10010000CB6F000ECC6F000ECD6FF6C0CEF0F8ECCA
:10011000FEF0600EC26FE50EC36F070EC46F020ED5
:10012000C56F000EC66F1A0EC76F050EC86F000EA2
:10013000C96F000ECA6F000ECB6F000ECC6F000EA1
:10014000CD6FF6C0CEF0F8ECFEF0010E01015B6F52
:10015000010E586F010E576F46EC08F0010175054E
:10016000D8A431D0010EC46F295104E1320E285DAC
:10017000D8A013D04504D8A410D0000E456E000EB0
:10018000296F000E286F010E556F00019A05D8A443
:1001900021D0010E0101536F1DD0295104E11E0E23
:1001A000285DD8A017D04550D8A414D0010E456EB4
:1001B000000E296F000E286F010E556F00019A0581
:1001C000D8B4E7D707D0000E296F000E286F000EB5
:1001D000C46FF2D701017405D8A41DD0010EC36FFE
:1001E000275104E1460E265DD8A005D07305D8A49A
:1001F00002D0000E0AD0275104E1140E265DD8A0CB
:1002000012D07351D8A40FD0010E736F000E276F58
:10021000000E266F06D0000E276F000E266F000E10
:10022000C36F010E5B6F00018751D8B404D0010188
:100230004805D8A463D000018651D8B404D0010188
:100240004305D8A45BD000018551D8B404D0010186
:100250004105D8A453D001015505D8A41ED00001F2
:100260009A05D8A407D076C0D6F077C0D7F0F2ECC4
:10027000C7F006D076C0D6F077C0D7F0DDECD3F06B
:1002800076C078F077C079F078C0BCF079C0BDF066
:1002900086EC06F0000E0101556F5305D8A40DD071
:1002A00070C0D6F071C0D7F0F2ECC7F070C072F039
:1002B00071C073F0000E0101536F5B05D8A409D023
:1002C00000018F51BBECF9F08FC03FF0000E01012F
:1002D0005B6F5805D8A406D0595127EC0DF0000EDD
:1002E0000101586F5705D8A409D000018D51EBECDE
:1002F0000DF08DC08EF0000E0101576F4905D8A496
:100300002BD04A5100018719D8B423D001014A05E6
:10031000D8A410D0000E0001D76F000ED66F100EBB
:10032000D86F020ED96F080EFEECD0F0010E01015D
:10033000C56F08D0010E00019F6F000E0101C56F4F
:10034000000E486F000E02016A6F000E696F4AC10D
:1003500087F0000E0101496F4205D8A428D03D5016
:1003600000018519D8B420D03D04D8A40FD0000EC8
:10037000D76F000ED66F100ED86F020ED96F070E12
:10038000FEECD0F0010E0101C56F07D0010E9F6F8A
:10039000000E0101C56F000E416F000E02016A6F71
:1003A000000E696F3DC085F0000E0101426F4405EB
:1003B000D8A41200455100018619D8B423D00101F8
:1003C0004505D8A410D0000E0001D76F000ED66FDF
:1003D000100ED86F020ED96F090EFEECD0F0010E90
:1003E0000101C56F08D0010E00019F6F000E0101D1
:1003F000C56F000E436F000E02016A6F000E696F39
:1004000045C186F0000E0101446F12000B0E111958
:10041000D8A42BD000019F05D8A413D0070ED66F07
:10042000F6C0D7F0010EA7EC13F06A0EEA6FFE0ECD
:10043000EB6F110EEC6F2BEC0EF0000E9F6F010EA8
:100440009E6F01015705D8B404D000019E05D8A4C1
:10045000120000018D51AAEC0DF08DC08EF0000E3F
:100460009E6F000E0101576F12000C0E1119D8A4D7
:10047000EBD1100E0F6F030E106F6C0E006F6C0E31
:10048000016F6C0E026F6C0E036F00019F05D8A404
:10049000CED01E0EC26FAF0EC36F440EC46F050EDA
:1004A000C56F000EC66F0FC4C7F010C4C8F0000EB1
:1004B000C96F000ECA6F010ECB6F000ECC6F000E1D
:1004C000CD6FF6C0CEF0F8ECFEF01E0EC26FAF0E90
:1004D000C36F440EC46F050EC56F0E0EC66F0FC4FA
:1004E000C7F010C4C8F0000EC96F000ECA6F010E2D
:1004F000CB6F000ECC6F000ECD6FF6C0CEF0F8ECD7
:10050000FEF0600EC26FE50EC36F070EC46F020EE1
:10051000C56F6C0EC66F04010F510C0F0001C76F41
:1005200004011051030F0001C86F000EC96F000EC7
:10053000CA6F010ECB6F000ECC6F000ECD6FF6C0F0
:10054000CEF0F8ECFEF0600EC26FE50EC36F070E42
:10055000C46F020EC56F6C0EC66F04010F51150FEC
:100560000001C76F04011051030F0001C86F000E96
:10057000C96F000ECA6F010ECB6F000ECC6F000E5C
:10058000CD6FF6C0CEF0F8ECFEF0600EC26FE50E57
:10059000C36F070EC46F020EC56F6C0EC66F0401E9
:1005A0000F511E0F0001C76F04011051030F00010E
:1005B000C86F000EC96F000ECA6F010ECB6F000E20
:1005C000CC6F000ECD6FF6C0CEF0F8ECFEF0600EF2
:1005D000C26FE50EC36F070EC46F020EC56F6C0EBF
:1005E000C66F04010F51270F0001C76F040110519E
:1005F000030F0001C86F000EC96F000ECA6F010E15
:10060000CB6F000ECC6F000ECD6FF6C0CEF0F8ECC5
:10061000FEF03E0EEA6FFF0EEB6F0B0EEC6F2BEC55
:100620000EF0000E9F6F010E9E6F010E986F01017C
:100630005505D8B404D000019E05D8A4FAD0E80E20
:100640000001765D030E7759D8A018D0270EBF6F32
:10065000100EBE6F76C0BCF077C0BDF07CEC14F01D
:10066000BCC0C2F0BDC0C3F0030EC56FE80EC46FBE
:100670002DEC13F0C251600F0401006F000177519F
:1006800004E1640E765DD8A018D0030EBF6FE80EAB
:10069000BE6F76C0BCF077C0BDF07CEC14F0BCC07F
:1006A000C2F0BDC0C3F0000EC56F640EC46F2DEC68
:1006B00013F0C251600F0401016F0001775104E192
:1006C0000A0E765DD8A018D0000EBF6F640EBE6F04
:1006D00076C0BCF077C0BDF07CEC14F0BCC0C2F0BA
:1006E000BDC0C3F0000EC56F0A0EC46F2DEC13F031
:1006F000C251600F0401026F76C0BCF077C0BDF03C
:10070000000E0001BF6F0A0EBE6F7CEC14F0BC51EE
:10071000600F0401036F600E0001C26FE50EC36F2E
:10072000070EC46F020EC56F00C4C6F004010F515E
:100730000C0F0001C76F04011051030F0001C86FB7
:10074000000EC96F000ECA6F010ECB6F000ECC6F8A
:10075000000ECD6FF6C0CEF0F8ECFEF0600EC26F6A
:10076000E50EC36F070EC46F020EC56F01C4C6F05D
:1007700004010F51150F0001C76F04011051030F41
:100780000001C86F000EC96F000ECA6F010ECB6F5B
:10079000000ECC6F000ECD6FF6C0CEF0F8ECFEF080
:1007A000600EC26FE50EC36F070EC46F020EC56FF9
:1007B00002C4C6F004010F511E0F0001C76F0401EF
:1007C0001051030F0001C86F000EC96F000ECA6FF1
:1007D000010ECB6F000ECC6F000ECD6FF6C0CEF0C9
:1007E000F8ECFEF0600EC26FE50EC36F070EC46F2B
:1007F000020EC56F03C4C6F004010F51270F00019C
:10080000C76F04011051030F0001C86F000EC96FBC
:10081000000ECA6F010ECB6F000ECC6F000ECD6FB5
:10082000F6C0CEF0F8ECFEF0000E9E6F000E010157
:10083000556F410E0001BC6F140EBD6F9851A1ECB5
:100840000CF00101556F1200640E1119D8A499D350
:1008500000019F05D8A415D0070ED66FF6C0D7F0BB
:10086000010EA7EC13F0280EEA6FFF0EEB6F0B0ED4
:10087000EC6F2BEC0EF0000E9F6F010E9E6F010EC1
:10088000946F9605D8B466D39E05D8A4120062D39F
:100890001E0EE96FFE0EEA6F080EEB6FA5C0ECF0BE
:1008A000020E23ECF2F0690EC26FFC0EC36F5A0EFB
:1008B000C46F010EC56F000EC66F000EC76F040E29
:1008C000C86F000EC96F000ECA6F000ECB6F000E0E
:1008D000CC6F000ECD6FF6C0CEF0F8ECFEF0160E29
:1008E000D66FFE0ED76F080ED86F030ED96F040EA9
:1008F000DA6F000EDB6F000EDC6F000EDD6F000E96
:10090000DE6F010EDF6F8DECE6F0690EC26FFC0E3C
:10091000C36F660EC46F010EC56F000EC66F000E6A
:10092000C76F050EC86F000EC96F000ECA6F000EAC
:10093000CB6F000ECC6F000ECD6FF6C0CEF0F8EC92
:10094000FEF0BF0ED66FFD0ED76F0B0ED86F030EE5
:10095000D96F050EDA6F000EDB6F000EDC6F000E34
:10096000DD6F000EDE6F010EDF6F8DECE6F0690EBD
:10097000C26FFC0EC36F660EC46F010EC56F000E12
:10098000C66F000EC76F060EC86F000EC96F000E4F
:10099000CA6F000ECB6F000ECC6F000ECD6FF6C08D
:1009A000CEF0F8ECFEF0330ED66FFE0ED76F060ECB
:1009B000D86F030ED96F060EDA6F000EDB6F000ED4
:1009C000DC6F000EDD6F000EDE6F010EDF6F8DEC51
:1009D000E6F0690EC26FFC0EC36F660EC46F010EA7
:1009E000C56F000EC66F000EC76F070EC86F000EF2
:1009F000C96F000ECA6F000ECB6F000ECC6F000ED9
:100A0000CD6FF6C0CEF0F8ECFEF0260ED66FFE0EDF
:100A1000D76F070ED86F030ED96F070EDA6F000E6F
:100A2000DB6F000EDC6F000EDD6F000EDE6F010E5F
:100A3000DF6F8DECE6F09ED2160EE96FFE0EEA6FC8
:100A4000080EEB6FA5C0ECF0030E23ECF2F0690E7C
:100A5000C26FFC0EC36F5A0EC46F010EC56F000E3D
:100A6000C66F000EC76F020EC86F000EC96F000E72
:100A7000CA6F000ECB6F000ECC6F000ECD6FF6C0AC
:100A8000CEF0F8ECFEF01E0ED66FFE0ED76F080EFD
:100A9000D86F030ED96F020EDA6F000EDB6F000EF7
:100AA000DC6F000EDD6F000EDE6F010EDF6F8DEC70
:100AB000E6F0690EC26FFC0EC36F5A0EC46F010ED2
:100AC000C56F000EC66F000EC76F050EC86F000E13
:100AD000C96F000ECA6F000ECB6F000ECC6F000EF8
:100AE000CD6FF6C0CEF0F8ECFEF0BF0ED66FFD0E67
:100AF000D76F0B0ED86F030ED96F050EDA6F000E8D
:100B0000DB6F000EDC6F000EDD6F000EDE6F010E7E
:100B1000DF6F8DECE6F02BD7BF0EE96FFD0EEA6FAD
:100B20000B0EEB6FA5C0ECF0040E23ECF2F0690E97
:100B3000C26FFC0EC36F5A0EC46F010EC56F000E5C
:100B4000C66F000EC76F020EC86F000EC96F000E91
:100B5000CA6F000ECB6F000ECC6F000ECD6FF6C0CB
:100B6000CEF0F8ECFEF01E0ED66FFE0ED76F080E1C
:100B7000D86F030ED96F020EDA6F000EDB6F000E16
:100B8000DC6F000EDD6F000EDE6F010EDF6F8DEC8F
:100B9000E6F0690EC26FFC0EC36F5A0EC46F010EF1
:100BA000C56F000EC66F000EC76F030EC86F000E34
:100BB000C96F000ECA6F000ECB6F000ECC6F000E17
:100BC000CD6FF6C0CEF0F8ECFEF0160ED66FFE0E2E
:100BD000D76F080ED86F030ED96F030EDA6F000EB1
:100BE000DB6F000EDC6F000EDD6F000EDE6F010E9E
:100BF000DF6F8DECE6F0690EC26FFC0EC36F5A0E0C
:100C0000C46F010EC56F000EC66F000EC76F060ED3
:100C1000C86F000EC96F000ECA6F000ECB6F000EBA
:100C2000CC6F000ECD6FF6C0CEF0F8ECFEF0BBD668
:100C3000330EE96FFE0EEA6F060EEB6FA5C0ECF007
:100C4000050E23ECF2F0690EC26FFC0EC36F5A0E54
:100C5000C46F010EC56F000EC66F000EC76F020E87
:100C6000C86F000EC96F000ECA6F000ECB6F000E6A
:100C7000CC6F000ECD6FF6C0CEF0F8ECFEF01E0E7D
:100C8000D66FFE0ED76F080ED86F030ED96F020E07
:100C9000DA6F000EDB6F000EDC6F000EDD6F000EF2
:100CA000DE6F010EDF6F8DECE6F0690EC26FFC0E99
:100CB000C36F5A0EC46F010EC56F000EC66F000ED3
:100CC000C76F030EC86F000EC96F000ECA6F000E0B
:100CD000CB6F000ECC6F000ECD6FF6C0CEF0F8ECEF
:100CE000FEF0160ED66FFE0ED76F080ED86F030EED
:100CF000D96F030EDA6F000EDB6F000EDC6F000E93
:100D0000DD6F000EDE6F010EDF6F8DECE6F0690E19
:100D1000C26FFC0EC36F5A0EC46F010EC56F000E7A
:100D2000C66F000EC76F040EC86F000EC96F000EAD
:100D3000CA6F000ECB6F000ECC6F000ECD6FF6C0E9
:100D4000CEF0F8ECFEF0BF0ED66FFD0ED76F0B0E97
:100D5000D86F030ED96F040EDA6F000EDB6F000E32
:100D6000DC6F000EDD6F000EDE6F010EDF6F8DECAD
:100D7000E6F0690EC26FFC0EC36F5A0EC46F010E0F
:100D8000C56F000EC66F000EC76F070EC86F000E4E
:100D9000C96F000ECA6F000ECB6F000ECC6F000E35
:100DA000CD6FF6C0CEF0F8ECFEF02FD6260EE96F30
:100DB000FE0EEA6F070EEB6FA5C0ECF0060E23ECFB
:100DC000F2F0690EC26FFC0EC36F5A0EC46F010EB3
:100DD000C56F000EC66F000EC76F020EC86F000E03
:100DE000C96F000ECA6F000ECB6F000ECC6F000EE5
:100DF000CD6FF6C0CEF0F8ECFEF01E0ED66FFE0EF4
:100E0000D76F080ED86F030ED96F020EDA6F000E7F
:100E1000DB6F000EDC6F000EDD6F000EDE6F010E6B
:100E2000DF6F8DECE6F0690EC26FFC0EC36F5A0ED9
:100E3000C46F010EC56F000EC66F000EC76F030EA4
:100E4000C86F000EC96F000ECA6F000ECB6F000E88
:100E5000CC6F000ECD6FF6C0CEF0F8ECFEF0160EA3
:100E6000D66FFE0ED76F080ED86F030ED96F030E24
:100E7000DA6F000EDB6F000EDC6F000EDD6F000E10
:100E8000DE6F010EDF6F8DECE6F0690EC26FFC0EB7
:100E9000C36F5A0EC46F010EC56F000EC66F000EF1
:100EA000C76F040EC86F000EC96F000ECA6F000E28
:100EB000CB6F000ECC6F000ECD6FF6C0CEF0F8EC0D
:100EC000FEF0BF0ED66FFD0ED76F0B0ED86F030E60
:100ED000D96F040EDA6F000EDB6F000EDC6F000EB0
:100EE000DD6F000EDE6F010EDF6F8DECE6F0690E38
:100EF000C26FFC0EC36F5A0EC46F010EC56F000E99
:100F0000C66F000EC76F050EC86F000EC96F000ECA
:100F1000CA6F000ECB6F000ECC6F000ECD6FF6C007
:100F2000CEF0F8ECFEF0330ED66FFE0ED76F060E45
:100F3000D86F030ED96F050EDA6F000EDB6F000E4F
:100F4000DC6F000EDD6F000EDE6F010EDF6F8DECCB
:100F5000E6F010D09451010AD8B49AD4030AD8B458
:100F60006BD5010AD8B4D8D5070AD8B461D6010A1E
:100F7000D8B41CD794C095F0000E966F000E9E6FEB
:100F80001200650E1119D8A470D000019F05D8A4D5
:100F900047D0070ED66FF6C0D7F0010EA7EC13F0BE
:100FA000AB0EEA6FFF0EEB6F080EEC6F2BEC0EF042
:100FB0001C0ED66FFF0ED76F0C0ED86F000ED96FB8
:100FC000020EDA6F000EDB6F000EDC6F000EDD6FBD
:100FD000000EDE6F000EDF6F1BEC05F0B105D8A42C
:100FE00006D05A0ED66F480E54ECFBF013D0020E0A
:100FF000B119D8A406D05A0ED66F200E54ECFBF0CF
:1010000009D0030EB119D8A405D05A0ED66F200E00
:1010100054ECFBF0000E9F6F010E9E6F010E986F57
:1010200001015505D8B404D000019E05D8A412D002
:1010300076C0D6F077C0D7F00A0E0001D86F040E44
:10104000D96FA5C0DAF00BECCBF0000E9E6F000E4E
:101050000101556F410E0001BC6F140EBD6F985118
:10106000A1EC0CF00101556F12006D0E1119D8A4FE
:1010700048D300019F05D8A494D1070ED66FF6C0BF
:10108000D7F0010EA7EC13F0630EEA6FFF0EEB6FC3
:10109000070EEC6F2BEC0EF09051D8B459D0870EA0
:1010A000D66FFD0ED76F0C0ED86F000ED96F020EE3
:1010B000DA6F000EDB6F000EDC6F000EDD6F000ECE
:1010C000DE6F010EDF6F8DECE6F0540ED66FFD0E75
:1010D000D76F0D0ED86F000ED96F030EDA6F000EAA
:1010E000DB6F000EDC6F000EDD6F000EDE6F010E99
:1010F000DF6F8DECE6F0DE0ED66FFD0ED76F0A0EB9
:10110000D86F000ED96F040EDA6F000EDB6F000E81
:10111000DC6F000EDD6F000EDE6F010EDF6F8DECF9
:10112000E6F0930ED66FFD0ED76F0B0ED86F000E44
:10113000D96F050EDA6F000EDB6F000EDC6F000E4C
:10114000DD6F000EDE6F010EDF6F8DECE6F058D024
:10115000880ED66FFF0ED76F090ED86F000ED96FAD
:10116000020EDA6F000EDB6F000EDC6F000EDD6F1B
:10117000000EDE6F010EDF6F8DECE6F0D90ED66F3C
:10118000FE0ED76F0E0ED86F000ED96F030EDA6FFA
:10119000000EDB6F000EDC6F000EDD6F000EDE6FE9
:1011A000010EDF6F8DECE6F0020ED66FFF0ED76FEB
:1011B0000D0ED86F000ED96F040EDA6F000EDB6FC4
:1011C000000EDC6F000EDD6F000EDE6F010EDF6FB4
:1011D0008DECE6F05F0ED66FFF0ED76F0B0ED86F5B
:1011E000000ED96F050EDA6F000EDB6F000EDC6F9C
:1011F000000EDD6F000EDE6F010EDF6F8DECE6F08E
:101200007B0ED66FFD0ED76F0C0ED86F000ED96F08
:10121000060EDA6F000EDB6F000EDC6F000EDD6F66
:10122000000EDE6F010EDF6F8DECE6F0D40ED66F90
:10123000FD0ED76F0A0ED86F000ED96F070EDA6F4A
:10124000000EDB6F000EDC6F000EDD6F000EDE6F38
:10125000010EDF6F8DECE6F0C70ED66FFF0ED76F75
:10126000050ED86F4F0ED96F020EDA6F000EDB6FCE
:10127000000EDC6F000EDD6F000EDE6F010EDF6F03
:101280008DECE6F0C70ED66FFF0ED76F050ED86F48
:101290004F0ED96F030EDA6F000EDB6F000EDC6F9E
:1012A000000EDD6F000EDE6F010EDF6F8DECE6F0DD
:1012B000C70ED66FFF0ED76F050ED86F4F0ED96FC2
:1012C000040EDA6F000EDB6F000EDC6F000EDD6FB8
:1012D000000EDE6F010EDF6F8DECE6F0C70ED66FED
:1012E000FF0ED76F050ED86F4F0ED96F050EDA6F50
:1012F000000EDB6F000EDC6F000EDD6F000EDE6F88
:10130000010EDF6F8DECE6F0C70ED66FFF0ED76FC4
:10131000050ED86F4F0ED96F060EDA6F000EDB6F19
:10132000000EDC6F000EDD6F000EDE6F010EDF6F52
:101330008DECE6F0390ED66FFE0ED76F030ED86F28
:10134000420ED96F070EDA6F000EDB6F000EDC6FF6
:10135000000EDD6F000EDE6F010EDF6F8DECE6F02C
:10136000F20ED66F020ED76F050ED86F4F0ED96FE3
:10137000070EDA6F000EDB6F000EDC6F000EDD6F04
:10138000000EDE6F010EDF6F8DECE6F0000E9F6F3A
:10139000010E0101666F010EB36F010EB16F010EF8
:1013A000AC6F00019051D8B4B3D001015E05D8A450
:1013B0002AD0FC0E0001D66FFE0ED76F060ED86F36
:1013C000430ED96F020EDA6F000EDB6F000EDC6F7A
:1013D000000EDD6F000EDE6F000EDF6F8DECE6F0AD
:1013E0000CC1D6F00DC1D7F04F0ED86F020ED96FD9
:1013F000000EDA6F000EDB6F000EDC6F9DECD6F096
:10140000000E01015E6F6305D8A429D0FC0E000117
:10141000D66FFE0ED76F060ED86F430ED96F030E30
:10142000DA6F000EDB6F000EDC6F000EDD6F000E5A
:10143000DE6F000EDF6F8DECE6F064C1D6F0D76B87
:101440004F0ED86F030ED96F000EDA6F000EDB6FF0
:10145000000EDC6F9DECD6F0000E0101636FB3054A
:10146000D8A429D0FC0E0001D66FFE0ED76F060E51
:10147000D86F430ED96F040EDA6F000EDB6F000ECB
:10148000DC6F000EDD6F000EDE6F000EDF6F8DEC87
:10149000E6F05AC0D6F0D76B4F0ED86F040ED96F56
:1014A000000EDA6F000EDB6F000EDC6F9DECD6F0E5
:1014B000000E0101B36F9E05D8A4F5D0FC0E00010B
:1014C000D66FFE0ED76F060ED86F430ED96F050E7E
:1014D000DA6F000EDB6F000EDC6F000EDD6F000EAA
:1014E000DE6F000EDF6F8DECE6F0A2C1D6F0D76B99
:1014F0004F0ED86F050ED96F000EDA6F000EDB6F3E
:10150000000EDC6F9DECD6F0000E01019E6FCBD07B
:1015100001016605D8A429D0FC0E0001D66FFE0E8D
:10152000D76F060ED86F430ED96F020EDA6F000E1A
:10153000DB6F000EDC6F000EDD6F000EDE6F000E45
:10154000DF6F8DECE6F041C0D6F0D76B4F0ED86F51
:10155000020ED96F000EDA6F000EDB6F000EDC6F2B
:101560009DECD6F0000E0101666FB105D8A44ED0F7
:10157000FC0E0001D66FFE0ED76F060ED86F430E1D
:10158000D96F030EDA6F000EDB6F000EDC6F000EFA
:10159000DD6F000EDE6F000EDF6F8DECE6F0B5C084
:1015A000D6F0D76B4F0ED86F030ED96F000EDA6FDF
:1015B000000EDB6F000EDC6F9DECD6F0FC0ED66FDC
:1015C000FE0ED76F060ED86F430ED96F040EDA6F7A
:1015D000000EDB6F000EDC6F000EDD6F000EDE6FA5
:1015E000000EDF6F8DECE6F0B2C0D6F0D76B4F0E79
:1015F000D86F040ED96F000EDA6F000EDB6F000E8D
:10160000DC6F9DECD6F0000E0101B16FAC05D8A4E3
:101610004AD0FC0E0001D66FFE0ED76F060ED86FB3
:10162000430ED96F050EDA6F000EDB6F000EDC6F14
:10163000000EDD6F000EDE6F000EDF6F8DECE6F04A
:10164000AF05D8A417D0BA0ED66FFF0ED76F060E0F
:10165000D86F4A0ED96F050EDA6F000EDB6F000EE1
:10166000DC6F000EDD6F000EDE6F010EDF6F8DECA4
:10167000E6F016D0EA0ED66FFF0ED76F060ED86FC3
:10168000490ED96F050EDA6F000EDB6F000EDC6FAE
:10169000000EDD6F000EDE6F010EDF6F8DECE6F0E9
:1016A000000E0101AC6F7E05D8A41200FC0E0001F3
:1016B000D66FFE0ED76F060ED86F430ED96F060E8B
:1016C000DA6F000EDB6F000EDC6F000EDD6F000EB8
:1016D000DE6F000EDF6F8DECE6F01AC1D6F01BC195
:1016E000D7F04F0ED86F060ED96F000EDA6F000ECE
:1016F000DB6F000EDC6F9DECD6F0000E01017E6FFB
:1017000012006E0E1119D8A496D300019F05D8A41B
:1017100015D0070ED66FF6C0D7F0010EA7EC13F068
:10172000E70EEA6FFE0EEB6F0E0EEC6F2BEC0EF079
:10173000000E9F6F010E9E6F010E946F9605D8B438
:1017400068D39E05D8A4120064D36E0EE96FFD0E17
:10175000EA6F0D0EEB6FA5C0ECF0020E23ECF2F079
:10176000690EC26FFC0EC36F5A0EC46F010EC56FB7
:10177000000EC66F000EC76F040EC86F000EC96F53
:10178000000ECA6F000ECB6F000ECC6F000ECD6F37
:10179000F6C0CEF0F8ECFEF0610ED66FFD0ED76FFE
:1017A0000D0ED86F030ED96F040EDA6F000EDB6FCB
:1017B000000EDC6F000EDD6F000EDE6F010EDF6FBE
:1017C0008DECE6F0690EC26FFC0EC36F660EC46F3F
:1017D000010EC56F000EC66F000EC76F050EC86FF5
:1017E000000EC96F000ECA6F000ECB6F000ECC6FDB
:1017F000000ECD6FF6C0CEF0F8ECFEF0B40ED66F52
:10180000FD0ED76F0B0ED86F030ED96F050EDA6F72
:10181000000EDB6F000EDC6F000EDD6F000EDE6F62
:10182000010EDF6F8DECE6F0690EC26FFC0EC36F28
:10183000660EC46F010EC56F000EC66F000EC76F37
:10184000060EC86F000EC96F000ECA6F000ECB6F78
:10185000000ECC6F000ECD6FF6C0CEF0F8ECFEF0AF
:10186000440ED66FFE0ED76F020ED86F030ED96FDF
:10187000060EDA6F000EDB6F000EDC6F000EDD6F00
:10188000000EDE6F010EDF6F8DECE6F0690EC26FA9
:10189000FC0EC36F660EC46F010EC56F000EC66FDF
:1018A000000EC76F070EC86F000EC96F000ECA6F1B
:1018B000000ECB6F000ECC6F000ECD6FF6C0CEF0D9
:1018C000F8ECFEF0420ED66FFE0ED76F020ED86F08
:1018D000030ED96F070EDA6F000EDB6F000EDC6FA0
:1018E000000EDD6F000EDE6F010EDF6F8DECE6F097
:1018F000BAEF87F0610EE96FFD0EEA6F0D0EEB6F28
:10190000A5C0ECF0030E23ECF2F0690EC26FFC0EE2
:10191000C36F5A0EC46F010EC56F000EC66F000E66
:10192000C76F020EC86F000EC96F000ECA6F000E9F
:10193000CB6F000ECC6F000ECD6FF6C0CEF0F8EC82
:10194000FEF06E0ED66FFD0ED76F0D0ED86F030E24
:10195000D96F020EDA6F000EDB6F000EDC6F000E27
:10196000DD6F000EDE6F010EDF6F8DECE6F0690EAD
:10197000C26FFC0EC36F5A0EC46F010EC56F000E0E
:10198000C66F000EC76F050EC86F000EC96F000E40
:10199000CA6F000ECB6F000ECC6F000ECD6FF6C07D
:1019A000CEF0F8ECFEF0B40ED66FFD0ED76F0B0E36
:1019B000D86F030ED96F050EDA6F000EDB6F000EC5
:1019C000DC6F000EDD6F000EDE6F010EDF6F8DEC41
:1019D000E6F02AD7B40EE96FFD0EEA6F0B0EEB6F3F
:1019E000A5C0ECF0040E23ECF2F0690EC26FFC0E01
:1019F000C36F5A0EC46F010EC56F000EC66F000E86
:101A0000C76F020EC86F000EC96F000ECA6F000EBE
:101A1000CB6F000ECC6F000ECD6FF6C0CEF0F8ECA1
:101A2000FEF06E0ED66FFD0ED76F0D0ED86F030E43
:101A3000D96F020EDA6F000EDB6F000EDC6F000E46
:101A4000DD6F000EDE6F010EDF6F8DECE6F0690ECC
:101A5000C26FFC0EC36F5A0EC46F010EC56F000E2D
:101A6000C66F000EC76F030EC86F000EC96F000E61
:101A7000CA6F000ECB6F000ECC6F000ECD6FF6C09C
:101A8000CEF0F8ECFEF0610ED66FFD0ED76F0D0EA6
:101A9000D86F030ED96F030EDA6F000EDB6F000EE6
:101AA000DC6F000EDD6F000EDE6F010EDF6F8DEC60
:101AB000E6F0690EC26FFC0EC36F5A0EC46F010EC2
:101AC000C56F000EC66F000EC76F060EC86F000E02
:101AD000C96F000ECA6F000ECB6F000ECC6F000EE8
:101AE000CD6FF6C0CEF0F8ECFEF0BAD6440EE96F3A
:101AF000FE0EEA6F020EEB6FA5C0ECF0050E23ECB4
:101B0000F2F0690EC26FFC0EC36F5A0EC46F010E65
:101B1000C56F000EC66F000EC76F020EC86F000EB5
:101B2000C96F000ECA6F000ECB6F000ECC6F000E97
:101B3000CD6FF6C0CEF0F8ECFEF06E0ED66FFD0E57
:101B4000D76F0D0ED86F030ED96F020EDA6F000E2D
:101B5000DB6F000EDC6F000EDD6F000EDE6F010E1E
:101B6000DF6F8DECE6F0690EC26FFC0EC36F5A0E8C
:101B7000C46F010EC56F000EC66F000EC76F030E57
:101B8000C86F000EC96F000ECA6F000ECB6F000E3B
:101B9000CC6F000ECD6FF6C0CEF0F8ECFEF0610E0B
:101BA000D66FFD0ED76F0D0ED86F030ED96F030ED3
:101BB000DA6F000EDB6F000EDC6F000EDD6F000EC3
:101BC000DE6F010EDF6F8DECE6F0690EC26FFC0E6A
:101BD000C36F5A0EC46F010EC56F000EC66F000EA4
:101BE000C76F040EC86F000EC96F000ECA6F000EDB
:101BF000CB6F000ECC6F000ECD6FF6C0CEF0F8ECC0
:101C0000FEF0B40ED66FFD0ED76F0B0ED86F030E1D
:101C1000D96F040EDA6F000EDB6F000EDC6F000E62
:101C2000DD6F000EDE6F010EDF6F8DECE6F0690EEA
:101C3000C26FFC0EC36F5A0EC46F010EC56F000E4B
:101C4000C66F000EC76F070EC86F000EC96F000E7B
:101C5000CA6F000ECB6F000ECC6F000ECD6FF6C0BA
:101C6000CEF0F8ECFEF02ED6420EE96FFE0EEA6FD3
:101C7000020EEB6FA5C0ECF0060E23ECF2F0690E3D
:101C8000C26FFC0EC36F5A0EC46F010EC56F000EFB
:101C9000C66F000EC76F020EC86F000EC96F000E30
:101CA000CA6F000ECB6F000ECC6F000ECD6FF6C06A
:101CB000CEF0F8ECFEF06E0ED66FFD0ED76F0D0E67
:101CC000D86F030ED96F020EDA6F000EDB6F000EB5
:101CD000DC6F000EDD6F000EDE6F010EDF6F8DEC2E
:101CE000E6F0690EC26FFC0EC36F5A0EC46F010E90
:101CF000C56F000EC66F000EC76F030EC86F000ED3
:101D0000C96F000ECA6F000ECB6F000ECC6F000EB5
:101D1000CD6FF6C0CEF0F8ECFEF0610ED66FFD0E82
:101D2000D76F0D0ED86F030ED96F030EDA6F000E4A
:101D3000DB6F000EDC6F000EDD6F000EDE6F010E3C
:101D4000DF6F8DECE6F0690EC26FFC0EC36F5A0EAA
:101D5000C46F010EC56F000EC66F000EC76F040E74
:101D6000C86F000EC96F000ECA6F000ECB6F000E59
:101D7000CC6F000ECD6FF6C0CEF0F8ECFEF0B40ED6
:101D8000D66FFD0ED76F0B0ED86F030ED96F040EF2
:101D9000DA6F000EDB6F000EDC6F000EDD6F000EE1
:101DA000DE6F010EDF6F8DECE6F0690EC26FFC0E88
:101DB000C36F5A0EC46F010EC56F000EC66F000EC2
:101DC000C76F050EC86F000EC96F000ECA6F000EF8
:101DD000CB6F000ECC6F000ECD6FF6C0CEF0F8ECDE
:101DE000FEF0440ED66FFE0ED76F020ED86F030EB4
:101DF000D96F050EDA6F000EDB6F000EDC6F000E80
:101E0000DD6F000EDE6F010EDF6F8DECE6F0BAEFD6
:101E100087F09451010AD8B498D4030AD8B46AD58B
:101E2000010AD8B4D7D5070AD8B460D6010AD8B405
:101E30001BD7BAEF87F06F0E1119D8A4BCD20001DE
:101E40009F05D8A4EED0070ED66FF6C0D7F0010ECE
:101E5000A7EC13F0AB0EEA6FFE0EEB6F100EEC6FFB
:101E60002BEC0EF0B3D0D20ED66FFF0ED76F060E4E
:101E7000D86F000ED96F020EDA6F000EDB6F000E06
:101E8000DC6F000EDD6F000EDE6F000EDF6F1BECEF
:101E900005F0D80ED66FFF0ED76F060ED86F000E66
:101EA000D96F040EDA6F000EDB6F000EDC6F000ED0
:101EB000DD6F000EDE6F000EDF6F1BEC05F04604D9
:101EC000D8A40AD0010ED66F020ED76F000ED86FBD
:101ED0006E51A8ECE0F016D0C70ED66FFF0ED76F8C
:101EE000050ED86F460ED96F020EDA6F000EDB6F4B
:101EF000000EDC6F000EDD6F000EDE6F000EDF6F78
:101F00001BEC05F001017605D8A40ED06AC0D6F00E
:101F10006BC0D7F0010E0001D86F040ED96F000E10
:101F2000DA6F57ECD9F059D0C60E0001D66FFF0E0C
:101F3000D76F060ED86F3E0ED96F040EDA6F000E03
:101F4000DB6F000EDC6F000EDD6F000EDE6F000E2B
:101F5000DF6F1BEC05F041D0D20ED66FFF0ED76FAE
:101F6000060ED86F000ED96F020EDA6F000EDB6F0F
:101F7000000EDC6F000EDD6F000EDE6F000EDF6FF7
:101F80001BEC05F04604D8A40AD0010ED66F020E51
:101F9000D76F000ED86F6E51A8ECE0F01ED0C70EC0
:101FA000D66FFF0ED76F050ED86F460ED96F020E93
:101FB000DA6F000EDB6F000EDC6F000EDD6F000EBF
:101FC000DE6F000EDF6F1BEC05F007D09D51010A9C
:101FD000D8B4C2D7020AD8B446D70A0EC26FC30E0D
:101FE000C36F440EC46F020EC56F010EC66F100E94
:101FF000C76F060EC86F000EC96F000ECA6F000EC5
:10200000CB6F000ECC6F000ECD6FF6C0CEF0F8ECAB
:10201000FEF0000E9F6F010E9E6F010E946F010E79
:10202000966F9605D8B420D130D1600EC26FE50E00
:10203000C36F070EC46F020EC56F000EC66F250E6C
:10204000C76F040EC86F000EC96F000ECA6F000E76
:10205000CB6F000ECC6F000ECD6FF6C0CEF0F8EC5B
:10206000FEF00A0EC26FC30EC36F440EC46F020EA1
:10207000C56F010EC66F100EC76F060EC86F000E3B
:10208000C96F000ECA6F000ECB6F000ECC6F000E32
:10209000CD6FF6C0CEF0F8ECFEF0600EC26FE50E2C
:1020A000C36F070EC46F020EC56F5F0EC66F250E9D
:1020B000C76F020EC86F000EC96F000ECA6F000E08
:1020C000CB6F000ECC6F000ECD6FF6C0CEF0F8ECEB
:1020D000FEF0D4D0600EC26FE50EC36F070EC46F62
:1020E000020EC56F000EC66F250EC76F020EC86FB9
:1020F000000EC96F000ECA6F000ECB6F000ECC6FC2
:10210000000ECD6FF6C0CEF0F8ECFEF09D05D8B411
:1021100039D00A0EC26FC30EC36F440EC46F020ED5
:10212000C56F010EC66F100EC76F060EC86F000E8A
:10213000C96F000ECA6F000ECB6F000ECC6F000E81
:10214000CD6FF6C0CEF0F8ECFEF0600EC26FE50E7B
:10215000C36F070EC46F020EC56F5F0EC66F250EEC
:10216000C76F040EC86F000EC96F000ECA6F000E55
:10217000CB6F000ECC6F000ECD6FF6C0CEF0F8EC3A
:10218000FEF07CD00A0EC26FC30EC36F440EC46F44
:10219000020EC56F020EC66F100EC76F060EC86F17
:1021A000000EC96F000ECA6F000ECB6F000ECC6F11
:1021B000000ECD6FF6C0CEF0F8ECFEF05FD0600EF2
:1021C000C26FE50EC36F070EC46F020EC56F000E1F
:1021D000C66F250EC76F020EC86F000EC96F000EC6
:1021E000CA6F000ECB6F000ECC6F000ECD6FF6C025
:1021F000CEF0F8ECFEF0600EC26FE50EC36F070E76
:10220000C46F020EC56F000EC66F250EC76F040E99
:10221000C86F000EC96F000ECA6F000ECB6F000EA4
:10222000CC6F000ECD6FF6C0CEF0F8ECFEF00A0ECB
:10223000C26FC30EC36F440EC46F020EC56F020E91
:10224000C66F100EC76F060EC86F000EC96F000E66
:10225000CA6F000ECB6F000ECC6F000ECD6FF6C0B4
:10226000CEF0F8ECFEF00AD09451010AD8B4DDD6D5
:10227000030AD8B42FD7010AD8B4A1D794C095F0D7
:10228000000E966F000E9E6F25D001013E05D8A46A
:102290000ED0010E0001D66F020ED76FA5C0D8F088
:1022A0006C51A8ECE0F0000E01013E6F13D03D052B
:1022B000D8A410D068C0D6F069C0D7F0010E0001D4
:1022C000D86F040ED96FA5C0DAF057ECD9F0000E24
:1022D00001013D6F00019E05D8A453D09C05D8A4F0
:1022E0000AD0010ED66F020ED76F010ED86F6C5157
:1022F000A8ECE0F043D09B05D8A40DD068C0D6F080
:1023000069C0D7F0010ED86F040ED96F010EDA6FD5
:1023100057ECD9F033D04604D8A430D09D05D8A4CA
:1023200004D0020E9519D8B40DD001017605D8A4B9
:1023300025D0030E00019519D8A420D0030E9D19B5
:10234000D8A41CD00A0EC26FC30EC36F440EC46F54
:10235000020EC56F030EC66F100EC76F060EC86F54
:10236000000EC96F000ECA6F000ECB6F000ECC6F4F
:10237000000ECD6FF6C0CEF0F8ECFEF0000E0001BE
:102380009E6F9C05D8A40AD0410EBC6F140EBD6F81
:102390009851A1EC0CF001013E6F12009B05D8A4EE
:1023A0001200410EBC6F140EBD6F9851A1EC0CF0E1
:1023B00001013D6F1200700E1119D8A46ED00001FA
:1023C0009F05D8A445D0070ED66FF6C0D7F0010EF2
:1023D000A7EC13F09B0EEA6FFE0EEB6F100EEC6F86
:1023E0002BEC0EF00F0ED66FFF0ED76F0D0ED86FC1
:1023F000000ED96F020EDA6F000EDB6F000EDC6F7D
:10240000000EDD6F000EDE6F000EDF6F1BEC05F0BF
:10241000B105D8A406D05A0ED66F480E54ECFBF086
:1024200013D0020EB119D8A406D05A0ED66F200EC2
:1024300054ECFBF009D0030EB119D8A405D05A0E04
:10244000D66F200E54ECFBF0000E9F6F010E9E6FB6
:1024500001013C05D8B404D000019E05D8A412D0D7
:1024600066C0D6F067C0D7F00A0E0001D86F040E20
:10247000D96FA5C0DAF00BECCBF0000E9E6F000E0A
:1024800001013C6F410E0001BC6F140EBD6F9851ED
:10249000A1EC0CF001013C6F1200780E1119D8A4C8
:1024A00096D300019F05D8A415D0070ED66FF6C0AD
:1024B000D7F0010EA7EC13F0E40EEA6FFF0EEB6FFE
:1024C000060EEC6F2BEC0EF0000E9F6F010E9E6F50
:1024D000010E946F9605D8B468D39E05D8A4120057
:1024E00064D3050EE96FFE0EEA6F090EEB6FA5C00F
:1024F000ECF0020E23ECF2F0690EC26FFC0EC36F1B
:102500005A0EC46F010EC56F000EC66F000EC76F66
:10251000040EC86F000EC96F000ECA6F000ECB6F9D
:10252000000ECC6F000ECD6FF6C0CEF0F8ECFEF0D2
:102530009E0ED66FFD0ED76F0B0ED86F030ED96FA0
:10254000040EDA6F000EDB6F000EDC6F000EDD6F25
:10255000000EDE6F010EDF6F8DECE6F0690EC26FCC
:10256000FC0EC36F660EC46F010EC56F000EC66F02
:10257000000EC76F050EC86F000EC96F000ECA6F40
:10258000000ECB6F000ECC6F000ECD6FF6C0CEF0FC
:10259000F8ECFEF0FC0ED66FFD0ED76F090ED86F6B
:1025A000030ED96F050EDA6F000EDB6F000EDC6FC5
:1025B000000EDD6F000EDE6F010EDF6F8DECE6F0BA
:1025C000690EC26FFC0EC36F660EC46F010EC56F3D
:1025D000000EC66F000EC76F060EC86F000EC96FE3
:1025E000000ECA6F000ECB6F000ECC6F000ECD6FC9
:1025F000F6C0CEF0F8ECFEF0E80ED66FFD0ED76F09
:102600000A0ED86F030ED96F060EDA6F000EDB6F5D
:10261000000EDC6F000EDD6F000EDE6F010EDF6F4F
:102620008DECE6F0690EC26FFC0EC36F660EC46FD0
:10263000010EC56F000EC66F000EC76F070EC86F84
:10264000000EC96F000ECA6F000ECB6F000ECC6F6C
:10265000000ECD6FF6C0CEF0F8ECFEF02D0ED66F6A
:10266000FE0ED76F060ED86F030ED96F070EDA6F06
:10267000000EDB6F000EDC6F000EDD6F000EDE6FF4
:10268000010EDF6F8DECE6F0BAEF87F09E0EE96F7A
:10269000FD0EEA6F0B0EEB6FA5C0ECF0030E23EC02
:1026A000F2F0690EC26FFC0EC36F5A0EC46F010EBA
:1026B000C56F000EC66F000EC76F020EC86F000E0A
:1026C000C96F000ECA6F000ECB6F000ECC6F000EEC
:1026D000CD6FF6C0CEF0F8ECFEF0050ED66FFE0E14
:1026E000D76F090ED86F030ED96F020EDA6F000E86
:1026F000DB6F000EDC6F000EDD6F000EDE6F010E73
:10270000DF6F8DECE6F0690EC26FFC0EC36F5A0EE0
:10271000C46F010EC56F000EC66F000EC76F050EA9
:10272000C86F000EC96F000ECA6F000ECB6F000E8F
:10273000CC6F000ECD6FF6C0CEF0F8ECFEF0FC0EC4
:10274000D66FFD0ED76F090ED86F030ED96F050E29
:10275000DA6F000EDB6F000EDC6F000EDD6F000E17
:10276000DE6F010EDF6F8DECE6F02AD7FC0EE96F0D
:10277000FD0EEA6F090EEB6FA5C0ECF0040E23EC22
:10278000F2F0690EC26FFC0EC36F5A0EC46F010ED9
:10279000C56F000EC66F000EC76F020EC86F000E29
:1027A000C96F000ECA6F000ECB6F000ECC6F000E0B
:1027B000CD6FF6C0CEF0F8ECFEF0050ED66FFE0E33
:1027C000D76F090ED86F030ED96F020EDA6F000EA5
:1027D000DB6F000EDC6F000EDD6F000EDE6F010E92
:1027E000DF6F8DECE6F0690EC26FFC0EC36F5A0E00
:1027F000C46F010EC56F000EC66F000EC76F030ECB
:10280000C86F000EC96F000ECA6F000ECB6F000EAE
:10281000CC6F000ECD6FF6C0CEF0F8ECFEF09E0E41
:10282000D66FFD0ED76F0B0ED86F030ED96F030E48
:10283000DA6F000EDB6F000EDC6F000EDD6F000E36
:10284000DE6F010EDF6F8DECE6F0690EC26FFC0EDD
:10285000C36F5A0EC46F010EC56F000EC66F000E17
:10286000C76F060EC86F000EC96F000ECA6F000E4C
:10287000CB6F000ECC6F000ECD6FF6C0CEF0F8EC33
:10288000FEF0BAD6E80EE96FFD0EEA6F0A0EEB6FA6
:10289000A5C0ECF0050E23ECF2F0690EC26FFC0E41
:1028A000C36F5A0EC46F010EC56F000EC66F000EC7
:1028B000C76F020EC86F000EC96F000ECA6F000E00
:1028C000CB6F000ECC6F000ECD6FF6C0CEF0F8ECE3
:1028D000FEF0050ED66FFE0ED76F090ED86F030EF1
:1028E000D96F020EDA6F000EDB6F000EDC6F000E88
:1028F000DD6F000EDE6F010EDF6F8DECE6F0690E0E
:10290000C26FFC0EC36F5A0EC46F010EC56F000E6E
:10291000C66F000EC76F030EC86F000EC96F000EA2
:10292000CA6F000ECB6F000ECC6F000ECD6FF6C0DD
:10293000CEF0F8ECFEF09E0ED66FFD0ED76F0B0EAC
:10294000D86F030ED96F030EDA6F000EDB6F000E27
:10295000DC6F000EDD6F000EDE6F010EDF6F8DECA1
:10296000E6F0690EC26FFC0EC36F5A0EC46F010E03
:10297000C56F000EC66F000EC76F040EC86F000E45
:10298000C96F000ECA6F000ECB6F000ECC6F000E29
:10299000CD6FF6C0CEF0F8ECFEF0FC0ED66FFD0E5B
:1029A000D76F090ED86F030ED96F040EDA6F000EC1
:1029B000DB6F000EDC6F000EDD6F000EDE6F010EB0
:1029C000DF6F8DECE6F0690EC26FFC0EC36F5A0E1E
:1029D000C46F010EC56F000EC66F000EC76F070EE5
:1029E000C86F000EC96F000ECA6F000ECB6F000ECD
:1029F000CC6F000ECD6FF6C0CEF0F8ECFEF02ED608
:102A00002D0EE96FFE0EEA6F060EEB6FA5C0ECF01F
:102A1000060E23ECF2F0690EC26FFC0EC36F5A0E65
:102A2000C46F010EC56F000EC66F000EC76F020E99
:102A3000C86F000EC96F000ECA6F000ECB6F000E7C
:102A4000CC6F000ECD6FF6C0CEF0F8ECFEF0050EA8
:102A5000D66FFE0ED76F090ED86F030ED96F020E18
:102A6000DA6F000EDB6F000EDC6F000EDD6F000E04
:102A7000DE6F010EDF6F8DECE6F0690EC26FFC0EAB
:102A8000C36F5A0EC46F010EC56F000EC66F000EE5
:102A9000C76F030EC86F000EC96F000ECA6F000E1D
:102AA000CB6F000ECC6F000ECD6FF6C0CEF0F8EC01
:102AB000FEF09E0ED66FFD0ED76F0B0ED86F030E75
:102AC000D96F030EDA6F000EDB6F000EDC6F000EA5
:102AD000DD6F000EDE6F010EDF6F8DECE6F0690E2C
:102AE000C26FFC0EC36F5A0EC46F010EC56F000E8D
:102AF000C66F000EC76F040EC86F000EC96F000EC0
:102B0000CA6F000ECB6F000ECC6F000ECD6FF6C0FB
:102B1000CEF0F8ECFEF0FC0ED66FFD0ED76F090E6E
:102B2000D86F030ED96F040EDA6F000EDB6F000E44
:102B3000DC6F000EDD6F000EDE6F010EDF6F8DECBF
:102B4000E6F0690EC26FFC0EC36F5A0EC46F010E21
:102B5000C56F000EC66F000EC76F050EC86F000E62
:102B6000C96F000ECA6F000ECB6F000ECC6F000E47
:102B7000CD6FF6C0CEF0F8ECFEF0E80ED66FFD0E8D
:102B8000D76F0A0ED86F030ED96F050EDA6F000EDD
:102B9000DB6F000EDC6F000EDD6F000EDE6F010ECE
:102BA000DF6F8DECE6F0BAEF87F09451010AD8B4EC
:102BB00098D4030AD8B46AD5010AD8B4D7D5070A7D
:102BC000D8B460D6010AD8B41BD7BAEF87F0790E13
:102BD0001119D8A45AD000019F05D8A42FD0070EF0
:102BE000D66FF6C0D7F0010EA7EC13F09A0EEA6F7D
:102BF000FF0EEB6F090EEC6F2BEC0EF0000E9F6FCB
:102C0000000E986FF80E9225D66FD76BFF0ED72364
:102C10002E0ED86F020ED96F000EDA6F000EDB6F2A
:102C2000000EDC6F1EECCEF0050ED66F9251F80F41
:102C3000D76F070E17EC0CF0080F926F01016A05B1
:102C4000D8A41200F80E6B250001D66FD76BFF0ECB
:102C5000D7232E0ED86F020ED96F000EDA6F000E3A
:102C6000DB6F000EDC6F1EECCEF0050ED66F01019F
:102C70006B51F80F0001D76F070E17EC0CF0080F1F
:102C8000926F000E01016A6F12007A0E1119D8A41A
:102C9000A1EF9BF000019F05D8A415D0070ED66FB9
:102CA000F6C0D7F0010EA7EC13F0CA0EEA6FFE0EC5
:102CB000EB6F0F0EEC6F2BEC0EF0000E9F6F010E02
:102CC000946F010E966F9605D8B483EF9AF092EF49
:102CD0009AF0B005D8A455D00A0EC26FC30EC36FC8
:102CE000440EC46F020EC56F110EC66F080EC76F7B
:102CF000020EC86F000EC96F000ECA6F000ECB6FB8
:102D0000000ECC6F000ECD6FF6C0CEF0F8ECFEF0EA
:102D10000A0EC26FC30EC36F440EC46F020EC56F9E
:102D2000160EC66F080EC76F040EC86F000EC96F6F
:102D3000000ECA6F000ECB6F000ECC6F000ECD6F71
:102D4000F6C0CEF0F8ECFEF00A0EC26FC30EC36FF1
:102D5000440EC46F020EC56F120EC66F080EC76F09
:102D6000060EC86F000EC96F000ECA6F000ECB6F43
:102D7000000ECC6F000ECD6FF6C0CEF0F8ECFEF07A
:102D8000B1D0020EB019D8A455D00A0EC26FC30E2E
:102D9000C36F440EC46F020EC56F0F0EC66F080ED0
:102DA000C76F020EC86F000EC96F000ECA6F000E0B
:102DB000CB6F000ECC6F000ECD6FF6C0CEF0F8ECEE
:102DC000FEF00A0EC26FC30EC36F440EC46F020E34
:102DD000C56F180EC66F080EC76F040EC86F000EC1
:102DE000C96F000ECA6F000ECB6F000ECC6F000EC5
:102DF000CD6FF6C0CEF0F8ECFEF00A0EC26FC30E37
:102E0000C36F440EC46F020EC56F120EC66F080E5C
:102E1000C76F060EC86F000EC96F000ECA6F000E96
:102E2000CB6F000ECC6F000ECD6FF6C0CEF0F8EC7D
:102E3000FEF058D0030EB019D8A454D00A0EC26FB9
:102E4000C30EC36F440EC46F020EC56F0F0EC66F64
:102E5000080EC76F020EC86F000EC96F000ECA6F52
:102E6000000ECB6F000ECC6F000ECD6FF6C0CEF013
:102E7000F8ECFEF00A0EC26FC30EC36F440EC46FAF
:102E8000020EC56F160EC66F080EC76F040EC86F10
:102E9000000EC96F000ECA6F000ECB6F000ECC6F14
:102EA000000ECD6FF6C0CEF0F8ECFEF00A0EC26F49
:102EB000C30EC36F440EC46F020EC56F140EC66FEF
:102EC000080EC76F060EC86F000EC96F000ECA6FDE
:102ED000000ECB6F000ECC6F000ECD6FF6C0CEF0A3
:102EE000F8ECFEF0600EC26FE50EC36F070EC46F04
:102EF000020EC56F000EC66F500EC76F040EC86F6E
:102F0000000EC96F000ECA6F000ECB6F000ECC6FA3
:102F1000000ECD6FF6C0CEF0F8ECFEF0600EC26F82
:102F2000E50EC36F070EC46F020EC56F000EC66FAD
:102F3000500EC76F060EC86F000EC96F000ECA6F25
:102F4000000ECB6F000ECC6F000ECD6FF6C0CEF032
:102F5000F8ECFEF0600EC26FE50EC36F070EC46F93
:102F6000020EC56F6B0EC66F500EC76F020EC86F94
:102F7000000EC96F000ECA6F000ECB6F000ECC6F33
:102F8000000ECD6FF6C0CEF0F8ECFEF0C7D2020E08
:102F9000B019D8A455D00A0EC26FC30EC36F440E29
:102FA000C46F020EC56F0E0EC66F080EC76F020EFD
:102FB000C86F000EC96F000ECA6F000ECB6F000EF7
:102FC000CC6F000ECD6FF6C0CEF0F8ECFEF00A0E1E
:102FD000C26FC30EC36F440EC46F020EC56F190ECD
:102FE000C66F080EC76F040EC86F000EC96F000EC3
:102FF000CA6F000ECB6F000ECC6F000ECD6FF6C007
:10300000CEF0F8ECFEF00A0EC26FC30EC36F440E92
:10301000C46F020EC56F120EC66F080EC76F060E84
:10302000C86F000EC96F000ECA6F000ECB6F000E86
:10303000CC6F000ECD6FF6C0CEF0F8ECFEF0B0D045
:10304000B005D8A455D00A0EC26FC30EC36F440E8C
:10305000C46F020EC56F100EC66F080EC76F020E4A
:10306000C86F000EC96F000ECA6F000ECB6F000E46
:10307000CC6F000ECD6FF6C0CEF0F8ECFEF00A0E6D
:10308000C26FC30EC36F440EC46F020EC56F170E1E
:10309000C66F080EC76F040EC86F000EC96F000E12
:1030A000CA6F000ECB6F000ECC6F000ECD6FF6C056
:1030B000CEF0F8ECFEF00A0EC26FC30EC36F440EE2
:1030C000C46F020EC56F120EC66F080EC76F060ED4
:1030D000C86F000EC96F000ECA6F000ECB6F000ED6
:1030E000CC6F000ECD6FF6C0CEF0F8ECFEF058D0ED
:1030F000030EB019D8A454D00A0EC26FC30EC36F0A
:10310000440EC46F020EC56F0E0EC66F080EC76F59
:10311000020EC86F000EC96F000ECA6F000ECB6F93
:10312000000ECC6F000ECD6FF6C0CEF0F8ECFEF0C6
:103130000A0EC26FC30EC36F440EC46F020EC56F7A
:10314000170EC66F080EC76F040EC86F000EC96F4A
:10315000000ECA6F000ECB6F000ECC6F000ECD6F4D
:10316000F6C0CEF0F8ECFEF00A0EC26FC30EC36FCD
:10317000440EC46F020EC56F140EC66F080EC76FE3
:10318000060EC86F000EC96F000ECA6F000ECB6F1F
:10319000000ECC6F000ECD6FF6C0CEF0F8ECFEF056
:1031A000600EC26FE50EC36F070EC46F020EC56FCF
:1031B000000EC66F500EC76F020EC86F000EC96FAB
:1031C000000ECA6F000ECB6F000ECC6F000ECD6FDD
:1031D000F6C0CEF0F8ECFEF0600EC26FE50EC36FE5
:1031E000070EC46F020EC56F000EC66F500EC76F7C
:1031F000060EC86F000EC96F000ECA6F000ECB6FAF
:10320000000ECC6F000ECD6FF6C0CEF0F8ECFEF0E5
:10321000600EC26FE50EC36F070EC46F020EC56F5E
:103220006B0EC66F500EC76F040EC86F000EC96FCD
:10323000000ECA6F000ECB6F000ECC6F000ECD6F6C
:10324000F6C0CEF0F8ECFEF069D1030EB019D8A4A8
:1032500055D00A0EC26FC30EC36F440EC46F020E68
:10326000C56F0E0EC66F080EC76F020EC86F000E38
:10327000C96F000ECA6F000ECB6F000ECC6F000E30
:10328000CD6FF6C0CEF0F8ECFEF00A0EC26FC30EA2
:10329000C36F440EC46F020EC56F160EC66F080EC4
:1032A000C76F040EC86F000EC96F000ECA6F000E04
:1032B000CB6F000ECC6F000ECD6FF6C0CEF0F8ECE9
:1032C000FEF00A0EC26FC30EC36F440EC46F020E2F
:1032D000C56F150EC66F080EC76F060EC86F000EBD
:1032E000C96F000ECA6F000ECB6F000ECC6F000EC0
:1032F000CD6FF6C0CEF0F8ECFEF0B0D0B005D8A49B
:1033000055D00A0EC26FC30EC36F440EC46F020EB7
:10331000C56F100EC66F080EC76F020EC86F000E85
:10332000C96F000ECA6F000ECB6F000ECC6F000E7F
:10333000CD6FF6C0CEF0F8ECFEF00A0EC26FC30EF1
:10334000C36F440EC46F020EC56F160EC66F080E13
:10335000C76F040EC86F000EC96F000ECA6F000E53
:10336000CB6F000ECC6F000ECD6FF6C0CEF0F8EC38
:10337000FEF00A0EC26FC30EC36F440EC46F020E7E
:10338000C56F130EC66F080EC76F060EC86F000E0E
:10339000C96F000ECA6F000ECB6F000ECC6F000E0F
:1033A000CD6FF6C0CEF0F8ECFEF058D0020EB0199A
:1033B000D8A454D00A0EC26FC30EC36F440EC46F9C
:1033C000020EC56F0E0EC66F080EC76F020EC86FD5
:1033D000000EC96F000ECA6F000ECB6F000ECC6FCF
:1033E000000ECD6FF6C0CEF0F8ECFEF00A0EC26F04
:1033F000C30EC36F440EC46F020EC56F180EC66FA6
:10340000080EC76F040EC86F000EC96F000ECA6F9A
:10341000000ECB6F000ECC6F000ECD6FF6C0CEF05D
:10342000F8ECFEF00A0EC26FC30EC36F440EC46FF9
:10343000020EC56F130EC66F080EC76F060EC86F5B
:10344000000EC96F000ECA6F000ECB6F000ECC6F5E
:10345000000ECD6FF6C0CEF0F8ECFEF0600EC26F3D
:10346000E50EC36F070EC46F020EC56F000EC66F68
:10347000500EC76F020EC86F000EC96F000ECA6FE4
:10348000000ECB6F000ECC6F000ECD6FF6C0CEF0ED
:10349000F8ECFEF0600EC26FE50EC36F070EC46F4E
:1034A000020EC56F000EC66F500EC76F040EC86FB8
:1034B000000EC96F000ECA6F000ECB6F000ECC6FEE
:1034C000000ECD6FF6C0CEF0F8ECFEF0600EC26FCD
:1034D000E50EC36F070EC46F020EC56F6B0EC66F8D
:1034E000500EC76F060EC86F000EC96F000ECA6F70
:1034F000000ECB6F000ECC6F000ECD6FF6C0CEF07D
:10350000F8ECFEF00BD09451010AD8B469EF96F0B4
:10351000030AD8B43CD5010AD8B497D694C095F024
:10352000000E966F9E05D8A412009505D8A455D01C
:103530000A0EC26FC30EC36F440EC46F020EC56F76
:10354000110EC66F080EC76F020EC86F000EC96F4E
:10355000000ECA6F000ECB6F000ECC6F000ECD6F49
:10356000F6C0CEF0F8ECFEF00A0EC26FC30EC36FC9
:10357000440EC46F020EC56F160EC66F080EC76FDD
:10358000040EC86F000EC96F000ECA6F000ECB6F1D
:10359000000ECC6F000ECD6FF6C0CEF0F8ECFEF052
:1035A0000A0EC26FC30EC36F440EC46F020EC56F06
:1035B000120EC66F080EC76F060EC86F000EC96FD9
:1035C000000ECA6F000ECB6F000ECC6F000ECD6FD9
:1035D000F6C0CEF0F8ECFEF0B1D0020E9519D8A4EA
:1035E00055D00A0EC26FC30EC36F440EC46F020ED5
:1035F000C56F0E0EC66F080EC76F020EC86F000EA5
:10360000C96F000ECA6F000ECB6F000ECC6F000E9C
:10361000CD6FF6C0CEF0F8ECFEF00A0EC26FC30E0E
:10362000C36F440EC46F020EC56F190EC66F080E2D
:10363000C76F040EC86F000EC96F000ECA6F000E70
:10364000CB6F000ECC6F000ECD6FF6C0CEF0F8EC55
:10365000FEF00A0EC26FC30EC36F440EC46F020E9B
:10366000C56F120EC66F080EC76F060EC86F000E2C
:10367000C96F000ECA6F000ECB6F000ECC6F000E2C
:10368000CD6FF6C0CEF0F8ECFEF058D0030E9519D1
:10369000D8A454D00A0EC26FC30EC36F440EC46FB9
:1036A000020EC56F0E0EC66F080EC76F020EC86FF2
:1036B000000EC96F000ECA6F000ECB6F000ECC6FEC
:1036C000000ECD6FF6C0CEF0F8ECFEF00A0EC26F21
:1036D000C30EC36F440EC46F020EC56F160EC66FC5
:1036E000080EC76F040EC86F000EC96F000ECA6FB8
:1036F000000ECB6F000ECC6F000ECD6FF6C0CEF07B
:10370000F8ECFEF00A0EC26FC30EC36F440EC46F16
:10371000020EC56F150EC66F080EC76F060EC86F76
:10372000000EC96F000ECA6F000ECB6F000ECC6F7B
:10373000000ECD6FF6C0CEF0F8ECFEF0000E9E6FDE
:1037400012007B0E1119D8A41AD000019F05D8A42D
:103750001200070ED66FF6C0D7F0010EA7EC13F0DB
:10376000910EEA6FFF0EEB6F090EEC6F2BEC0EF073
:10377000000E9F6F010E9E6F010E946F12007C0E63
:103780001119D8A40AD100019F05D8A441D0070E71
:10379000D66FF6C0D7F0010EA7EC13F06A0EEA6FF1
:1037A000FF0EEB6F0A0EEC6F2BEC0EF0460ED66F91
:1037B000FE0ED76F130ED86F000ED96F020EDA6FA0
:1037C000000EDB6F000EDC6F000EDD6F000EDE6F93
:1037D000010EDF6F8DECE6F0590ED66FFE0ED76F3F
:1037E000110ED86F000ED96F030EDA6F000EDB6F6B
:1037F000000EDC6F000EDD6F000EDE6F010EDF6F5E
:103800008DECE6F0000E9F6F020E946F010E966F26
:103810009605D8B4B9D09E05D8A41200B5D09E059F
:10382000D8A41DD00A0EC26FC30EC36F440EC46F5E
:10383000020EC56F090EC66F100EC76F040EC86F5B
:10384000000EC96F000ECA6F000ECB6F000ECC6F5A
:10385000000ECD6FF6C0CEF0F8ECFEF01CD00A0ED4
:10386000C26FC30EC36F440EC46F020EC56F080E45
:10387000C66F100EC76F040EC86F000EC96F000E22
:10388000CA6F000ECB6F000ECC6F000ECD6FF6C06E
:10389000CEF0F8ECFEF00A0EC26FC30EC36F440EFA
:1038A000C46F020EC56F1D0EC66F100EC76F060ED9
:1038B000C86F000EC96F000ECA6F000ECB6F000EEE
:1038C000CC6F000ECD6FF6C0CEF0F8ECFEF0BAEF84
:1038D00087F00A0EC26FC30EC36F440EC46F020E90
:1038E000C56F070EC66F100EC76F040EC86F000EAF
:1038F000C96F000ECA6F000ECB6F000ECC6F000EAA
:10390000CD6FF6C0CEF0F8ECFEF09E05D8A41ED028
:103910000A0EC26FC30EC36F440EC46F020EC56F92
:103920001F0EC66F100EC76F060EC86F000EC96F50
:10393000000ECA6F000ECB6F000ECC6F000ECD6F65
:10394000F6C0CEF0F8ECFEF0BAEF87F00A0EC26FC8
:10395000C30EC36F440EC46F020EC56F1E0EC66F3A
:10396000100EC76F060EC86F000EC96F000ECA6F2B
:10397000000ECB6F000ECC6F000ECD6FF6C0CEF0F8
:10398000F8ECFEF0BAEF87F09451010AD8B447D7AB
:10399000030AD8B49ED7BAEF87F0810E1119D8A4C4
:1039A0006CD000019F05D8A41200070ED66FF6C098
:1039B000D7F0010EA7EC13F0F00EEA6FFF0EEB6FDD
:1039C000060EEC6F2BEC0EF07B0ED66FFE0ED76F53
:1039D000100ED86F060ED96F030EDA6F000EDB6F74
:1039E000000EDC6F000EDD6F000EDE6F000EDF6F6D
:1039F0008DECE6F0BB0ED66FFE0ED76F0F0ED86FB4
:103A00000A0ED96F040EDA6F000EDB6F000EDC6F4A
:103A1000000EDD6F000EDE6F000EDF6F8DECE6F046
:103A2000DE0ED66FFF0ED76F060ED86F240ED96F3D
:103A3000050EDA6F000EDB6F000EDC6F000EDD6F1F
:103A4000000EDE6F000EDF6F8DECE6F08B0ED66F92
:103A5000FE0ED76F100ED86F080ED96F060EDA6FF4
:103A6000000EDB6F000EDC6F000EDD6F000EDE6FF0
:103A7000000EDF6F8DECE6F07BD6820E1119D8A414
:103A800096D300019F05D8A415D0070ED66FF6C0B7
:103A9000D7F0010EA7EC13F0540EEA6FFF0EEB6F98
:103AA0000B0EEC6F2BEC0EF0000E9F6F010E9E6F55
:103AB000010E946F9605D8B468D39E05D8A4120061
:103AC00064D3A90EE96FFD0EEA6F0B0EEB6FA5C074
:103AD000ECF0020E23ECF2F0690EC26FFC0EC36F25
:103AE0005A0EC46F010EC56F000EC66F000EC76F71
:103AF000040EC86F000EC96F000ECA6F000ECB6FA8
:103B0000000ECC6F000ECD6FF6C0CEF0F8ECFEF0DC
:103B1000F20ED66FFD0ED76F0A0ED86F030ED96F57
:103B2000040EDA6F000EDB6F000EDC6F000EDD6F2F
:103B3000000EDE6F010EDF6F8DECE6F0690EC26FD6
:103B4000FC0EC36F660EC46F010EC56F000EC66F0C
:103B5000000EC76F050EC86F000EC96F000ECA6F4A
:103B6000000ECB6F000ECC6F000ECD6FF6C0CEF006
:103B7000F8ECFEF0400ED66FFE0ED76F020ED86F37
:103B8000030ED96F050EDA6F000EDB6F000EDC6FCF
:103B9000000EDD6F000EDE6F010EDF6F8DECE6F0C4
:103BA000690EC26FFC0EC36F660EC46F010EC56F47
:103BB000000EC66F000EC76F060EC86F000EC96FED
:103BC000000ECA6F000ECB6F000ECC6F000ECD6FD3
:103BD000F6C0CEF0F8ECFEF03E0ED66FFE0ED76FBC
:103BE000020ED86F030ED96F060EDA6F000EDB6F70
:103BF000000EDC6F000EDD6F000EDE6F010EDF6F5A
:103C00008DECE6F0690EC26FFC0EC36F660EC46FDA
:103C1000010EC56F000EC66F000EC76F070EC86F8E
:103C2000000EC96F000ECA6F000ECB6F000ECC6F76
:103C3000000ECD6FF6C0CEF0F8ECFEF03C0ED66F65
:103C4000FE0ED76F020ED86F030ED96F070EDA6F14
:103C5000000EDB6F000EDC6F000EDD6F000EDE6FFE
:103C6000010EDF6F8DECE6F0BAEF87F0F20EE96F30
:103C7000FD0EEA6F0A0EEB6FA5C0ECF0030E23EC0D
:103C8000F2F0690EC26FFC0EC36F5A0EC46F010EC4
:103C9000C56F000EC66F000EC76F020EC86F000E14
:103CA000C96F000ECA6F000ECB6F000ECC6F000EF6
:103CB000CD6FF6C0CEF0F8ECFEF0A90ED66FFD0E7B
:103CC000D76F0B0ED86F030ED96F020EDA6F000E8E
:103CD000DB6F000EDC6F000EDD6F000EDE6F010E7D
:103CE000DF6F8DECE6F0690EC26FFC0EC36F5A0EEB
:103CF000C46F010EC56F000EC66F000EC76F050EB4
:103D0000C86F000EC96F000ECA6F000ECB6F000E99
:103D1000CC6F000ECD6FF6C0CEF0F8ECFEF0400E8A
:103D2000D66FFE0ED76F020ED86F030ED96F050E39
:103D3000DA6F000EDB6F000EDC6F000EDD6F000E21
:103D4000DE6F010EDF6F8DECE6F02AD7400EE96FD3
:103D5000FE0EEA6F020EEB6FA5C0ECF0040E23EC32
:103D6000F2F0690EC26FFC0EC36F5A0EC46F010EE3
:103D7000C56F000EC66F000EC76F020EC86F000E33
:103D8000C96F000ECA6F000ECB6F000ECC6F000E15
:103D9000CD6FF6C0CEF0F8ECFEF0A90ED66FFD0E9A
:103DA000D76F0B0ED86F030ED96F020EDA6F000EAD
:103DB000DB6F000EDC6F000EDD6F000EDE6F010E9C
:103DC000DF6F8DECE6F0690EC26FFC0EC36F5A0E0A
:103DD000C46F010EC56F000EC66F000EC76F030ED5
:103DE000C86F000EC96F000ECA6F000ECB6F000EB9
:103DF000CC6F000ECD6FF6C0CEF0F8ECFEF0F20EF8
:103E0000D66FFD0ED76F0A0ED86F030ED96F030E53
:103E1000DA6F000EDB6F000EDC6F000EDD6F000E40
:103E2000DE6F010EDF6F8DECE6F0690EC26FFC0EE7
:103E3000C36F5A0EC46F010EC56F000EC66F000E21
:103E4000C76F060EC86F000EC96F000ECA6F000E56
:103E5000CB6F000ECC6F000ECD6FF6C0CEF0F8EC3D
:103E6000FEF0BAD63E0EE96FFE0EEA6F020EEB6F61
:103E7000A5C0ECF0050E23ECF2F0690EC26FFC0E4B
:103E8000C36F5A0EC46F010EC56F000EC66F000ED1
:103E9000C76F020EC86F000EC96F000ECA6F000E0A
:103EA000CB6F000ECC6F000ECD6FF6C0CEF0F8ECED
:103EB000FEF0A90ED66FFD0ED76F0B0ED86F030E56
:103EC000D96F020EDA6F000EDB6F000EDC6F000E92
:103ED000DD6F000EDE6F010EDF6F8DECE6F0690E18
:103EE000C26FFC0EC36F5A0EC46F010EC56F000E79
:103EF000C66F000EC76F030EC86F000EC96F000EAD
:103F0000CA6F000ECB6F000ECC6F000ECD6FF6C0E7
:103F1000CEF0F8ECFEF0F20ED66FFD0ED76F0A0E63
:103F2000D86F030ED96F030EDA6F000EDB6F000E31
:103F3000DC6F000EDD6F000EDE6F010EDF6F8DECAB
:103F4000E6F0690EC26FFC0EC36F5A0EC46F010E0D
:103F5000C56F000EC66F000EC76F040EC86F000E4F
:103F6000C96F000ECA6F000ECB6F000ECC6F000E33
:103F7000CD6FF6C0CEF0F8ECFEF0400ED66FFE0E20
:103F8000D76F020ED86F030ED96F040EDA6F000ED2
:103F9000DB6F000EDC6F000EDD6F000EDE6F010EBA
:103FA000DF6F8DECE6F0690EC26FFC0EC36F5A0E28
:103FB000C46F010EC56F000EC66F000EC76F070EEF
:103FC000C86F000EC96F000ECA6F000ECB6F000ED7
:103FD000CC6F000ECD6FF6C0CEF0F8ECFEF02ED612
:103FE0003C0EE96FFE0EEA6F020EEB6FA5C0ECF01F
:103FF000060E23ECF2F0690EC26FFC0EC36F5A0E70
:10400000C46F010EC56F000EC66F000EC76F020EA3
:10401000C86F000EC96F000ECA6F000ECB6F000E86
:10402000CC6F000ECD6FF6C0CEF0F8ECFEF0A90E0E
:10403000D66FFD0ED76F0B0ED86F030ED96F020E21
:10404000DA6F000EDB6F000EDC6F000EDD6F000E0E
:10405000DE6F010EDF6F8DECE6F0690EC26FFC0EB5
:10406000C36F5A0EC46F010EC56F000EC66F000EEF
:10407000C76F030EC86F000EC96F000ECA6F000E27
:10408000CB6F000ECC6F000ECD6FF6C0CEF0F8EC0B
:10409000FEF0F20ED66FFD0ED76F0A0ED86F030E2C
:1040A000D96F030EDA6F000EDB6F000EDC6F000EAF
:1040B000DD6F000EDE6F010EDF6F8DECE6F0690E36
:1040C000C26FFC0EC36F5A0EC46F010EC56F000E97
:1040D000C66F000EC76F040EC86F000EC96F000ECA
:1040E000CA6F000ECB6F000ECC6F000ECD6FF6C006
:1040F000CEF0F8ECFEF0400ED66FFE0ED76F020E3B
:10410000D86F030ED96F040EDA6F000EDB6F000E4E
:10411000DC6F000EDD6F000EDE6F010EDF6F8DECC9
:10412000E6F0690EC26FFC0EC36F5A0EC46F010E2B
:10413000C56F000EC66F000EC76F050EC86F000E6C
:10414000C96F000ECA6F000ECB6F000ECC6F000E51
:10415000CD6FF6C0CEF0F8ECFEF03E0ED66FFE0E40
:10416000D76F020ED86F030ED96F050EDA6F000EEF
:10417000DB6F000EDC6F000EDD6F000EDE6F010ED8
:10418000DF6F8DECE6F0BAEF87F09451010AD8B4F6
:1041900098D4030AD8B46AD5010AD8B4D7D5070A87
:1041A000D8B460D6010AD8B41BD7BAEF87F0830E13
:1041B0001119D8A4B1D300019F05D8A43CD0070E93
:1041C000D66FF6C0D7F0010EA7EC13F0330EEA6FEE
:1041D000FF0EEB6F0B0EEC6F2BEC0EF0F60ED66FA6
:1041E000FF0ED76F050ED86F000ED96F020EDA6F73
:1041F000000EDB6F000EDC6F000EDD6F000EDE6F59
:10420000000EDF6F1BEC05F09A05D8A404D0000E59
:10421000916F030E03D0010E916F010E946F000E8B
:104220009F6F35503610D8A404D0000E366E010EA4
:10423000356E010E966F9605D8B46AD27AD2600EAA
:10424000C26FE50EC36F070EC46F020EC56F000E7E
:10425000C66F450EC76F040EC86F000EC96F000E03
:10426000CA6F000ECB6F000ECC6F000ECD6FF6C084
:10427000CEF0F8ECFEF0600EC26FE50EC36F070ED5
:10428000C46F020EC56F6B0EC66F450EC76F020E70
:10429000C86F000EC96F000ECA6F000ECB6F000E04
:1042A000CC6F000ECD6FF6C0CEF0F8ECFEF072C011
:1042B000D6F073C0D7F01E0ED86F020ED96F000E65
:1042C000DA6F000EDB6F000EDC6F1EECCEF0B75124
:1042D000D8A41DD00A0EC26FC30EC36F440EC46FA4
:1042E000020EC56F0A0EC66F000EC76F040EC86FB0
:1042F000000EC96F000ECA6F000ECB6F000ECC6FA0
:10430000000ECD6FF6C0CEF0F8ECFEF01CD00A0E19
:10431000C26FC30EC36F440EC46F020EC56F0C0E86
:10432000C66F000EC76F040EC86F000EC96F000E77
:10433000CA6F000ECB6F000ECC6F000ECD6FF6C0B3
:10434000CEF0F8ECFEF09105D8A41DD00A0EC26F95
:10435000C30EC36F440EC46F020EC56F040EC66F4A
:10436000000EC76F060EC86F000EC96F000ECA6F31
:10437000000ECB6F000ECC6F000ECD6FF6C0CEF0EE
:10438000F8ECFEF01CD00A0EC26FC30EC36F440ED1
:10439000C46F020EC56F1A0EC66F000EC76F060EF1
:1043A000C86F000EC96F000ECA6F000ECB6F000EF3
:1043B000CC6F000ECD6FF6C0CEF0F8ECFEF0B1057C
:1043C000D8A406D05A0ED66F200E54ECFBF0AAD11A
:1043D000020EB119D8A406D05A0ED66F200E54EC96
:1043E000FBF0A0D1030EB119D8A49CD15A0ED66F00
:1043F000200E54ECFBF096D1600EC26FE50EC36F39
:10440000070EC46F020EC56F000EC66F450EC76F54
:10441000020EC86F000EC96F000ECA6F000ECB6F80
:10442000000ECC6F000ECD6FF6C0CEF0F8ECFEF0B3
:10443000600EC26FE50EC36F070EC46F020EC56F2C
:104440006B0EC66F450EC76F040EC86F000EC96FA6
:10445000000ECA6F000ECB6F000ECC6F000ECD6F3A
:10446000F6C0CEF0F8ECFEF072C0D6F073C0D7F014
:104470001E0ED86F020ED96F000EDA6F000EDB6FC2
:10448000000EDC6F1EECCEF0B751D8A41DD00A0E82
:10449000C26FC30EC36F440EC46F020EC56F0B0E06
:1044A000C66F000EC76F040EC86F000EC96F000EF6
:1044B000CA6F000ECB6F000ECC6F000ECD6FF6C032
:1044C000CEF0F8ECFEF01CD00A0EC26FC30EC36F24
:1044D000440EC46F020EC56F0D0EC66F000EC76F7F
:1044E000040EC86F000EC96F000ECA6F000ECB6FAE
:1044F000000ECC6F000ECD6FF6C0CEF0F8ECFEF0E3
:104500009105D8A41DD00A0EC26FC30EC36F440E0E
:10451000C46F020EC56F040EC66F000EC76F060E85
:10452000C86F000EC96F000ECA6F000ECB6F000E71
:10453000CC6F000ECD6FF6C0CEF0F8ECFEF01CD0C4
:104540000A0EC26FC30EC36F440EC46F020EC56F56
:104550001A0EC66F000EC76F060EC86F000EC96F29
:10456000000ECA6F000ECB6F000ECC6F000ECD6F29
:10457000F6C0CEF0F8ECFEF0780ED66F780E54EC64
:10458000FBF0D0D0600EC26FE50EC36F070EC46F94
:10459000020EC56F000EC66F450EC76F020EC86FC4
:1045A000000EC96F000ECA6F000ECB6F000ECC6FED
:1045B000000ECD6FF6C0CEF0F8ECFEF0600EC26FCC
:1045C000E50EC36F070EC46F020EC56F000EC66FF7
:1045D000450EC76F040EC86F000EC96F000ECA6F7C
:1045E000000ECB6F000ECC6F000ECD6FF6C0CEF07C
:1045F000F8ECFEF072C0D6F073C0D7F01E0ED86F84
:10460000020ED96F000EDA6F000EDB6F000EDC6F4A
:104610001EECCEF0B751D8A41DD00A0EC26FC30E47
:10462000C36F440EC46F020EC56F0A0EC66F000E34
:10463000C76F040EC86F000EC96F000ECA6F000E60
:10464000CB6F000ECC6F000ECD6FF6C0CEF0F8EC45
:10465000FEF01CD00A0EC26FC30EC36F440EC46FAF
:10466000020EC56F0C0EC66F000EC76F040EC86F2A
:10467000000EC96F000ECA6F000ECB6F000ECC6F1C
:10468000000ECD6FF6C0CEF0F8ECFEF09105D8A488
:104690001DD00A0EC26FC30EC36F440EC46F020E4C
:1046A000C56F050EC66F000EC76F060EC86F000EF1
:1046B000C96F000ECA6F000ECB6F000ECC6F000EDC
:1046C000CD6FF6C0CEF0F8ECFEF01CD00A0EC26F33
:1046D000C30EC36F440EC46F020EC56F1B0EC66FB0
:1046E000000EC76F060EC86F000EC96F000ECA6FAE
:1046F000000ECB6F000ECC6F000ECD6FF6C0CEF06B
:10470000F8ECFEF0780ED66F780E54ECFBF00AD081
:104710009451010AD8B493D5030AD8B46DD6010ACE
:10472000D8B430D794C095F0000E966F000E9E6FEF
:1047300020D001015305D8A41CD000017051711183
:10474000D8A404D0000E716F010E706F70C0D6F047
:1047500071C0D7F01E0ED86F020ED96F000EDA6F3F
:10476000000EDB6F000EDC6F1EECCEF0000E0101C0
:10477000536F00019E05D8A4C5D08C05D8A436D0AF
:1047800070C0D6F071C0D7F01E0ED86F020ED96F70
:10479000000EDA6F000EDB6F000EDC6F1EECCEF049
:1047A00070C072F071C073F09151D8A4A9D00A0EF4
:1047B000C26FC30EC36F440EC46F020EC56F040EEA
:1047C000C66F000EC76F060EC86F000EC96F000ED1
:1047D000CA6F000ECB6F000ECC6F000ECD6FF6C00F
:1047E000CEF0F8ECFEF0010E916F8AD0020E951912
:1047F000D8A446D001015205D8A41FD00A0E00014A
:10480000C26FC30EC36F440EC46F020EC56F0D0E90
:10481000C66F000EC76F040EC86F000EC96F000E82
:10482000CA6F000ECB6F000ECC6F000ECD6FF6C0BE
:10483000CEF0F8ECFEF0010E1ED00A0E0001C26FA1
:10484000C30EC36F440EC46F020EC56F0B0EC66F4E
:10485000000EC76F040EC86F000EC96F000ECA6F3E
:10486000000ECB6F000ECC6F000ECD6FF6C0CEF0F9
:10487000F8ECFEF0000EB76F9151D8B498D740D045
:10488000030E9519D8A43CD09105D8A41DD00A0ECA
:10489000C26FC30EC36F440EC46F020EC56F060E07
:1048A000C66F000EC76F060EC86F000EC96F000EF0
:1048B000CA6F000ECB6F000ECC6F000ECD6FF6C02E
:1048C000CEF0F8ECFEF01CD00A0EC26FC30EC36F20
:1048D000440EC46F020EC56F1C0EC66F000EC76F6C
:1048E000060EC86F000EC96F000ECA6F000ECB6FA8
:1048F000000ECC6F000ECD6FF6C0CEF0F8ECFEF0DF
:10490000000E9E6F410EBC6F140EBD6F9851A1EC4E
:104910000CF00101536F1200840E1119D8A458D263
:10492000360E0A6F1B0E0E6F5F0E0D6F00019F0596
:10493000D8A448D0070ED66FF6C0D7F0010EA7EC6A
:1049400013F0490EEA6FFF0EEB6F0B0EEC6F2BECC2
:104950000EF0A30ED66FFF0ED76F080ED86F000EA5
:10496000D96F020EDA6F000EDB6F000EDC6F000EE7
:10497000DD6F000EDE6F000EDF6F1BEC05F0CC0E5E
:10498000D66FFF0ED76F060ED86F000ED96F040ECC
:10499000DA6F000EDB6F000EDC6F000EDD6F000EB5
:1049A000DE6F000EDF6F1BEC05F0000E9F6F010E37
:1049B0009E6F010E946F010E966F010E0101406F04
:1049C000010E3F6F00019605D8B427D137D1600E94
:1049D000C26FE50EC36F070EC46F020EC56F000EE7
:1049E000C66F0DC4C7F0040EC86F000EC96F000E6D
:1049F000CA6F000ECB6F000ECC6F000ECD6FF6C0ED
:104A0000CEF0F8ECFEF0600EC26FE50EC36F070E3D
:104A1000C46F020EC56F6B0EC66F0DC4C7F0020ED9
:104A2000C86F000EC96F000ECA6F000ECB6F000E6C
:104A3000CC6F000ECD6FF6C0CEF0F8ECFEF08451D6
:104A4000D8A41DD0860EC26FEE0EC36F320EC46F97
:104A5000020EC56F010EC66F0EC4C7F0060EC86FFA
:104A6000000EC96F000ECA6F000ECB6F000ECC6F28
:104A7000000ECD6FF6C0CEF0F8ECFEF0D8D0860E6A
:104A8000C26FEE0EC36F320EC46F020EC56F040EFE
:104A9000C66F0EC4C7F0060EC86F000EC96F000EB9
:104AA000CA6F000ECB6F000ECC6F000ECD6FF6C03C
:104AB000CEF0F8ECFEF0BBD0600EC26FE50EC36F17
:104AC000070EC46F020EC56F000EC66F0DC4C7F08F
:104AD000020EC86F000EC96F000ECA6F000ECB6FBA
:104AE000000ECC6F000ECD6FF6C0CEF0F8ECFEF0ED
:104AF000600EC26FE50EC36F070EC46F020EC56F66
:104B00006B0EC66F0DC4C7F0040EC86F000EC96FE0
:104B1000000ECA6F000ECB6F000ECC6F000ECD6F73
:104B2000F6C0CEF0F8ECFEF08451D8B48BD7A7D7FE
:104B3000600EC26FE50EC36F070EC46F020EC56F25
:104B4000000EC66F0DC4C7F0020EC86F000EC96F0D
:104B5000000ECA6F000ECB6F000ECC6F000ECD6F33
:104B6000F6C0CEF0F8ECFEF0600EC26FE50EC36F3B
:104B7000070EC46F020EC56F000EC66F0DC4C7F0DE
:104B8000040EC86F000EC96F000ECA6F000ECB6F07
:104B9000000ECC6F000ECD6FF6C0CEF0F8ECFEF03C
:104BA0008451D8A41DD0860EC26FEE0EC36F320E94
:104BB000C46F020EC56F020EC66F0EC4C7F0060E9C
:104BC000C86F000EC96F000ECA6F000ECB6F000ECB
:104BD000CC6F000ECD6FF6C0CEF0F8ECFEF027D013
:104BE000860EC26FEE0EC36F320EC46F020EC56F1B
:104BF000050EC66F0EC4C7F0060EC86F000EC96F53
:104C0000000ECA6F000ECB6F000ECC6F000ECD6F82
:104C1000F6C0CEF0F8ECFEF00AD09451010AD8B4F8
:104C2000D6D6030AD8B448D7010AD8B481D794C0DD
:104C300095F0000E966F000E9E6F40D0010140056A
:104C4000D8A41DD031503210D8A404D0000E326E3A
:104C5000010E316E31C0D6F032C0D7F00AC4D8F0A0
:104C6000020E0001D96F000EDA6F000EDB6F000E2E
:104C7000DC6F1EECCEF0000E0101406F1FD03F052F
:104C8000D8A41CD02F503010D8A404D0000E306E01
:104C9000010E2F6E2FC0D6F030C0D7F00AC4D8F066
:104CA000040E0001D96F000EDA6F000EDB6F000EEC
:104CB000DC6F1EECCEF0000E01013F6F00019E057F
:104CC000D8A46CD08305D8A413D031C0D6F032C09C
:104CD000D7F00AC4D8F0020ED96F000EDA6F000EBA
:104CE000DB6F000EDC6F1EECCEF0000E986F54D020
:104CF0008205D8A411D02FC0D6F030C0D7F00AC496
:104D0000D8F0040ED96F000EDA6F000EDB6F000EC4
:104D1000DC6F1EECCEF0E9D7030E9519D8A43CD079
:104D20008451D8A41DD0860EC26FEE0EC36F320E12
:104D3000C46F020EC56F030EC66F0EC4C7F0060E19
:104D4000C86F000EC96F000ECA6F000ECB6F000E49
:104D5000CC6F000ECD6FF6C0CEF0F8ECFEF01CD09C
:104D6000860EC26FEE0EC36F320EC46F020EC56F99
:104D7000060EC66F0EC4C7F0060EC86F000EC96FD0
:104D8000000ECA6F000ECB6F000ECC6F000ECD6F01
:104D9000F6C0CEF0F8ECFEF0000E9E6F8305D8A4AE
:104DA0000AD0410EBC6F140EBD6F9851A1EC0CF0EF
:104DB0000101406F12008205D8A41200410EBC6FA1
:104DC000140EBD6F9851A1EC0CF001013F6F120061
:104DD0001105D8A4F3D000019F05D8A427D0000E58
:104DE000C26FDF0EC36F660EC46F040EC56F010E77
:104DF000C66F650EC76F000EC86F000EC96F000E3C
:104E0000CA6F000ECB6F000ECC6F000ECD6FF6C0D8
:104E1000CEF0F8ECFEF0010E436E000E0201A36F1F
:104E2000010E0101C16F000E00019F6F060E01010E
:104E3000C0651200650E436002D0432A3ED0000ECA
:104E40000001C26FDF0EC36F660EC46F040EC56F24
:104E5000020EC66F160EC76F040EC86F000EC96F24
:104E6000000ECA6F000ECB6F000ECC6F000ECD6F20
:104E7000F6C0CEF0F8ECFEF0890EC26FF70EC36FED
:104E80000F0EC46F020EC56F0A0EC66F590EC76FA4
:104E9000060EC86F000EC96F000ECA6F000ECB6FF2
:104EA000000ECC6F000ECD6FF6C0CEF0F8ECFEF029
:104EB000000E0101C16F010EBF6F3A0E436430D086
:104EC000F20E0001D66F020ED76F050ED86F435059
:104ED0006508D96F040EDA6F000EDB6F000EDC6F11
:104EE000000EDD6F000EDE6F010EDF6F8DECE6F061
:104EF000000ED66FFF0ED76F020ED86F43507B089F
:104F0000D96F040EDA6F000EDB6F000EDC6F000E3F
:104F1000DD6F000EDE6F010EDF6F8DECE6F02DD041
:104F20000E0E0001D66FFE0ED76F080ED86F000E62
:104F3000D96F040EDA6F000EDB6F000EDC6F000E0F
:104F4000DD6F000EDE6F010EDF6F8DECE6F0F20E0E
:104F5000D66F020ED76F050ED86F2A0ED96F040ECA
:104F6000DA6F000EDB6F000EDC6F000EDD6F000EDF
:104F7000DE6F010EDF6F8DECE6F0000EC26FDF0E0C
:104F8000C36F660EC46F040EC56F010EC66F43502B
:104F90006508C76F000EC86F000EC96F000ECA6F9C
:104FA000000ECB6F000ECC6F000ECD6FF6C0CEF0B2
:104FB000F8ECFEF0000E0101C06F1200030E111993
:104FC000D8A44AD000019F05D8A41BD08105D8A43D
:104FD0000BD044C0D6F0D76B100ED86F020ED96F2D
:104FE000020EFEECD0F00BD0000ED76F000ED66F85
:104FF000100ED86F020ED96F050EFEECD0F0000E29
:105000009F6F01017105D8A4120000018105D8A489
:105010001200600EC26FE50EC36F070EC46F020E62
:10502000C56F4450600FC66F290EC76F050EC86F5D
:10503000000EC96F000ECA6F010ECB6F000ECC6F51
:10504000000ECD6FF6C0CEF0F8ECFEF044C072F169
:10505000000E0101716F1200040E1119D8A442D084
:10506000100E056F020E066F00019F05D8A40CD02C
:1050700093C0D6F0D76B05C4D8F006C4D9F0040E9F
:10508000FEECD0F0000E9F6F01016F05D8A4120056
:10509000600E0001C26FE50EC36F070EC46F020EF3
:1050A000C56F9351600FC66F04010551190F0001C0
:1050B000C76F04010651030F0001C86F000EC96FCE
:1050C000000ECA6F010ECB6F000ECC6F000ECD6FBD
:1050D000F6C0CEF0F8ECFEF093C070F1000E0101C6
:1050E0006F6F1200050E1119D8A49DD0100E0B6F12
:1050F000020E0C6F020E096F090E046F00019F056E
:10510000D8A40DD0000ED76F1E0ED66F0BC4D8F0EA
:105110000CC4D9F0030EFEECD0F0000E9F6F01011D
:105120006F05D8A412000A0E0001C06F935138EC2D
:1051300015F0600F0401096F0A0E0001BC6F935156
:10514000A9EC16F0600F0401046F600E0919D8B4C1
:1051500024D0600E0001C26FE50EC36F070EC46F4E
:10516000020EC56F09C4C6F004010B51150F0001F2
:10517000C76F04010C51030F0001C86F000EC96F07
:10518000000ECA6F010ECB6F000ECC6F000ECD6FFC
:10519000F6C0CEF0F8ECFEF023D0600E0001C26F36
:1051A000E50EC36F070EC46F020EC56F6C0EC66F9F
:1051B00004010B51150F0001C76F04010C51030FBF
:1051C0000001C86F000EC96F000ECA6F010ECB6FD1
:1051D000000ECC6F000ECD6FF6C0CEF0F8ECFEF0F6
:1051E000600EC26FE50EC36F070EC46F020EC56F6F
:1051F00004C4C6F004010B511E0F0001C76F040167
:105200000C51030F0001C86F000EC96F000ECA6F6A
:10521000010ECB6F000ECC6F000ECD6FF6C0CEF03E
:10522000F8ECFEF059D7060E1119D8A41200100E92
:10523000076F020E086F00019F05D8A40CD042C072
:10524000D6F0D76B07C4D8F008C4D9F00D0EFEEC29
:10525000D0F0000E9F6F01016805D8A41200600E07
:105260000001C26FE50EC36F070EC46F020EC56F5B
:105270004250600FC66F04010751190F0001C76F3C
:1052800004010851030F0001C86F000EC96F000E22
:10529000CA6F010ECB6F000ECC6F000ECD6FF6C043
:1052A000CEF0F8ECFEF042C069F1000E0101686F2B
:1052B000120069EC0DF0BCECEFF0000E0001BD6FC8
:1052C000000EBC6F27EC18F0A00AD8B409D0000E6D
:1052D0000001BD6F000EBC6FA00EBE6F5BEC14F042
:1052E000A00EB0EC12F0C6EC18F0210E3A01136FCC
:1052F0003D017399D28ED28C010E7FEC13F0F66FC4
:10530000F651BDEC09F0010E0001A26F010E506EC6
:10531000C682200EC1EC17F00101E46FC4EC18F056
:1053200069ECDEF0CBEC15F0000E0001CC6F39C05B
:10533000CDF03AC0CEF0020ED06F020ECF6F040E49
:10534000D26F040ED16F090E09ECDCF0CCC039F03D
:10535000CDC03AF0010E0101B96F0101AE05D8A42C
:1053600003D00201614B622B00019051D8A41DECC7
:1053700011F000019051D8A420EC0FF027EC17F0A9
:1053800084EC18F089ECFAF000019051D8A41EECDE
:1053900004F004EC13F0D1EC0BF09DEC04F034ECD1
:1053A000F6F01AEC15F001015C05D8A422D0040E29
:1053B0000001A219D8B41DD0030EA219D8B419D077
:1053C000A205D8B416D0050EA219D8B412D09051A7
:1053D000D8B40FD0B451D8A40CD0AD51D8A409D0B2
:1053E000A2C0A1F0050EA26F010E9F6F010E010178
:1053F000C66F5050D8B4E9EC10F00101AC51D8B4EC
:105400000FD000019051D8A40BD0010E0101776F8D
:105410006D0E0001A219D8B403D0000E0101AC6FCB
:10542000020149514A11D8B403D04907D8A04A070C
:1054300001017705D8A423D00001A205D8B41FD05C
:10544000020149514A11D8A41AD0000E4A6F400EE9
:10545000496FADC0EAF0B4C0EBF0AEC0ECF062C191
:10546000EDF099C0EEF043C2EFF044C2F0F081C11C
:10547000F1F00101605137ECF5F00101776F0A0E90
:105480000001A219D8A478D39905D8A40BD0000E96
:10549000996F7AC043F27BC044F2010E0101776F2D
:1054A000000E476F0001AE05D8B403D0AF05D8A4F5
:1054B000DCD001015051D8A46DD0000178517A1987
:1054C00004E179517B19D8B458D0000E0101236F43
:1054D000000E226F010E0001B36F4AD084EC18F069
:1054E000000178517A1910E179517B19D8A40CD0B8
:1054F000000E0101A96F000E236F000E226F000E37
:105500000001B36F010E9F6F0101235104E1C80E2A
:10551000225DD8A02DD0000E0001D76F000ED66FEF
:10552000100ED86F020ED96F060EFEECD0F07A5135
:10553000351806E17B513618D8A402D0000E9A6FB8
:10554000010E0101A96F000E236F000E226F000EE5
:105550000001B36F010E9F6F410E0001F46FF00E5A
:10556000F36F330EE82EFED7F32FFCD7F42FFAD7C4
:105570000001B305D8A406D0B1D7000E0101A96F70
:10558000000E516F00017A517B11D8A403D0010E97
:105590000101506F01014F51D8A467D0355036102A
:1055A000D8A402D0010E4F6F00017251351804E1EA
:1055B00073513618D8B459D0000E0101236F000E74
:1055C000226F010E0001B36F4CD084EC18F0000183
:1055D0007251351817E173513618D8A413D0785189
:1055E0007A1910E179517B19D8A40CD0000E010171
:1055F000A96F000E236F000E226F000E0001B36F23
:10560000010E9F6F0101235104E1640E225DD8A0B9
:1056100028D0000E0001D76F000ED66F100ED86F85
:10562000020ED96F060EFEECD0F0000E9A6F72C01B
:1056300035F073C036F0000E0101236F000E226FAB
:10564000000E0001B36F010E9F6F410E0001F46F59
:10565000F00EF36F330EE82EFED7F32FFCD7F42FA6
:10566000FAD70001B305D8B4B0D70101A905D8B461
:1056700004D000018605D8A402D0010E09D0010192
:10568000A951D8A407D000018651D8A403D0000E98
:105690000101756F5A0E0001A619D8B404D05A0E34
:1056A00069EC0EF0A66FB051B119D8B404D0B05166
:1056B00014ECF8F0B16F4850D8B435D0A551D8A447
:1056C00030D0000ECA6F100EC96F3BEC17F0000906
:1056D000D8A427D0B8C0BCF03F50B3EC0AF08F6F0D
:1056E0008505D8A41AD0120E8F6502D0120E07D0ED
:1056F000030E8F6105D0010E3F6402D0020E8F6F42
:10570000050E8F610AD0020E8E6107D0020E8D6FDA
:105710008DC08EF0010E0101576F010E01015B6F0C
:1057200002D0000E486E010159510001B819D8B4D9
:1057300011D001015951B4EC18F0B86F010E0101FC
:10574000586F0001B851B71901015A6F000E4A6F26
:10575000010E496F0001A505D8A416D0010E010164
:10576000CD6F2F5104E13D0E2E5DD8A00DD00B0E54
:105770000001A26F000E0101CD6F000E2F6F000E11
:105780002E6F010E00019F6F0001A405D8A423D045
:1057900001012F5120E13D0E2E5DD8B01CD0000E2E
:1057A000CD6F000E2F6F000E2E6F47A006D0000E9B
:1057B00000018F6F010E01015B6F47A20CD03F50BB
:1057C000D8A409D00001B851010A0101596F000E97
:1057D0004A6F010E496F000E0001CA6F100EC96FAB
:1057E000DCEC14F00009D8B406D0AA51D8A403D038
:1057F000010E0101C86F000E0001CA6F100EC96FC3
:10580000FBEC14F00009D8B408D0000E0101C86FF9
:10581000000E02016E6F000E6D6F0001A905D8A485
:1058200015D002016E5104E1330E6D5DD8A00ED08B
:105830000C0E0001A26F000E0101C86F000E0201E4
:105840006E6F000E6D6F010E00019F6F02016A51B5
:1058500004E1960E695DD8A020D0010E00019F6F73
:10586000000E0101C56F000E02016A6F000E696F24
:1058700000018705D8A403D0010E0101486F000183
:105880008505D8A403D0010E0101416F00018605F2
:10589000D8A403D0010E0101436F70ECEBF00101BD
:1058A0007F51D8B402D0000E7F6F000E0001CA6F86
:1058B000100EC96FDCEC14F0E806D8B409D0000E65
:1058C000CA6F100EC96FFBEC14F0E806D8A41CD008
:1058D000AA51D8A40DD0A9C0CCF092C1CDF085C1F9
:1058E000CEF0000ECF6F0A0E9AECE4F0A96F0CD048
:1058F0004BC0CCF090C1CDF083C1CEF0000ECF6F85
:105900000C0E9AECE4F04B6E000ECA6F200EC96FBD
:10591000DCEC14F0E806D8B409D0000ECA6F200EF3
:10592000C96FFBEC14F0E806D8A41CD0AA51D8A487
:105930000DD0A8C0CCF091C1CDF084C1CEF0000E46
:10594000CF6F0B0E9AECE4F0A86F0CD0A7C0CCF090
:105950008FC1CDF082C1CEF0000ECF6F0D0E9AEC4C
:10596000E4F0A76FA705D8A40BD04EECFEF005D04D
:1059700084EC18F01BECFCF04F6E4F50D8B4F8D705
:105980000001B005D8A404D0A751BFEC16F007D091
:10599000020EB019D8A405D0A851BFEC16F03D6E88
:1059A00018D0030EB019D8A414D08851BFEC16F04B
:1059B0003D6E8905D8A402D0010E01D0000E010170
:1059C000456F0001865101014519D8B402D0010E7E
:1059D000446F000185513D18D8B411D03D04D8A4BE
:1059E00005D08EC056F1010E8D6F02D056C18DF0DC
:1059F0008DC08EF0010E0101576F010E426F000E37
:105A00000101806F0001A005D8A412D0A0C0CCF085
:105A1000000ECD6F000ECE6F000ECF6F140E9AECFD
:105A2000E4F0A06FA051D8A41AD0A1C0A2F00BD06E
:105A3000000ECA6F800EC96FFBEC14F0E806D8A404
:105A400006D0640EA26F010E9F6F010E06D0000EED
:105A5000CA6F800EC96F3BEC17F00101806F020E18
:105A60000001CA6F000EC96FFBEC14F0E806D8B451
:105A700009D0020ECA6F000EC96FDCEC14F0E80604
:105A8000D8A414D0AAC0CCF0010ECD6F010ECE6FF9
:105A9000000ECF6F0E0E9AECE4F0AA6F030EB11950
:105AA000D8A4AAC081F1010E0101776F0101325122
:105AB000D8A41BECFCF0000E0001CA6F400EC96FA9
:105AC000DCEC14F0E806D8A40BD0010E0101CC6F79
:105AD000000E00017F6F000E7E6F010E0101476F07
:105AE000000E0001CA6F400EC96F3BEC17F0E806CC
:105AF000D8A416D07F5104E1320E7E5DD8A010D01C
:105B0000000E0101476F00019051D8B409D04EEC4E
:105B1000FEF0A2C0A1F0040E0001A26F010E9F6F63
:105B2000000ECA6F400EC96FFBEC14F0E806D8A453
:105B300016D07F5114E1320E7E5DD8B010D0000E29
:105B40000101CC6F000E00017F6F000E7E6F01011E
:105B50004705D8A404D0010E4A1B010E496F87C027
:105B600074F100018005D8A47FEFC3F0A2C0A1F0BA
:105B7000030EA26F55EFC2F00B0EA219D8A434D0B9
:105B80009951D8A409D0010E996F7AC043F27BC015
:105B900044F2010E0101776F1E0E0001A619D8B460
:105BA00004D01E0E69EC0EF0A66F4850D8B407D092
:105BB0008E51F3EC13F08D6F010E0101576F000150
:105BC000A405D8A40CD00A0EA26F000E0101CD6F5F
:105BD000000E2F6F000E2E6F010E00019F6F8005CB
:105BE000D8B4C4D77FEFC3F00C0EA219D8A415D136
:105BF0009951D8A417D0010E996F7AC043F27BC097
:105C000044F2010E0101776F000E0001CA6F100E01
:105C1000C96F3BEC17F00009D8A404D00A0EA26F9C
:105C2000010E9F6FDC0EA619D8B404D0DC0E69EC0F
:105C30000EF0A66F4850D8B40DD076C0BCF077C037
:105C4000BDF05DEC0CF0BCC076F0BDC077F0010E8D
:105C50000101556F00017651335C77513458D8B04B
:105C600007D033C076F034C077F0010E0101556FD4
:105C7000000176517711D8A407D0000E776F010E7E
:105C8000766F010E0101556F000E0001CC6F000E02
:105C9000CD6F000ECE6F000ECF6F120E9AECE4F0B7
:105CA000E806D8A407D074C076F075C077F0010E6E
:105CB0000101556F000E0001CC6F000ECD6F000E7C
:105CC000CE6F000ECF6F130E9AECE4F0E806D8A466
:105CD00007D037C076F038C077F0010E0101556F5C
:105CE000000E0001CA6F100EC96FFBEC14F0000922
:105CF000D8B455D0000EA96F000E986F76517A195E
:105D000004E177517B19D8B432D074C037F075C034
:105D100038F07AC074F07BC075F0000E8B6F000E07
:105D20008A6F000E896F000E886F000E01014E6FA2
:105D3000000E4D6F000E4C6F000E4B6F000187057B
:105D4000D8A405D0000E01014A6F010E496F000E64
:105D500000018F6F010E01015B6F010E00018D6F5D
:105D6000010E0101576F000E516F000E506F78C089
:105D700043F279C044F2355000017A1906E13650F9
:105D80007B19D8A402D0000E9A6F0A0EA26F010EE2
:105D90009F6F9051D8A403D0050E37ECF3F0000E9E
:105DA0000001CA6F100EC96FDCEC14F0E806D8B41D
:105DB00009D0000ECA6F100EC96FFBEC14F0E80694
:105DC000D8A40CD0A9C0CCF092C1CDF085C1CEF042
:105DD000000ECF6F0A0E9AECE4F0A96F000ECA6FA6
:105DE000200EC96FDCEC14F0E806D8B409D0000E20
:105DF000CA6F200EC96FFBEC14F0E806D8A4EFD6EA
:105E0000A8C0CCF091C1CDF084C1CEF0000ECF6F10
:105E10000B0E9AECE4F0A86FE2D6640EA219D8A497
:105E200088D09951D8A409D0010E996F7AC043F255
:105E30007BC044F2010E0101776F1E0E0001A6190E
:105E4000D8B404D01E0E69EC0EF0A66F4850D8B43A
:105E500008D0A2C0BCF09551FDEC0AF0946F010E81
:105E6000966FA305D8A402D0010E9E6FA405D8B4E6
:105E70000ED020D0650E09D06E0E07D0820E05D050
:105E8000780E03D06D0E01D0640EA26F11D0955123
:105E9000010AD8B4EFD7030AD8B4EED7010AD8B4B0
:105EA000EDD7070AD8B4ECD7010AD8B4EBD7ECD7B2
:105EB000010E9F6F000ECA6F400EC96FDCEC14F02C
:105EC000E806D8A408D0010E0101CC6F000E000135
:105ED0007F6F000E7E6F000ECA6F400EC96F3BECE5
:105EE00017F0E806D8A412D07F5104E1510E7E5D70
:105EF000D8A00CD00A0EA26F010E9F6F000E0101F8
:105F0000CC6F000E00017F6F000E7E6F000ECA6F17
:105F1000400EC96FFBEC14F0E806D8A460D67F51A0
:105F200007E1510E7E5DD8B05AD60A0E8EEFC1F051
:105F300056D6650EA219D8A4DBD19951D8A409D0A0
:105F4000010E996F7AC043F27BC044F2010E010149
:105F5000776FDC0E0001A619D8B404D0DC0E69EC12
:105F60000EF0A66F4850D8B40DD076C0BCF077C004
:105F7000BDF05DEC0CF0BCC076F0BDC077F0010E5A
:105F80000101556F0001A305D8A404D0010E9E6F36
:105F9000000E986FA405D8A451D076517A1904E167
:105FA00077517B19D8B432D074C037F075C038F04F
:105FB0007AC074F07BC075F0000E8B6F000E8A6F94
:105FC000000E896F000E886F000E01014E6F000EEB
:105FD0004D6F000E4C6F000E4B6F00018705D8A46B
:105FE00005D0000E01014A6F010E496F000E00013D
:105FF0008F6F010E01015B6F010E00018D6F010EAD
:106000000101576F000E516F000E506F78C043F2C0
:1060100079C044F2355000017A1906E136507B19F7
:10602000D8A402D0000E9A6F0A0EA26F010E9F6FC5
:106030009051D8A403D0050E37ECF3F0000E000108
:10604000CC6F000ECD6F000ECE6F000ECF6F120E14
:106050009AECE4F0E806D8A407D074C076F075C0D6
:1060600077F0010E0101556F000E0001CC6F000E9C
:10607000CD6F000ECE6F000ECF6F130E9AECE4F0D2
:10608000E806D8A407D037C076F038C077F0010E04
:106090000101556F000E0001CC6F000ECD6F000E98
:1060A000CE6F000ECF6F0F0E9AECE4F0E806D8A486
:1060B0007BD0030EB119D8A441D0390EF66EFE0E76
:1060C000F76E000EF86E0800F550420AD8A413D0FF
:1060D00076C0C9F077C0CAF05A0ECB6F8CEC02F0D4
:1060E000F36F090EF36105D00A0E7627000E7723B1
:1060F00021D05A0E55D076C0C9F077C0CAF05A0EDA
:10610000CB6F8CEC02F0F36F060EF36105D00A0E34
:106110007627000E772304D03C0E765F000E775B67
:10612000775104E13E0E765DD8A004D0000E776F63
:106130003D0E766F010E0101556F36D0020EB1197A
:10614000D8A409D076C0C9F077C0CAF05A0ECB6F78
:106150008CEC02F0C5D7B105D8A426D076C0C9F022
:1061600077C0CAF0540ECB6F8CEC02F00009D8A4B3
:1061700009D076C0C9F077C0CAF05A0ECB6F8CEC4C
:1061800002F0AED776C0C9F077C0CAF05A0ECB6F16
:106190008CEC02F0F36F020EF36101D0A5D7140E60
:1061A000765F000E775BC6D7000E0001CC6F000E45
:1061B000CD6F000ECE6F000ECF6F100E9AECE4F094
:1061C000E806D8A42CD0020EB119D8B428D0B10555
:1061D000D8A425D076C0C9F077C0CAF0540ECB6FD2
:1061E0008CEC02F00009D8A413D076C0C9F077C0B7
:1061F000CAF0480ECB6F8CEC02F0F36F090EF3611E
:1062000005D0640E7627000E772306D0840E01D0C9
:10621000E80E765F030E775B010E0101556F0001FA
:106220007651335C77513458D8B007D033C076F00C
:1062300034C077F0010E0101556F000176517711DE
:10624000D8A407D0000E776F010E766F010E010102
:10625000556F000E0001CA6F400EC96FDCEC14F0E0
:10626000E806D8A40ED0000E986F010E0101CC6F85
:10627000000E00017F6F000E7E6F7AC076F07BC04B
:1062800077F0000ECA6F400EC96F3BEC17F0E806BE
:10629000D8A412D07F5104E1510E7E5DD8A00CD05D
:1062A0000A0EA26F010E9F6F000E0101CC6F000E4F
:1062B00000017F6F000E7E6F000ECA6F400EC96F27
:1062C000FBEC14F0E806D8A48AD47F5110E1510EFB
:1062D0007E5DD8B084D4640EA26F000E0101CC6F35
:1062E000000E00017F6F000E7E6F010E77D477D411
:1062F0006E0EA219D8A488D09951D8A409D0010E45
:10630000996F7AC043F27BC044F2010E0101776FAE
:106310001E0E0001A619D8B404D01E0E69EC0EF0B2
:10632000A66F4850D8B408D0A2C0BCF09551FDEC7F
:106330000AF0946F010E966FA305D8A402D0010E47
:106340009E6FA405D8B412D023D06F0EA26F030E97
:10635000B9EC18F01AD06F0EA26F010EB9EC18F05C
:1063600014D0700E01D0640EA26F0FD09551010AA7
:10637000D8B4EBD7030AD8B4EED7010AD8B4F1D712
:10638000070AD8B4F0D7010AEED7010E00019F6FBB
:10639000000ECA6F400EC96FDCEC14F0E806D8A4FA
:1063A00008D0010E0101CC6F000E00017F6F000EBE
:1063B0007E6F000ECA6F400EC96F3BEC17F0E80607
:1063C000D8A412D07F5104E1510E7E5DD8A00CD02C
:1063D0000A0EA26F010E9F6F000E0101CC6F000E1E
:1063E00000017F6F000E7E6F000ECA6F400EC96FF6
:1063F000FBEC14F0E806D8A4EFEFADF07F5102E11A
:1064000088EFC1F0EFEFADF06F0EA219D8A413D34F
:106410009951D8A409D0010E996F7AC043F27BC07C
:1064200044F2010E0101776F080E3F6405D0080E9B
:1064300000018F6F080E3F6E010E00018D6F010E7F
:106440008E6F9C51D8A40BD09B51D8A408D01E0E9F
:10645000A619D8B404D01E0E69EC0EF015D09C0518
:10646000D8A408D0A00EA619D8B404D0A00E69EC08
:106470000EF00AD09B05D8A408D0DC0EA619D8B41B
:1064800004D0DC0E69EC0EF0A66F4850D8B435D0BD
:106490009C51D8A414D09B51D8A411D0A2C0BCF058
:1064A0009551FDEC0AF0946F9D05D8A405D0020E1D
:1064B000946502D0020E946F010E966F1ED09C055B
:1064C000D8A40BD06C51CEEC13F0F36FF3516C6F7A
:1064D0006D6B010E01013E6F10D09B05D8A40DD04D
:1064E00068C0BCF069C0BDF05CEC0FF0BCC068F0E7
:1064F000BDC069F0010E01013D6F0001A305D8A4E4
:1065000004D0000E986F010E9E6FA405D8A46ED023
:106510009C51D8A461D09B51D8B43DD05DD0010E20
:106520009C6F000E466E000E9B6F0BD09D05D8B47D
:106530000BD0010E9B6F000E0101766F000E000163
:106540009C6F010E986F52D04604D8A44FD0010E14
:1065500001019C6F000E000114D04604D8A446D05F
:1065600001017605D8A442D000019D05D8B40AD017
:106570006E51E4EC0EF001019C6F00016E516BEC6A
:1065800007F0AC6F000E0101A86F6F0E0001A26F43
:10659000010E9F6F2BD09551010AD8B4C0D7030AC2
:1065A000D8B4C4D7010AD8B4D8D720D0000E9C6F75
:1065B000010E466E6CC06EF06DC06FF014D09D057C
:1065C000D8B411D0000E9B6F010E0101766F68C028
:1065D0006AF069C06BF007D09551010AD8B4E6D7CC
:1065E000030AD8B4ECD7010E0001966F01019C0597
:1065F000D8B404D00001AC05D8A407D00101A8513B
:10660000D8A403D0010E0001B36F0001B305D8B4C4
:1066100056D059D084EC18F000016E5102013B199C
:106620001DE100016F5102013C19D8A417D00001EF
:106630006A510201391912E100016B5102013A1944
:10664000D8A40CD0000E0101A86F000E236F000E1D
:10665000226F000E0001B36F010E9F6F01012351E5
:1066600004E1C80E225DD8A02AD0000E0001D76F29
:10667000000ED66F100ED86F020ED96F0B0EFEEC07
:10668000D0F0010E0101A86F000E9C6F000E0001FA
:10669000AC6F000E0101236F000E226F000E00018F
:1066A000B36F010E9F6F410E0001F46FF00EF36F98
:1066B000330EE82EFED7F32FFCD7F42FFAD70001C4
:1066C000B305D8B4A7D7A0C0CCF0000ECD6F000E94
:1066D000CE6F000ECF6F140E9AECE4F0A06FA00501
:1066E000D8A406D0A2C0A1F00A0EA26F010E9F6F1F
:1066F000000ECC6F000ECD6F000ECE6F000ECF6F70
:106700000F0E9AECE4F0E806D8A4DFD0B105D8A4C7
:106710006ED09B05D8A434D068C0C9F069C0CAF057
:10672000480ECB6F8CEC02F0F36F020EF36113D0C6
:1067300068C0C9F069C0CAF05A0ECB6F8CEC02F089
:10674000F36F090EF36105D00A0E6827000E692366
:1067500013D05A0E0ED068C0C9F069C0CAF05A0EE4
:10676000CB6F8CEC02F0F36F050EF36101D0ECD728
:10677000320E685F000E695B010E01013D6FA5D00E
:106780009C51D8B4A2D06CC0C9F06DC0CAF0480EFC
:10679000CB6F8CEC02F0F36F020EF36113D06CC080
:1067A000C9F06DC0CAF05A0ECB6F8CEC02F0F36FDB
:1067B000090EF36105D00A0E6C27000E6D2313D06D
:1067C0005A0E0ED06CC0C9F06DC0CAF05A0ECB6F15
:1067D0008CEC02F0F36F050EF36101D0ECD7320EB2
:1067E0006C5F000E6D5B010E01013E6F6ED0020EFC
:1067F000B119D8A433D09B05D8A424D068C0C9F05F
:1068000069C0CAF0480ECB6F8CEC02F0F36F020E39
:10681000F36109D068C0C9F069C0CAF05A0ECB6FE5
:106820008CEC02F08DD768C0C9F069C0CAF05A0E6E
:10683000CB6F8CEC02F0F36F030EF36101D084D7C1
:106840001E0E97D79C51D8B440D06CC0C9F06DC013
:10685000CAF05A0ECB6F8CEC02F0A9D7030EB11917
:10686000D8A433D09B05D8A41ED068C0C9F069C095
:10687000CAF0480ECB6F8CEC02F0F36F020EF3619E
:1068800009D068C0C9F069C0CAF05A0ECB6F8CEC51
:1068900002F056D768C0C9F069C0CAF05A0ECB6F73
:1068A0008CEC02F0C8D79C51D8B40FD06CC0C9F0A2
:1068B0006DC0CAF05A0ECB6F8CEC02F0F36F070E6E
:1068C000F36101D078D7460E8BD7000E0001CC6F54
:1068D000000ECD6F000ECE6F000ECF6F100E9AEC33
:1068E000E4F0E806D8A44BD0B105D8A438D09B0575
:1068F000D8A419D068C0C9F069C0CAF0480ECB6FDF
:106900008CEC02F0F36F020EF36105D0640E682781
:10691000000E692304D0C80E685F000E695B010E8B
:1069200001013D6F2CD09C51D8B429D06CC0C9F066
:106930006DC0CAF0480ECB6F8CEC02F0F36F020E04
:10694000F36105D0640E6C27000E6D2304D0C80ED1
:106950006C5F000E6D5B010E01013E6F10D0020EE8
:10696000B119D8A40CD09B05D8A409D068C0C9F02F
:1069700069C0CAF0480ECB6F8CEC02F0C3D73E5012
:106980000001F36FF46B6C51F35D6D51F459D8B0A5
:1069900003D03EC06CF06D6B68510101085D0001D1
:1069A000695101010959D8B004D008C168F009C182
:1069B00069F0000E0001CA6F400EC96FDCEC14F0E4
:1069C000E806D8A40ED0000E986F010E0101CC6F1E
:1069D000000E00017F6F000E7E6F000E9B6F000E99
:1069E0009C6F000ECA6F400EC96F3BEC17F0E806B3
:1069F000D8A412D07F5104E1510E7E5DD8A00CD0F6
:106A00000A0EA26F010E9F6F000E0101CC6F000EE7
:106A100000017F6F000E7E6F000ECA6F400EC96FBF
:106A2000FBEC14F0E806D8A4EFEFADF07F5101E1E4
:106A30001BD2EFEFADF0700EA219D8A41FD299515E
:106A4000D8A409D0010E996F7AC043F27BC044F2FA
:106A5000010E0101776F000E00018F6F000E3F6E77
:106A6000DC0EA619D8B404D0DC0E69EC0EF0A66FCB
:106A70004850D8B40DD066C0BCF067C0BDF05DEC26
:106A80000CF0BCC066F0BDC067F0010E01013C6FA8
:106A90000001A305D8A404D0000E986F010E9E6FCC
:106AA000A405D8A432D066517A1904E167517B1944
:106AB000D8B428D0000E8B6F000E8A6F000E896F3D
:106AC000000E886F000E01014E6F000E4D6F000E1C
:106AD0004C6F000E4B6F00018705D8A405D0000E47
:106AE00001014A6F010E496F010E00018D6F010E09
:106AF0008E6F66C000F167C001F1010E01019D6F4C
:106B0000000EA86F000E00019A6F01019D05D8A428
:106B100006D0A851D8A403D0010E0001B36F000124
:106B2000B305D8B458D05BD084EC18F00101005103
:106B3000021922E101510319D8A41ED0000EA86F3A
:106B400002C176F003C177F002C178F003C179F099
:106B500078C0BCF079C0BDF086EC06F0000E0101F3
:106B60009D6F000E236F000E226F000E0001B36FA9
:106B70000A0EA26F010E9F6F0101235104E1C80E9E
:106B8000225DD8A028D0000E0001D76F000ED66F6E
:106B9000100ED86F020ED96F0B0EFEECD0F0010E66
:106BA0000101A86F000E9D6F000E236F000E226F73
:106BB000000E0001B36F0A0EA26F010E9F6F410E0F
:106BC0000001F46FF00EF36F330EE82EFED7F32FB3
:106BD000FCD7F42FFAD70001B305D8B4A5D7000E1F
:106BE000CC6F000ECD6F000ECE6F000ECF6F120E69
:106BF0009AECE4F0E806D8A407D074C066F075C03B
:106C000067F0010E01013C6F000E0001CC6F000E19
:106C1000CD6F000ECE6F000ECF6F130E9AECE4F026
:106C2000E806D8A407D037C066F038C067F0010E78
:106C300001013C6F000E0001CC6F000ECD6F000E05
:106C4000CE6F000ECF6F0F0E9AECE4F0E806D8A4DA
:106C50007BD0030EB119D8A441D0390EF66EFE0ECA
:106C6000F76E000EF86E0800F550420AD8A413D053
:106C700066C0C9F067C0CAF05A0ECB6F8CEC02F048
:106C8000F36F090EF36105D00A0E6627000E672325
:106C900021D05A0E55D066C0C9F067C0CAF05A0E4E
:106CA000CB6F8CEC02F0F36F060EF36105D00A0E89
:106CB0006627000E672304D03C0E665F000E675BFC
:106CC000675104E13E0E665DD8A004D0000E676FE8
:106CD0003D0E666F010E01013C6F36D0020EB119F8
:106CE000D8A409D066C0C9F067C0CAF05A0ECB6FED
:106CF0008CEC02F0C5D7B105D8A426D066C0C9F087
:106D000067C0CAF0540ECB6F8CEC02F00009D8A417
:106D100009D066C0C9F067C0CAF05A0ECB6F8CECC0
:106D200002F0AED766C0C9F067C0CAF05A0ECB6F8A
:106D30008CEC02F0F36F020EF36101D0A5D7140EB4
:106D4000665F000E675BC6D7000E0001CC6F000EB9
:106D5000CD6F000ECE6F000ECF6F100E9AECE4F0E8
:106D6000E806D8A42CD0020EB119D8B428D0B105A9
:106D7000D8A425D066C0C9F067C0CAF0540ECB6F46
:106D80008CEC02F00009D8A413D066C0C9F067C02B
:106D9000CAF0480ECB6F8CEC02F0F36F090EF36172
:106DA00005D0640E6627000E672306D0840E01D03E
:106DB000E80E665F030E675B010E01013C6F000188
:106DC0006651335C67513458D8B007D033C066F091
:106DD00034C067F0010E01013C6F0001665167117C
:106DE000D8A407D0000E676F010E666F010E010177
:106DF0003C6F000E0001CA6F400EC96FDCEC14F04E
:106E0000E806D8A40AD0000E986F010E0101CC6FDD
:106E1000000E00017F6F000E7E6F000ECA6F400EE5
:106E2000C96F3BEC17F0E806D8A412D07F5104E1FB
:106E3000510E7E5DD8A00CD00A0EA26F010E9F6F7E
:106E4000000E0101CC6F000E00017F6F000E7E6FFF
:106E5000000ECA6F400EC96FFBEC14F0E806D8A410
:106E6000EFEFADF07F5108E1510E7E5DD8B0EFEF4E
:106E7000ADF06E0E8EEFC1F0EFEFADF0780EA2190F
:106E8000D8A483D09951D8A409D0010E996F7AC0A3
:106E900043F27BC044F2010E0101776F1E0E000128
:106EA000A619D8B404D01E0E69EC0EF0A66F485097
:106EB000D8B408D0A2C0BCF09551FDEC0AF0946F94
:106EC000010E966FA305D8A402D0010E9E6FA405F3
:106ED000D8B40CD01ED0790E07D07A0E05D0780E1B
:106EE00003D07C0E01D0810EA26F11D09551010A02
:106EF000D8B4F1D7030AD8B4F0D7010AD8B4EFD781
:106F0000070AD8B4EED7010AD8B4EDD7E8D7010EF6
:106F10009F6F000ECA6F400EC96FDCEC14F0E806DC
:106F2000D8A408D0010E0101CC6F000E00017F6FC4
:106F3000000E7E6F000ECA6F400EC96F3BEC17F05B
:106F4000E806D8A412D07F5104E1510E7E5DD8A08E
:106F50000CD00A0EA26F010E9F6F000E0101CC6FC4
:106F6000000E00017F6F000E7E6F000ECA6F400E94
:106F7000C96FFBEC14F0E806D8A4EFEFADF07F5139
:106F800002E188EFC1F0EFEFADF0790EA219D8A4BD
:106F900079D09951D8A409D0010E996F7AC043F2E3
:106FA0007BC044F2010E0101776F1E0E0001A6198D
:106FB000D8B404D01E0E69EC0EF0A66F4850D8B4B9
:106FC00008D001016B5156EC13F001016B6F010EFB
:106FD0006A6F0001A405D8A404D0780EA26F010E38
:106FE0009F6FA0C0CCF0000ECD6F000ECE6F000ED4
:106FF000CF6F140E9AECE4F0A06FA005D8A406D0D1
:10700000A2C0A1F00A0EA26F010E9F6F000ECA6F00
:10701000400EC96FDCEC14F0E806D8A408D0010ECD
:107020000101CC6F000E00017F6F000E7E6F000E1D
:10703000CA6F400EC96F3BEC17F0E806D8A412D017
:107040007F5104E1510E7E5DD8A00CD00A0EA26FD4
:10705000010E9F6F000E0101CC6F000E00017F6FCB
:10706000000E7E6F000ECA6F400EC96FFBEC14F06D
:10707000E806D8A4EFEFADF07F5102E19FEFBCF03E
:10708000EFEFADF07A0EA219D8A4D8D09951D8A4B8
:1070900009D0010E996F7AC043F27BC044F2010E11
:1070A0000101776F1E0E0001A619D8B404D01E0E80
:1070B00069EC0EF0A66F4850D8B408D0A2C0BCF05E
:1070C0009551FDEC0AF0946F010E966FA305D8A4BC
:1070D00002D0010E9E6FA405D8B408D012D0010EC4
:1070E00003D0020E01D0030EB06F0BD09551010AF0
:1070F000D8B4F5D7030AD8B4F4D7010AD8B4F3D773
:10710000EED7B051B119D8B448D0000E8F6F010E30
:1071100001015B6F010E00018D6F010E0101576FC0
:107120000001B05114ECF8F0B16F000E8B6F000E3F
:107130008A6F000E896F000E886F000E01014E6F7E
:10714000000E4D6F000E4C6F000E4B6F000E0001D5
:10715000A96F000EA86F000E4B6E000EA76F000EF9
:107160000101816F00018705D8A405D0000E01013F
:107170004A6F010E496F00018605D8A405D0000EA4
:107180000101456F010E446F00018505D8A405D0AB
:10719000000E3D6E010E0101426FA0C0CCF0000E4A
:1071A0000001CD6F000ECE6F000ECF6F140E9AEC63
:1071B000E4F0A06FA005D8A406D0A2C0A1F00A0EEA
:1071C000A26F010E9F6F000ECA6F400EC96FDCECFC
:1071D00014F0E806D8A408D0010E0101CC6F000E0F
:1071E00000017F6F000E7E6F000ECA6F400EC96FE8
:1071F0003BEC17F0E806D8A412D07F5104E1510E01
:107200007E5DD8A00CD00A0EA26F010E9F6F000EFB
:107210000101CC6F000E00017F6F000E7E6F000E2B
:10722000CA6F400EC96FFBEC14F0E806D8A4EFEF6C
:10723000ADF07F5101E183D3EFEFADF07B0EA219EA
:10724000D8A448D09951D8A409D0010E996F7AC01A
:1072500043F27BC044F2010E0101776F000E000182
:10726000CA6F400EC96FDCEC14F0E806D8A408D051
:10727000010E0101CC6F000E00017F6F000E7E6FCA
:10728000000ECA6F400EC96F3BEC17F0E806D8A499
:1072900012D07F5104E1510E7E5DD8A00CD00A0EB1
:1072A000A26F010E9F6F000E0101CC6F000E000156
:1072B0007F6F000E7E6F000ECA6F400EC96FFBEC31
:1072C00014F0E806D8A4EFEFADF07F5101E137D319
:1072D000EFEFADF07C0EA219D8A491D29951D8A4A9
:1072E00009D0010E996F7AC043F27BC044F2010EBF
:1072F0000101776F1E0E0001A619D8B404D01E0E2E
:1073000069EC0EF0A66F4850D8B408D0A2C0BCF00B
:107310009551FDEC0AF0946F010E966FA305D8A469
:1073200002D0010E9E6FA405D8B426D22CD2780EBE
:10733000A26F010E9F6F27D2000E4E6E010E4D6E92
:10734000000E596E000E5A6E13D284EC18F0000134
:10735000B351D8A48CD0070ED66FF6C0D7F0020E6A
:10736000A7EC13F0000ED76F000ED66F100ED86F7B
:10737000030ED96F0A0EFEECD0F03F0EC26FFD0E69
:10738000C36F070EC46F010EC56F010EC66F1E0ED0
:10739000C76F060EC86F000EC96F000ECA6F000ED1
:1073A000CB6F000ECC6F000ECD6FF6C0CEF0F8ECB8
:1073B000FEF03F0EC26FFD0EC36F070EC46F010ECD
:1073C000C56F010EC66F250EC76F060EC86F000E83
:1073D000C96F000ECA6F000ECB6F000ECC6F000E8F
:1073E000CD6FF6C0CEF0F8ECFEF03F0EC26FFD0E92
:1073F000C36F070EC46F010EC56F010EC66F2C0E52
:10740000C76F060EC86F000EC96F000ECA6F000E60
:10741000CB6F000ECC6F000ECD6FF6C0CEF0F8EC47
:10742000FEF03F0EC26FFD0EC36F070EC46F010E5C
:10743000C56F010EC66F330EC76F060EC86F000E04
:10744000C96F000ECA6F000ECB6F000ECC6F000E1E
:10745000CD6FF6C0CEF0F8ECFEF0000EF56F010E29
:107460000101C16F000EAD6F010E0001B36F1D0E63
:107470000101C065F8D0000EC06F0001F52BF505C5
:10748000D8A439D03F0EC26FFD0EC36F070EC46F74
:10749000010EC56F010EC66F330EC76F060EC86FA3
:1074A000000EC96F000ECA6F000ECB6F000ECC6FBE
:1074B000000ECD6FF6C0CEF0F8ECFEF03F0EC26FBE
:1074C000FD0EC36F070EC46F010EC56F020EC66FAF
:1074D0001E0EC76F060EC86F000EC96F000ECA6F72
:1074E000000ECB6F000ECC6F000ECD6FF6C0CEF04D
:1074F000F8ECFEF0B8D0020EF519D8A439D03F0E42
:10750000C26FFD0EC36F070EC46F010EC56F010E73
:10751000C66F1E0EC76F060EC86F000EC96F000E35
:10752000CA6F000ECB6F000ECC6F000ECD6FF6C091
:10753000CEF0F8ECFEF03F0EC26FFD0EC36F070EEB
:10754000C46F010EC56F020EC66F250EC76F060E03
:10755000C86F000EC96F000ECA6F000ECB6F000E11
:10756000CC6F000ECD6FF6C0CEF0F8ECFEF07BD005
:10757000030EF519D8A439D03F0EC26FFD0EC36FAC
:10758000070EC46F010EC56F010EC66F250EC76FC3
:10759000060EC86F000EC96F000ECA6F000ECB6FCB
:1075A000000ECC6F000ECD6FF6C0CEF0F8ECFEF002
:1075B0003F0EC26FFD0EC36F070EC46F010EC56F85
:1075C000020EC66F2C0EC76F060EC86F000EC96F75
:1075D000000ECA6F000ECB6F000ECC6F000ECD6F89
:1075E000F6C0CEF0F8ECFEF03ED0040EF519D8A4AB
:1075F0003AD03F0EC26FFD0EC36F070EC46F010E6F
:10760000C56F010EC66F2C0EC76F060EC86F000E39
:10761000C96F000ECA6F000ECB6F000ECC6F000E4C
:10762000CD6FF6C0CEF0F8ECFEF03F0EC26FFD0E4F
:10763000C36F070EC46F010EC56F020EC66F330E07
:10764000C76F060EC86F000EC96F000ECA6F000E1E
:10765000CB6F000ECC6F000ECD6FF6C0CEF0F8EC05
:10766000FEF0000EF56F4E04D8A448D0000E0101C4
:10767000C16F000EC06F000E236F000E226F000E50
:107680000001B36F000E4D6E000E0101AD6F000ED4
:10769000516F070E0001D66FF6C0D7F0040EA7ECAD
:1076A00013F0000ED76F000ED66F100ED86F020EBB
:1076B000D96F0C0EFEECD0F07A0E0001F46FC10E03
:1076C000F36F810EE82EFED7F32FFCD7F42FFAD7F5
:1076D00000D00A0E0001A26F010E9F6F9051D8B426
:1076E00007D0030E37ECF3F0040E37ECF3F006D0BE
:1076F000010E37ECF3F0020E37ECF3F0DC0E010173
:10770000225D050E2359D8A033D0000EC16F000EA4
:10771000C06F000E236F000E226F000E0001B36FCA
:10772000000E4D6E010E0101AD6F070E0001D66F08
:10773000F6C0D7F0040EA7EC13F0000ED76F000EC2
:10774000D66F100ED86F020ED96F0B0EFEECD0F074
:107750007A0E0001F46FC10EF36F810EE82EFED792
:10776000F32FFCD7F42FFAD700D0010E00019F6F42
:107770004D04D8A408D0E9D59551010AD8B4D7D57D
:10778000030AD8B4D9D5000E0001CA6F400EC96FE4
:10779000DCEC14F0E806D8A408D0010E0101CC6F8F
:1077A000000E00017F6F000E7E6F000ECA6F400E4C
:1077B000C96F3BEC17F0E806D8A412D07F5104E162
:1077C000510E7E5DD8A00CD00A0EA26F010E9F6FE5
:1077D000000E0101CC6F000E00017F6F000E7E6F66
:1077E000000ECA6F400EC96FFBEC14F0E806D8A477
:1077F000EFEFADF07F5101E1A2D0EFEFADF0810EE0
:10780000A219D8A4A6D09951D8A409D0010E996F75
:107810007AC043F27BC044F2010E0101776F000190
:10782000A305D8A403D0010E0101A56F0001A40592
:10783000D8A44CD00101A505D8A448D057ECEEF04F
:107840000009D8B4FBD7070E0001C46F0D0E1BEC66
:1078500016F0070E0001C46F0F0E1BEC16F0070E9A
:107860000001C46F0E0E1BEC16F0070E0001C46F72
:10787000100E1BEC16F069ECDEF0410E0001F46F07
:10788000F00EF36F330EE82EFED7F32FFCD7F42F54
:10789000FAD7020E0001C46F0D0E1BEC16F0020E9B
:1078A0000001C46F0F0E1BEC16F0030E0001C46F35
:1078B0000E0E1BEC16F0030E0001C46F100E1BEC35
:1078C00016F00A0E0001A26F010E9F6F000E00015C
:1078D000CA6F400EC96FDCEC14F0E806D8A408D0DB
:1078E000010E0101CC6F000E00017F6F000E7E6F54
:1078F000000ECA6F400EC96F3BEC17F0E806D8A423
:1079000012D07F5104E1510E7E5DD8A00CD00A0E3A
:10791000A26F010E9F6F000E0101CC6F000E0001DF
:107920007F6F000E7E6F000ECA6F400EC96FFBECBA
:1079300014F0E806D8A4EFEFADF07F5108E1510E46
:107940007E5DD8B0EFEFADF0780E8EEFC1F0EFEFC7
:10795000ADF0820EA219D8A47DD09951D8A409D037
:10796000010E996F7AC043F27BC044F2010E01010F
:10797000776F1E0E0001A619D8B404D01E0E69EC54
:107980000EF0A66F4850D8B408D0A2C0BCF09551F4
:10799000FDEC0AF0946F010E966FA305D8A402D0F7
:1079A000010E9E6FA405D8B40FD018D0830E0AD054
:1079B000840EA26F000E8F6F000E3F6E000E9A6F46
:1079C0000BD0820EA26F08D09551010AD8B4EED721
:1079D000030AD8B4EDD7F5D7010E9F6F000ECA6F1A
:1079E000400EC96FDCEC14F0E806D8A408D0010EF4
:1079F0000101CC6F000E00017F6F000E7E6F000E44
:107A0000CA6F400EC96F3BEC17F0E806D8A412D03D
:107A10007F5104E1510E7E5DD8A00CD00A0EA26FFA
:107A2000010E9F6F000E0101CC6F000E00017F6FF1
:107A3000000E7E6F000ECA6F400EC96FFBEC14F093
:107A4000E806D8A4EFEFADF07F5102E188EFC1F076
:107A5000EFEFADF0830EA219D8A419D29951D8A492
:107A600009D0010E996F7AC043F27BC044F2010E37
:107A70000101776F00018C05D8A408D0DC0EA6198F
:107A8000D8B404D0DC0E69EC0EF00AD08C51D8A426
:107A900008D01E0EA619D8B404D01E0E69EC0EF044
:107AA000A66F4850D8B419D08C05D8A40ED070C099
:107AB000BCF071C0BDF05DEC0CF0BCC070F0BDC09E
:107AC00071F0010E0101536F08D0A2C0BCF09551B6
:107AD000FDEC0AF0946F010E966F0001A305D8A487
:107AE00004D0000E986F010E9E6FA405D8A485D017
:107AF0008C51D8B46ED078D0010E8C6F000E9A6F76
:107B0000010E986F010E916F78D0B751010A0101F3
:107B1000526F52C1B7F00001B851B71901015A6F45
:107B2000010E0001916F010E9E6F000E986F65D0DF
:107B30009105D8A43ED07A51701904E17B51711996
:107B4000D8B402D0010E01D0000E9A6F70513518D2
:107B500004E171513618D8B42ED09A05D8A42BD090
:107B6000000E8B6F000E8A6F000E896F000E886FFB
:107B7000000E01014E6F000E4D6F000E4C6F000E97
:107B80004B6F00018705D8A405D0000E01014A6F94
:107B9000010E496F000E00018F6F010E01015B6F36
:107BA000010E00018D6F010E0101576F000E4F6F26
:107BB00002D0000E9A6F000E0001986F0A0EA26F9D
:107BC000010E9F6F9051D8A418D0060E37ECF3F039
:107BD00014D09551010AD8B48FD7030AD8B495D7D9
:107BE000010AD8B4A5D709D09505D8A404D0000EB1
:107BF0008C6F000E986F010E966FA0C0CCF0000E37
:107C00000001CD6F000ECE6F000ECF6F140E9AECF8
:107C1000E4F0A06FA005D8A406D0A2C0A1F00A0E7F
:107C2000A26F010E9F6F8C05D8A4D3D0000ECC6F2D
:107C3000000ECD6F000ECE6F000ECF6F120E9AECBD
:107C4000E4F0E806D8A407D074C070F075C071F0F5
:107C5000010E0101536F000E0001CC6F000ECD6FBD
:107C6000000ECE6F000ECF6F130E9AECE4F0E80614
:107C7000D8A407D037C070F038C071F0010E0101F0
:107C8000536F000E0001CC6F000ECD6F000ECE6F53
:107C9000000ECF6F0F0E9AECE4F0E806D8A45ED089
:107CA000030EB119D8B404D0020EB119D8A423D050
:107CB00070C0C9F071C0CAF05A0ECB6F8CEC02F0E4
:107CC000F36F060EF36105D00A0E7027000E7123C4
:107CD00004D03C0E705F000E715B715104E13E0EEA
:107CE000705DD8A004D0000E716F3D0E706F010E54
:107CF0000101536F33D0B105D8A430D070C0C9F0A2
:107D000071C0CAF0540ECB6F8CEC02F00009D8A4FD
:107D100013D070C0C9F071C0CAF05A0ECB6F8CEC92
:107D200002F0F36F090EF36105D00A0E7027000E02
:107D30007123DDD75A0E0ED070C0C9F071C0CAF0E1
:107D40005A0ECB6F8CEC02F0F36F020EF36101D090
:107D5000ECD7140E705F000E715BC9D7000E0001E6
:107D6000CC6F000ECD6F000ECE6F000ECF6F100ED9
:107D70009AECE4F0E806D8A42CD0020EB119D8B4DD
:107D800028D0B105D8A425D070C0C9F071C0CAF000
:107D9000540ECB6F8CEC02F00009D8A413D070C045
:107DA000C9F071C0CAF0480ECB6F8CEC02F0F36FD3
:107DB000090EF36105D0640E7027000E712306D002
:107DC000840E01D0E80E705F030E715B010E01019D
:107DD000536F0001705101010A5D000171510101F1
:107DE0000B59D8B006D00AC170F00BC171F0010E6A
:107DF000536F000170517111D8A407D0000E716F3C
:107E0000010E706F010E0101536F000E0001CA6F69
:107E1000400EC96FDCEC14F0E806D8A40ED0000EBA
:107E2000986F010E0101CC6F000E00017F6F000EF4
:107E30007E6F000E9A6F000E8C6F000ECA6F400EA0
:107E4000C96F3BEC17F0E806D8A412D07F5104E1CB
:107E5000510E7E5DD8A00CD00A0EA26F010E9F6F4E
:107E6000000E0101CC6F000E00017F6F000E7E6FCF
:107E7000000ECA6F400EC96FFBEC14F0E806D8A4E0
:107E8000EFEFADF07F5101E1F1D1EFEFADF0840EF6
:107E9000A219D8A4F4D19951D8A409D0010E996F90
:107EA0007AC043F27BC044F2010E0101776F0001FA
:107EB0008305D8B403D08205D8A408D0C80EA6196B
:107EC000D8B404D0C80E69EC0EF007D01E0EA61967
:107ED000D8B404D01E0E69EC0EF0A66F4850D8B48A
:107EE00030D08351D8A40CD08251D8A409D0A2C0DC
:107EF000BCF09551FDEC0AF0946F010E966F21D005
:107F00008305D8A40ED031C0BCF032C0BDF05DEC0A
:107F10000CF0BCC031F0BDC032F0010E0101406F69
:107F200010D08205D8A40DD02FC0BCF030C0BDF059
:107F30005DEC0CF0BCC02FF0BDC030F0010E0101B3
:107F40003F6F0001A305D8A404D0000E986F010E66
:107F50009E6FA405D8A4A5D08351D8A49AD08251ED
:107F6000D8B458D096D0010E836F000E826F04D023
:107F7000010E826F000E836F010E986F92D08451B4
:107F8000D8A425D0AF51D8A403D0AE51D8B43ED098
:107F9000010E0101B76F000E00018D6F000E8E6F94
:107FA000000E8F6F000E3F6E000E0101596F000E24
:107FB0000001B86F06C176F007C177F006C178F00E
:107FC00007C179F0010E3C6E010E846F1FD03C0496
:107FD000D8B41CD0000E846F000E0101B76F000EE4
:107FE0001F6F000E1E6F010E00018D6F010E8E6F50
:107FF000000E8F6F000E3F6E000E0101596F000ED4
:108000000001B86F0A0EA26F010E9F6F010E0001F2
:10801000966F47D09551010AD8B4A5D7030AD8B4B2
:10802000A7D7010AD8B4ABD73CD0000E836F31C0BC
:1080300006F132C007F101010451065D05510759EF
:10804000D8A0E4D7010E31242F6E000E3220306EFE
:108050002FC004F130C005F1010E3F6FD7D7000EDD
:10806000826F2FC004F130C005F101010451065D9B
:1080700005510759D8A0CAD7FF0E2F24316EFF0E25
:108080003020326E31C006F132C007F1010E406F70
:10809000BDD79551010AD8B4C8D7030AD8B4DFD7E1
:1080A000B5D7AF51D8A403D0AE51D8B492D084057F
:1080B000D8A47DD03C04D8A412D001011F5104E102
:1080C0000A0E1E5DD8A00BD0000E1F6F000E1E6F93
:1080D000020E3C6E0C0E00018F6F0C0E2FD0020EA4
:1080E0003C18D8A416D001011F5104E1640E1E5D96
:1080F000D8A00FD0000E1F6F000E1E6F030E3C6E37
:10810000010E596F010E0001B86F080E8F6F080E37
:1081100015D0030E3C18D8A413D001011F5104E15F
:108120008C0E1E5DD8A00CD0000E1F6F000E1E6FAF
:10813000040E3C6E000E00018F6F000E3F6E37D0B4
:10814000040E3C18D8A433D001011F5104E1280EBD
:108150001E5DD8A02CD0000E1F6F000E1E6F000EEB
:10816000596F000E0001B86F010104510001785DE4
:108170000101055100017959D8B009D0010E3C6EBA
:10818000764B772B76C078F077C079F010D0000E60
:10819000846F000E0101B76F000E1F6F000E1E6F7F
:1081A000010E00018D6F010E8E6F010E966F0001A2
:1081B0007A510201431906E100017B510201441981
:1081C000D8B407D07AC043F27BC044F2010E01015B
:1081D000776F000E0001CA6F400EC96FDCEC14F01F
:1081E000E806D8A41CD0000E846F000E0101B76F02
:1081F000000E1F6F000E1E6F000E00018F6F000E2D
:108200003F6E000E826F000E836F000E986F010E9E
:108210000101CC6F000E00017F6F000E7E6F000E1B
:10822000CA6F400EC96F3BEC17F0E806D8A412D015
:108230007F5104E1510E7E5DD8A00CD00A0EA26FD2
:10824000010E9F6F000E0101CC6F000E00017F6FC9
:10825000000E7E6F000ECA6F400EC96FFBEC14F06B
:10826000E806D8A4EFEFADF07F5107E1510E7E5D37
:10827000D8B0EFEFADF0820E51D0EFEFADF06D0E54
:10828000A219D8A458D09951D8A409D0010E996F39
:108290007AC043F27BC044F2010E0101776F000EF9
:1082A0000001CA6F400EC96FDCEC14F0E806D8A4D8
:1082B00008D0010E0101CC6F000E00017F6F000E8F
:1082C0007E6F000ECA6F400EC96F3BEC17F0E806D8
:1082D000D8A412D07F5104E1510E7E5DD8A00CD0FD
:1082E0000A0EA26F010E9F6F000E0101CC6F000EEF
:1082F00000017F6F000E7E6F000ECA6F400EC96FC7
:10830000FBEC14F0E806D8A4EFEFADF07F5111E1DB
:10831000510E7E5DD8B0EFEFADF0640EA26F010E8E
:108320009F6F000E0101CC6F000E00017F6F000EE9
:108330007E6FEFEFADF0A205D8A488D00F0E926F3C
:10834000000ECA6F800EC96F3BEC17F0506E020131
:10835000685104E18C0E675DD8A027D05050D8A496
:1083600024D0000E0101BF6F000E0201686F000EE5
:10837000676F0A0E0001A26F010E9F6F000EBD6FA6
:10838000070EBC6F27EC18F05A0AD8A408D0000ECC
:108390000001BD6F080EBC6F27EC18F001D00D0E68
:1083A0000001926F010E0101AE6F00018005D8A49B
:1083B00006D0A2C0A1F0030EA26F010E9F6F000EA7
:1083C000CA6F400EC96FDCEC14F0E806D8A408D0E0
:1083D000010E0101CC6F000E00017F6F000E7E6F59
:1083E000000ECA6F400EC96F3BEC17F0E806D8A428
:1083F00010D07F5104E1320E7E5DD8A00AD0040E69
:10840000A26F0A0EA16F010E9F6F000E7F6F630EA9
:108410007E6F000ECA6F400EC96FFBEC14F0E806C9
:10842000D8A46DD17F5103E1320E7E5DD8B067D103
:10843000000E0101CC6F000E00017F6F000E7E6FF9
:10844000000E0201686F8C0E676F59D1030EA219DE
:10845000D8A42ED001012C5140080001C26F0101A7
:108460002D51D8A0E82A01080001C36F000EC56F86
:10847000640EC46F2DEC13F0C251446E01017251B1
:108480004418D8B402D0010E716F00018051D8A4F5
:1084900036D18105D8A433D1A251A119D8A403D0D3
:1084A0000A0EA26F02D0A1C0A2F0010E9F6F27D1C9
:1084B000040EA219D8A447D07E514008C26F7F5144
:1084C000D8A0E82A0108C36F000EC56F640EC46F00
:1084D0002DEC13F0C251936F0101705100019319FB
:1084E000D8B409D0410E7E5D010E7F59D8B003D0BB
:1084F000010E01016F6F000E0001CA6F400EC96FBF
:108500003BEC17F0E806D8A40FD0400E7E5D010EBC
:108510007F59D8B004D008D01BECFCF04F6E4F5000
:10852000D8B4FAD7C1EC18F0000E0001CA6F400EA3
:10853000C96FFBEC14F0E806D8A4E1D0A251A11950
:10854000D8B4AED7B0D7050EA219D8A499D00B0EC7
:10855000CB6FB80ECA6F97EC0FF001015C51D8B425
:1085600003D05D05D8A40CD00001A251A119D8A454
:1085700003D00A0EA26F02D0A1C0A2F0010E9F6F1D
:10858000000E0001CA6F100EC96FDCEC14F0E80693
:10859000D8B409D0000ECA6F100EC96FFBEC14F0EE
:1085A000E806D8A40CD0A9C0CCF092C1CDF085C10A
:1085B000CEF0000ECF6F0A0E9AECE4F0A96F000E19
:1085C000CA6F200EC96FDCEC14F0E806D8B409D0ED
:1085D000000ECA6F200EC96FFBEC14F0E806D8A499
:1085E0000CD0A8C0CCF091C1CDF084C1CEF0000E6B
:1085F000CF6F0B0E9AECE4F0A86F8005D8A406D0DC
:10860000A2C0A1F0030EA26F010E9F6F000ECA6FF1
:10861000400EC96FDCEC14F0E806D8A408D0010EB7
:108620000101CC6F000E00017F6F000E7E6F000E07
:10863000CA6F400EC96F3BEC17F0E806D8A410D003
:108640007F5104E1320E7E5DD8A00AD0A2C0A1F015
:10865000040EA26F010E9F6F000E7F6F630E7E6F80
:10866000000ECA6F400EC96FFBEC14F0E806D8A4E8
:1086700046D07F5144E1320E7E5DD8A0D9D63FD09E
:10868000060EA219D8A43BD0E00E0101205D2E0EEB
:108690002159D8A032D02F0E205D310E2159D8B0EB
:1086A00013D020512E080001C26F01012151D8A022
:1086B000E82A31080001C36F000EC56F640EC46F55
:1086C0002DEC13F0C251426E010169514218D8B429
:1086D00002D0010E686F6951D8A411D04250D8A4BD
:1086E0000ED04EECFEF003D01BECFCF04F6E4F5062
:1086F000D8B4FAD7C1EC18F002D000011FD700019E
:10870000A25188ECC3F0A25100EC80F0ADEFA9F0CB
:10871000DC6F3B50D8A431D06E0E0001DC19D8B408
:1087200020D06F0EDC19D8B41CD0700EDC19D8B470
:1087300018D0780EDC19D8B414D0790EDC19D8B45E
:1087400010D07A0EDC19D8B40CD07B0EDC19D8B45A
:1087500008D07C0EDC19D8B404D0810EDC19D8A462
:1087600006D04AC0CCF0020EF3ECE9F00BD04AC0C0
:10877000CCF0010EF3ECE9F005D04AC0CCF0030ECA
:10878000F3ECE9F00A0E0001A219D8A4B7D2AA515D
:10879000D8A47CD1B005D8A47BD08BC0CCF018C1B4
:1087A000CDF019C1CEF0020ED06F020ECF6F040EC5
:1087B000D26F040ED16F010E09ECDCF0CCC018F1C1
:1087C000CDC019F18AC0CCF016C1CDF017C1CEF0E2
:1087D000020ED06F020ECF6F040ED26F040ED16F57
:1087E000020E09ECDCF0CCC016F1CDC017F189C047
:1087F000CCF014C1CDF015C1CEF0020ED06F020E38
:10880000CF6F040ED26F040ED16F030E09ECDCF0B3
:10881000CCC014F1CDC015F188C0CCF012C1CDF0A0
:1088200013C1CEF0020ED06F020ECF6F040ED26FC6
:10883000040ED16F040E09ECDCF0CCC012F1CDC0F7
:1088400013F1A9C0CCF010C1CDF011C1CEF0020ED1
:10885000D06F020ECF6F040ED26F040ED16F050ED3
:1088600009ECDCF0CCC010F1CDC011F1A8C0CCF007
:108870000EC1CDF00FC1CEF0020ED06F020ECF6F41
:10888000040ED26F040ED16F060E09ECDCF0D1D1CC
:10889000020EB019D8A47BD08BC0CCF018C1CDF09B
:1088A00019C1CEF0020ED06F020ECF6F040ED26F40
:1088B000040ED16F010E09ECDCF0CCC018F1CDC074
:1088C00019F18AC0CCF016C1CDF017C1CEF0020E5E
:1088D000D06F020ECF6F040ED26F040ED16F020E56
:1088E00009ECDCF0CCC016F1CDC017F189C0CCF09A
:1088F00014C1CDF015C1CEF0020ED06F020ECF6FB5
:10890000040ED26F040ED16F030E09ECDCF0CCC064
:1089100014F1CDC015F188C0CCF012C1CDF013C157
:10892000CEF0020ED06F020ECF6F040ED26F040E87
:10893000D16F040E09ECDCF0CCC012F1CDC013F104
:10894000A9C0CCF010C1CDF011C1CEF0020ED06F95
:10895000020ECF6F040ED26F040ED16F050E09EC1C
:10896000DCF0CCC010F1CDC011F1A8C0CCF00EC12C
:10897000CDF00FC1CEF0020ED06F020ECF6F100EF1
:10898000D26F100ED16F060E09ECDCF052D1030E3F
:10899000B019D8A452D18BC0CCF018C1CDF019C1F8
:1089A000CEF0020ED06F020ECF6F040ED26F040E07
:1089B000D16F010E09ECDCF0CCC018F1CDC019F17B
:1089C0008AC0CCF016C1CDF017C1CEF0020ED06F28
:1089D000020ECF6F040ED26F040ED16F020E09EC9F
:1089E000DCF0CCC016F1CDC017F189C0CCF014C1B9
:1089F000CDF015C1CEF0020ED06F020ECF6F040E77
:108A0000D26F040ED16F030E09ECDCF0CCC014F170
:108A1000CDC015F188C0CCF012C1CDF013C1CEF09D
:108A2000020ED06F020ECF6F100ED26F100ED16FEC
:108A3000040E09ECDCF0CCC012F1CDC013F1A9C0DA
:108A4000CCF010C1CDF011C1CEF0020ED06F020EED
:108A5000CF6F040ED26F040ED16F050E09ECDCF05F
:108A6000CCC010F1CDC011F1A8C0CCF00EC1CDF03A
:108A70000FC1CEF0020ED06F020ECF6F040ED26F78
:108A8000040ED16F060E09ECDCF0D3D0B005D8A4EB
:108A90007BD04EC1CCF018C1CDF019C1CEF0020E82
:108AA000D06F020ECF6F040ED26F040ED16F010E85
:108AB00009ECDCF0CCC018F1CDC019F14DC1CCF0FF
:108AC00016C1CDF017C1CEF0020ED06F020ECF6FDF
:108AD000040ED26F040ED16F020E09ECDCF0CCC094
:108AE00016F1CDC017F14CC1CCF014C1CDF015C1B9
:108AF000CEF0020ED06F020ECF6F040ED26F040EB6
:108B0000D16F030E09ECDCF0CCC014F1CDC015F12F
:108B10004BC1CCF012C1CDF013C1CEF0020ED06F1C
:108B2000020ECF6F040ED26F040ED16F040E09EC4B
:108B3000DCF0CCC012F1CDC013F14BC0CCF010C1B1
:108B4000CDF011C1CEF0020ED06F020ECF6F040E29
:108B5000D26F040ED16F050E09ECDCF0CCC010F121
:108B6000CDC011F1A7C0CCF00EC1CDF00FC1CEF039
:108B7000020ED06F020ECF6F100ED26F100ED16F9B
:108B8000060E09ECDCF055D0020EB019D8A427D09F
:108B90004BC0CCF010C1CDF011C1CEF0020ED06FA1
:108BA000020ECF6F040ED26F040ED16F050E09ECCA
:108BB000DCF0CCC010F1CDC011F1A7C0CCF00EC1DB
:108BC000CDF00FC1CEF0020ED06F020ECF6F040EAB
:108BD000D26F040ED16F060E09ECDCF02AD0030E22
:108BE000B019D8A42AD04BC0CCF010C1CDF011C11F
:108BF000CEF0020ED06F020ECF6F040ED26F040EB5
:108C0000D16F050E09ECDCF0CCC010F1CDC011F134
:108C1000A7C0CCF00EC1CDF00FC1CEF0020ED06FC8
:108C2000020ECF6F040ED26F040ED16F060E09EC48
:108C3000DCF0CCC00EF1CDC00FF1AAC0CCF04BC21D
:108C4000CDF04CC2CEF0020ED06F020ECF6F040EEC
:108C5000D26F040ED16F0A0E09ECDCF0CCC04BF2DF
:108C6000CDC04CF280C1CCF04DC2CDF04EC2CEF0A2
:108C7000020ED06F020ECF6F040ED26F040ED16FB2
:108C8000080E09ECDCF0CCC04DF2CDC04EF2010173
:108C90004851D8A41CD0000E0001CA6F400EC96F05
:108CA0003BEC17F0CC6F7CC0CDF07DC0CEF0020E57
:108CB000D06F020ECF6F040ED26F040ED16F070E6D
:108CC00009ECDCF0CCC07CF0CDC07DF0120048C1D6
:108CD000CCF07CC0CDF07DC0CEF0020E0001D06F94
:108CE000020ECF6F200ED26F200ED16F070E09EC4F
:108CF000DCF0CCC07CF0CDC07DF01200040EDC199D
:108D0000D8A41BD0000ECA6F400EC96F3BEC17F001
:108D1000CC6F7CC0CDF07DC0CEF0020ED06F020EC5
:108D2000CF6F100ED26F100ED16F070E09ECDCF072
:108D3000CCC07CF0CDC07DF012006D0EA219D8A47D
:108D40001BD0000ECA6F400EC96F3BEC17F0CC6F02
:108D50007CC0CDF07DC0CEF0020ED06F020ECF6F82
:108D6000040ED26F040ED16F070E09ECDCF0CCC0FC
:108D70007CF0CDC07DF01200780EA219D8A41BD0D3
:108D8000000ECA6F400EC96F3BEC17F0CC6F7CC071
:108D9000CDF07DC0CEF0020ED06F020ECF6F040E6C
:108DA000D26F040ED16F070E09ECDCF0CCC07CF062
:108DB000CDC07DF01200700EA219D8A41BD0000EF9
:108DC000CA6F400EC96F3BEC17F0CC6F7CC0CDF082
:108DD0007DC0CEF0020ED06F020ECF6F040ED26FA8
:108DE000040ED16F070E09ECDCF0CCC07CF0CDC0D6
:108DF0007DF012006F0EA219D8A41BD0000ECA6F0E
:108E0000400EC96F3BEC17F0CC6F7CC0CDF07DC03D
:108E1000CEF0020ED06F020ECF6F040ED26F040E92
:108E2000D16F070E09ECDCF0CCC07CF0CDC07DF03A
:108E300012006E0EA219D8A41BD0000ECA6F400EED
:108E4000C96F3BEC17F0CC6F7CC0CDF07DC0CEF08D
:108E5000020ED06F020ECF6F040ED26F040ED16FD0
:108E6000070E09ECDCF0CCC07CF0CDC07DF0120028
:108E7000830EA219D8A41BD0000ECA6F400EC96F72
:108E80003BEC17F0CC6F7CC0CDF07DC0CEF0020E75
:108E9000D06F020ECF6F040ED26F040ED16F070E8B
:108EA00009ECDCF0CCC07CF0CDC07DF01200650E8A
:108EB000A219D8A41BD0000ECA6F400EC96F3BEC9C
:108EC00017F0CC6F7CC0CDF07DC0CEF0020ED06F1D
:108ED000020ECF6F040ED26F040ED16F070E09EC95
:108EE000DCF0CCC07CF0CDC07DF01200640EA21985
:108EF000D8A41BD0000ECA6F400EC96F3BEC17F010
:108F0000CC6F7CC0CDF07DC0CEF0020ED06F020ED3
:108F1000CF6F040ED26F040ED16F070E09ECDCF098
:108F2000CCC07CF0CDC07DF012000B0EA219D8A4ED
:108F30001BD0000ECA6F400EC96F3BEC17F0CC6F10
:108F40007CC0CDF07DC0CEF0020ED06F020ECF6F90
:108F5000040ED26F040ED16F070E09ECDCF0CCC00A
:108F60007CF0CDC07DF01200820EA219D8A41BD0D7
:108F7000000ECA6F400EC96F3BEC17F0CC6F7CC07F
:108F8000CDF07DC0CEF0020ED06F020ECF6F040E7A
:108F9000D26F040ED16F070E09ECDCF0CCC07CF070
:108FA000CDC07DF01200840EA219D8A41200000ECC
:108FB000CA6F400EC96F3BEC17F0CC6F7CC0CDF090
:108FC0007DC0CEF0020ED06F020ECF6F040ED26FB6
:108FD000040ED16F070E09ECDCF0CCC07CF0CDC0E4
:108FE0007DF0120000017651D61906E17751D719AC
:108FF000D8A402D0000E08D07051D61906E17151E4
:10900000D719D8A402D0010EDD6F040ED75DD8A009
:1090100004D0030ED76FD66908D0D651D711D8A483
:1090200004D0000ED76F010ED66FD6C0C2F0D7C0E5
:10903000C3F0030EC56FE80EC46F2DEC13F0C251E0
:10904000100FD86F030EBF6FE80EBE6FD6C0BCF016
:10905000D7C0BDF07CEC14F0BCC0C2F0BDC0C3F002
:10906000000EC56F640EC46F2DEC13F0C251100FCB
:10907000D96F000EBF6F640EBE6FD6C0BCF0D7C0F4
:10908000BDF07CEC14F0BCC0C2F0BDC0C3F0000E5B
:10909000C56F0A0EC46F2DEC13F0C251100FDA6FBA
:1090A000D6C0BCF0D7C0BDF0000EBF6F0A0EBE6FB9
:1090B0007CEC14F0BC51100FDB6F4504D8B404D025
:1090C00001017551D8A429D200019A05D8A425D24E
:1090D000E80ED65D030ED759D8A07DD0600EC26FC2
:1090E000E50EC36F070EC46F020EC56FD8C0C6F081
:1090F000000EC76FDD51020DF350030FC86F000E55
:10910000C96F000ECA6F000ECB6F000ECC6F000E41
:10911000CD6FF6C0CEF0F8ECFEF0600EC26FE50E3B
:10912000C36F070EC46F020EC56FD9C0C6F0090E1B
:10913000C76FDD51020DF350030FC86F000EC96FEA
:10914000000ECA6F000ECB6F000ECC6F000ECD6FFD
:10915000F6C0CEF0F8ECFEF0600EC26FE50EC36F05
:10916000070EC46F020EC56FDAC0C6F0120EC76FCD
:10917000DD51020DF350030FC86F000EC96F000ED2
:10918000CA6F000ECB6F000ECC6F000ECD6FF6C015
:10919000CEF0F8ECFEF0600EC26FE50EC36F070E66
:1091A000C46F020EC56FDBC0C6F01A0EC76FDD516B
:1091B000020DF350030FC86F000EC96F000ECA6F87
:1091C000000ECB6F000ECC6F000ECD6FF6C0CEF050
:1091D000F8ECFEF01200D75104E1640ED65DD8A081
:1091E0009CD0600EC26FE50EC36F070EC46F020EF7
:1091F000C56F000EC66F000EC76FDD51020DF35034
:10920000030FC86F000EC96F000ECA6F000ECB6F40
:10921000000ECC6F000ECD6FF6C0CEF0F8ECFEF075
:10922000600EC26FE50EC36F070EC46F020EC56FEE
:10923000D9C0C6F0000EC76FDD51020DF350030F09
:10924000C86F000EC96F000ECA6F000ECB6F000E04
:10925000CC6F000ECD6FF6C0CEF0F8ECFEF0600ED5
:10926000C26FE50EC36F070EC46F020EC56FDAC082
:10927000C6F0090EC76FDD51020DF350030FC86F22
:10928000000EC96F000ECA6F000ECB6F000ECC6FC0
:10929000000ECD6FF6C0CEF0F8ECFEF0600EC26F9F
:1092A000E50EC36F070EC46F020EC56FDBC0C6F0BC
:1092B000120EC76FDD51020DF350030FC86F000E81
:1092C000C96F000ECA6F000ECB6F000ECC6F000E80
:1092D000CD6FF6C0CEF0F8ECFEF0600EC26FE50E7A
:1092E000C36F070EC46F020EC56F000EC66F1A0E55
:1092F000C76FDD51020DF350030FC86F000EC96F29
:10930000000ECA6F000ECB6F000ECC6F000ECD6F3B
:10931000F6C0CEF0F8ECFEF01200D75104E10A0ED0
:10932000D65DD8A07DD0600EC26FE50EC36F070E6C
:10933000C46F020EC56F000EC66F000EC76FDD5101
:10934000020DF350030FC86F000EC96F000ECA6FF5
:10935000000ECB6F000ECC6F000ECD6FF6C0CEF0BE
:10936000F8ECFEF0600EC26FE50EC36F070EC46F1F
:10937000020EC56FDAC0C6F0090EC76FDD51020DCF
:10938000F350030FC86F000EC96F000ECA6F000EB6
:10939000CB6F000ECC6F000ECD6FF6C0CEF0F8ECA8
:1093A000FEF0600EC26FE50EC36F070EC46F020EB3
:1093B000C56FDBC0C6F0120EC76FDD51020DF35052
:1093C000030FC86F000EC96F000ECA6F000ECB6F7F
:1093D000000ECC6F000ECD6FF6C0CEF0F8ECFEF0B4
:1093E000600EC26FE50EC36F070EC46F020EC56F2D
:1093F000000EC66F1A0EC76FDD51020DF350030F3A
:10940000C86F000EC96F000ECA6F000ECB6F000E42
:10941000CC6F000ECD6FF6C0CEF0F8ECFEF012006F
:10942000600EC26FE50EC36F070EC46F020EC56FEC
:10943000000EC66F000EC76FDD51020DF350030F13
:10944000C86F000EC96F000ECA6F000ECB6F000E02
:10945000CC6F000ECD6FF6C0CEF0F8ECFEF0600ED3
:10946000C26FE50EC36F070EC46F020EC56F000E0C
:10947000C66F090EC76FDD51020DF350030FC86FA1
:10948000000EC96F000ECA6F000ECB6F000ECC6FBE
:10949000000ECD6FF6C0CEF0F8ECFEF0600EC26F9D
:1094A000E50EC36F070EC46F020EC56FDBC0C6F0BA
:1094B000120EC76FDD51020DF350030FC86F000E7F
:1094C000C96F000ECA6F000ECB6F000ECC6F000E7E
:1094D000CD6FF6C0CEF0F8ECFEF0600EC26FE50E78
:1094E000C36F070EC46F020EC56F000EC66F1A0E53
:1094F000C76FDD51020DF350030FC86F000EC96F27
:10950000000ECA6F000ECB6F000ECC6F000ECD6F39
:10951000F6C0CEF0F8ECFEF01200600E0001C26F53
:10952000E50EC36F070EC46F020EC56F000EC66F47
:10953000000EC76FDD51020DF350030FC86F000E10
:10954000C96F000ECA6F000ECB6F000ECC6F000EFD
:10955000CD6FF6C0CEF0F8ECFEF0600EC26FE50EF7
:10956000C36F070EC46F020EC56F000EC66F090EE3
:10957000C76FDD51020DF350030FC86F000EC96FA6
:10958000000ECA6F000ECB6F000ECC6F000ECD6FB9
:10959000F6C0CEF0F8ECFEF0600EC26FE50EC36FC1
:1095A000070EC46F020EC56F000EC66F120EC76F96
:1095B000DD51020DF350030FC86F000EC96F000E8E
:1095C000CA6F000ECB6F000ECC6F000ECD6FF6C0D1
:1095D000CEF0F8ECFEF0600EC26FE50EC36F070E22
:1095E000C46F020EC56F000EC66F1A0EC76FDD5135
:1095F000020DF350030FC86F000EC96F000ECA6F43
:10960000000ECB6F000ECC6F000ECD6FF6C0CEF00B
:10961000F8ECFEF01200D841E8423F0B030D6F005A
:10962000CCFFDFF0DA05D8A458D0690EC26FFC0E6B
:10963000C36FDF516608C46F010EC56F000EC66FA1
:10964000DFC0C7F0D9C0C8F0000EC96F000ECA6FE6
:10965000010ECB6F000ECC6F000ECD6FF6C0CEF0BA
:10966000F8ECFEF0690EC26FFC0EC36FDF516608A6
:10967000C46F010EC56F000EC66FDFC0C7F0D929D9
:10968000C86F000EC96F000ECA6F010ECB6F000EBF
:10969000CC6F000ECD6FF6C0CEF0F8ECFEF0690E88
:1096A000C26FFC0EC36FDF516608C46F010EC56F39
:1096B000000EC66FDFC0C7F0D951020FC86F000E91
:1096C000C96F000ECA6F010ECB6F000ECC6F000E7B
:1096D000CD6FF6C0CEF0F8ECFEF0040ED75DD8A04A
:1096E00004D0030ED76FD66908D0D651D711D8A4AD
:1096F00004D0000ED76F010ED66FD6C0C2F0D7C00F
:10970000C3F0030EC56FE80EC46F2DEC13F0C25109
:10971000DB6F030EBF6FE80EBE6FD6C0BCF0D7C0C4
:10972000BDF07CEC14F0BCC0C2F0BDC0C3F0000EB4
:10973000C56F640EC46F2DEC13F0C251DC6F000EC8
:10974000BF6F640EBE6FD6C0BCF0D7C0BDF07CEC5E
:1097500014F0BCC0C2F0BDC0C3F0000EC56F0A0E4D
:10976000C46F2DEC13F0C251DD6FD6C0BCF0D7C072
:10977000BDF0000EBF6F0A0EBE6F7CEC14F0BC5142
:10978000DE6F9705D8B403D09851D8A4FED1E80E67
:10979000D65D030ED759D8A074D0420EC26FF10E19
:1097A000C36F0A0EC46F030EC56FDBC0C6F0D8C00E
:1097B000C7F0D9C0C8F0000EC96F000ECA6FDAC07A
:1097C000CBF0000ECC6F000ECD6FF6C0CEF0F8ECF3
:1097D000FEF0420EC26FF10EC36F0A0EC46F030E8D
:1097E000C56FDCC0C6F0D8510D0FC76FD9C0C8F027
:1097F000000EC96F000ECA6FDAC0CBF0000ECC6F3E
:10980000000ECD6FF6C0CEF0F8ECFEF0420EC26F47
:10981000F10EC36F0A0EC46F030EC56FDDC0C6F034
:10982000D8511A0FC76FD9C0C8F0000EC96F000E0B
:10983000CA6FDAC0CBF0000ECC6F000ECD6FF6C051
:10984000CEF0F8ECFEF0420EC26FF10EC36F0A0EBE
:10985000C46F030EC56FDEC0C6F0D851260FC76FA8
:10986000D9C0C8F0000EC96F000ECA6FDAC0CBF0C5
:10987000000ECC6F000ECD6FF6C0CEF0F8ECFEF00F
:109880001200D75104E1640ED65DD8A090D0420EEC
